:100000000C944B2E0C9450310C947B310C94A631F3
:100010000C94D1310C94FC310C9427320C94523254
:100020000C947D320C947C2E0C947C2E0C947C2EA3
:100030000C947C2E0C947C2E0C947C2E0C947C2E98
:100040000C947C2E0C9461C50C947C2E0C947C2E0C
:100050000C947C2E0C947C2E0C946DB80C947E2EFB
:100060000C947C2E0C94DAA30C9486A40C947C2E15
:100070000C947C2E0C947C2E0C947C2E0C947C2E58
:100080000C947C2E0C947C2E0C947C2E0C947C2E48
:100090000C947C2E0C947C2E0C947C2E0C947C2E38
:1000A0000C947C2E0C947C2E0C947C2E0C947C2E28
:1000B0000C947C2E0C947C2E0C947C2E0C947C2E18
:1000C0000C947C2E0C947C2E0C947C2E0C947C2E08
:1000D0000C947C2E0C947C2E0C947C2E0C947C2EF8
:1000E0000C947C2EC62FCB2FD02FDA2FE42F5D302F
:1000F000EE2FF62FFE2F083012301C302B3035300B
:100100005D303F3049305330813084307330773048
:100110007D30BB3088308C30923096309A30A030B1
:10012000A430A830BB30AE30B230B6300566E565DD
:10013000EB65E865EE65F165F4650066F7651266E6
:10014000FA65FD6515A113A137A134A132A169A1FA
:1001500066A164A1C2A190A18DA18BA10DA413A43D
:1001600024A42FA437A44CA43BA44CA43FA443A490
:100170004CA449A4084AD73B3BCE016E84BCBFFDCA
:10018000C12F3D6C74319ABD56833DDA3D00C77F67
:1001900011BED9E4BB4C3E916BAAAABE0000008000
:1001A0003F05A84CCDB2D44EB93836A9020C50B98F
:1001B000918688083CA6AAAA2ABE000000803F00BB
:1001C0000D9483010D94873D0D943F4C0D94315156
:1001D0004E414E494E495459494E46CDCCCC3D0A2C
:1001E000D7233C17B7D13877CC2B329595E6241F0F
:1001F000B14F0A000020410000C84200401C4620C8
:10020000BCBE4CCA1B0E5AAEC59D7400000A0B0240
:10021000090C0D0E08070304010000000000000097
:1002200000000000000000000000000000000000CE
:10023000000000000000001211100000000000008B
:1002400000000000000000000000000000000000AE
:1002500000010210202008081020401020408002D9
:1002600001020108040201010204081020408080FC
:100270004020100804020180040201804020100880
:100280000402010804020101020408102040800158
:100290000204081020408005050505070508080828
:1002A00008020202020A0A08080404040401010107
:1002B000010101010103030303030303030407070F
:1002C000070C0C0C0C0C0C0C0C02020202060606AD
:1002D00006060606060B0B0B0B0B0B0B0B00002088
:1002E000002300260029002C002F0032000001000E
:1002F0000003010601090100002200250028002B4F
:10030000002E003100340002010000050108010B3D
:100310000100002100240027002A002D00300033B6
:100320000001010000040107010A0101060D00FEA1
:1003300009016602D620FFFE0BFE0AFE0D006022B8
:100340001969808080808080800080183363A0A03D
:10035000A00357675050F850F85050025969207860
:10036000A0A0702828F02002596948A85010204009
:1003700050A89002586840A0A040A0989068281308
:1003800063808080113B6B20404080808080804073
:100390004020113B6B8040402020202020404080A6
:1003A00006556520A870A8200455652020F8202057
:1003B000113363604080065161F811336340E040BF
:1003C00002596908081010204040808002596920B5
:1003D00050888888888850200259692060A0202091
:1003E000202020F80259697088880810204080F881
:1003F000025969F8081020700808887002596910BD
:100400001030505090F81010025969F88080B0C830
:100410000808887002596970888080F08888887020
:10042000025969F8081010202040404002596970B4
:100430008888887088888870025969708888887868
:100440000808887011386840E040000040E0401122
:10045000386840E040000060408002596908102080
:10046000408040201008045464F80000F8025969E4
:100470008040201008102040800259697088880848
:10048000102020002002596970888898A8A8B080A0
:10049000780259692050888888F8888888025969C4
:1004A000F048484870484848F00259697088808090
:1004B0008080808870025969F04848484848484818
:1004C000F0025969F8808080F0808080F8025969D4
:1004D000F8808080F08080808002596970888080F8
:1004E000809888887002596988888888F888888800
:1004F00088123969E040404040404040E00259697C
:10050000381010101010109060025969888890A05F
:10051000C0A0908888025969808080808080808017
:10052000F80259698888D8A8A888888888025969F3
:1005300088C8C8A8A8989888880259697088888847
:100540008888888870025969F0888888F08080805F
:1005500080015A6A70888888888888A8700802593B
:1005600069F0888888F0A09088880259697088802E
:10057000807008088870025969F820202020202007
:10058000202002596988888888888888887002595C
:100590006988888888505050202002596988888846
:1005A00088A8A8A8A850025969888850502050509F
:1005B00088880259698888505020202020200259BC
:1005C00069F808101020404080F8113B6BE08080F3
:1005D00080808080808080E0025969808040402057
:1005E00010100808113B6BE0202020202020202044
:1005F00020E0085363205088015161F82A2262806C
:100600004002566670087888986802596980808030
:10061000F088888888F0025666708880808870022A
:10062000596908080878888888887802566670882A
:10063000F880887002596930484040F0404040409E
:1006400000586870888888780888700259698080A6
:1006500080B0C8888888881238684000C040404010
:1006600040E0004A6A1000301010101090906002B4
:10067000596980808090A0C0A09088123969C040DC
:10068000404040404040E0025666D0A8A8A8A88854
:10069000025666B0C888888888025666708888883E
:1006A0008870005868F0888888F0808080005868DA
:1006B0007888888878080808025666B0C8808080E4
:1006C000800256667088601088700258684040F05A
:1006D00040404048300256668888888898680256AC
:1006E000668888885050200256668888A8A8A85036
:1006F000025666885020205088005868888888985C
:1007000068088870025666F810204080F8015B6B1C
:100710001820202020C02020202018221969808045
:1007200080808080808080015B6BC020202020182A
:1007300020202020C008536348A890FFFFFFFFFF40
:10074000FFFFFFFFFFFFFFFFFFFFFFFFFFFFFFFFB9
:10075000FFFFFFFFFFFFFFFFFFFFFFFF0D00602216
:1007600019698000808080808080800358682070B4
:10077000A8A0A0A8702002596930484040E040403D
:1007800048B003566688705050708802596988884E
:100790005050F820F8202022196980808080008045
:1007A000808080124A6A60908060909060109060B3
:1007B0001A3262A0A00359697088A8D8C8D8A8883E
:1007C00070045767700878887800F80356662850D8
:1007D000A0A05028045363F80808163161E00359BB
:1007E000697088E8D8D8E8D888700A5161F8174449
:1007F00064609090600357672020F8202000F8077D
:10080000356540A02040E007356540A04020C02A63
:10081000226240800058688888888898E880800232
:10082000596978E8E8E8E868282828262161C02086
:100830002262408007356540C04040E00457677041
:100840008888887000F8035666A050282850A002B7
:100850005A6A40C04040E00818283808025A6A40E6
:10086000C04040E01028081038025A6A40A04020DA
:10087000A0481828380802596920002020408088A4
:100880008870025A6A40200020508888F8888802C0
:100890005A6A10200020508888F88888025A6A30E6
:1008A000480020508888F88888025A6A285000201A
:1008B000508888F88888025A6A50500020508888EA
:1008C000F88888025A6A20502020508888F8888842
:1008D00002596958A0A0A0B0E0A0A0B8005B6B705E
:1008E00088808080808088702040025A6A40200082
:1008F000F88080F08080F8025A6A102000F880802A
:10090000F08080F8025A6A304800F88080F08080D9
:10091000F8025A6A505000F88080F08080F8123A4D
:100920006A804000E04040404040E0123A6A204087
:1009300000E04040404040E0124A6A609000E040E1
:1009400040404040E0123A6AA0A000E040404040F1
:1009500040E0025969F0484848E8484848F0025ADF
:100960006A2850008888C8A8988888025A6A402057
:100970000070888888888870025A6A102000708801
:100980008888888870025A6A304800708888888809
:100990008870025A6A285000708888888888700297
:1009A0005A6A505000708888888888700355658816
:1009B00050205088015B6B08709898A8A8A8C8C8F8
:1009C0007080025A6A40200088888888888870026F
:1009D0005A6A10200088888888888870025A6A308D
:1009E000480088888888888870025A6A5050008831
:1009F000888888888870025A6A1020008888502069
:100A000020202002596980F0888888F08080800248
:100A10005969609090A0A0908888B00259694020E0
:100A2000007008788898680259691020007008786A
:100A30008898680259693048007008788898680278
:100A40005969285000700878889868025969505090
:100A500000700878889868025A6A30483000700838
:100A600078889868025666702870A0A85000586868
:100A7000708880808870204002596940200070880A
:100A8000F88088700259691020007088F88088709A
:100A90000259693048007088F8808870025969509E
:100AA00050007088F8808870123969804000C0401A
:100AB000404040E0123969204000C040404040E0E2
:100AC000124969609000C040404040E0123969A07E
:100AD000A000C040404040E0025A6A5020601070C0
:100AE0008888888870025969285000B0C88888882A
:100AF0008802596940200070888888887002596986
:100B00001020007088888888700259693048007009
:100B10008888888870025969285000708888888879
:100B20007002596950500070888888887003576730
:100B3000202000F8002020015868087098A8A8C854
:100B40007080025969402000888888889868025916
:100B500069102000888888889868025969304800A0
:100B600088888888986802596950500088888888E1
:100B70009868005B6B1020008888889868088870E7
:100B8000005A6A8080B0C88888C8B08080005B6BDB
:100B9000505000888888986808887001050700FE12
:100BA0000500FB01F220FFFE05FE05FE02004002EB
:100BB00015258080800080053242A0A00255655036
:100BC000F850F8500146562070C030E020025565BC
:100BD0009010204048025565608068906805122298
:100BE000808002253540808080400225358040404D
:100BF0004080043343A040A003334340E04001223F
:100C0000324080043141E002112180025565081014
:100C10002040800245556090909060022535C0408C
:100C2000404040024555E0106080F0024555E0101C
:100C30006010E00245552060A0F020024555F0808C
:100C4000E010E00245556080E09060024555F010EC
:100C5000204040024555609060906002455560908C
:100C600070106003132380008002142480008080B1
:100C70000235452040804020033343E000E0023548
:100C8000458040204080024555E0106000400255FC
:100C9000657088B8A870024555609090F090024544
:100CA00055E090E090E0023545608080806002452C
:100CB00055E0909090E0023545E080E080E002351C
:100CC00045E080E080800245557080B0907002451C
:100CD000559090F09090023545E0404040E002454C
:100CE00055301010906002455590A0C0A09002357C
:100CF0004580808080E002556588D8A888880245B4
:100D00005590D0B09090024555609090906002450B
:100D100055E09090E08001465660909090601002FF
:100D20004555E09090E09002455570806010E002DB
:100D30003545E0404040400245559090909060021B
:100D400045559090A0A04002556588A8A8A85002DB
:100D500045559090609090024555909070106002BB
:100D60003545E0204080E0022535C0808080C0020B
:100D700055658040201008022535C0404040C00520
:100D8000324240A0024151F00522328040024454D8
:100D90007090907002455580E09090E0023444607D
:100DA000808060024555107090907002445460B08D
:100DB000C0600235452040E04040004656709090AB
:100DC00070106002455580E09090900215258000DB
:100DD00080808000273740004040404080024555D9
:100DE0008090A0E09002152580808080800254646D
:100DF000F0A8A8A8024454E0909090024454609057
:100E00009060004656E09090E080800046567090DA
:100E100090701010023444A0C0808002445470C00E
:100E200030E002354540E04040200244549090902C
:100E3000700244549090A040025464A8A8505002FC
:100E40003444A04040A0004656909090701060023C
:100E50004454F02040F00235456040804060021567
:100E6000258080808080023545C0402040C00542FA
:100E70005250A0FFFFFFFFFFFFFFFFFFFFFFFFFF3D
:100E8000FFFFFFFFFFFFFFFFFFFFFFFFFFFFFFFF72
:100E9000FFFFFFFF020040FFFFFFFFFFFFFFFFFF1D
:100EA000FFFFFFFFFFFFFFFFFFFFFFFFFFFFFFFF52
:100EB000FFFFFFFFFFFFFFFFFFFFFFFFFFFFFFFF42
:100EC000FFFFFFFFFFFFFFFFFFFFFFFFFFFFFFFF32
:100ED000FFFFFFFFFFFFFFFFFFFFFFFFFFFFFFFF22
:100EE000FFFFFFFFFFFFFFFFFFFFFFFFFFFFFFFF12
:100EF000FFFFFFFFFFFF01050800FF06012102358C
:100F000020FFFF07FF06FF09005022165680808051
:100F1000800080153353A0A0A00257575050F850BE
:100F2000F850500257572070A07028702013355584
:100F300080A040A02002475740A0A040A0A050257C
:100F40001353808080122656408080808040122675
:100F5000568040404040800245559060F0609002CD
:100F600055552020F8202011335360408004415112
:100F7000F011335340E0400246561010204080806C
:100F800012365640A0A0A0A04012365640C04040A5
:100F900040E00246566090106080F0024656F02015
:100FA000601090600246562060A0F0202002465655
:100FB000F080E01090600246566080E09090600201
:100FC0004656F010202040400246566090609090B7
:100FD00060024656609090701060122555C0C000A7
:100FE000C0C0113656606000604080123656204006
:100FF00080804020034353F000F01236568040209A
:1010000020408012365640A0204000400158583001
:101010004898A8A8904030024656609090F0909072
:10102000024656E090E09090E00246566090808044
:101030009060024656E090909090E0024656F08014
:10104000E08080F0024656F080E0808080024656C4
:10105000609080B090600246569090F09090901210
:101060003656E040404040E002465670202020A026
:101070004002465690A0C0A0A090024656808080B4
:101080008080F002465690F0F09090900246569084
:10109000D0F0B0B0900246566090909090600246BA
:1010A00056E09090E08080014757609090D0B0600B
:1010B00010024656E09090E09090024656609040B4
:1010C000209060123656E040404040400246569024
:1010D000909090906002465690909090606002468A
:1010E00056909090F0F090024656909060609090EC
:1010F000025656888850202020024656F010204084
:1011000080F0123656E080808080E0024656808073
:1011100040201010123656E020202020E0163252D7
:1011200040A0014151F01622528040024454709078
:1011300090700246568080E09090E01234546080B7
:10114000806002465610107090907002445460B057
:10115000C060024656205040E04040014555609036
:101160007010600246568080E09090901236564093
:1011700000C04040E01137572000202020A040024E
:101180004656808090E09090123656C040404040D5
:10119000E0025454D0A8A8A8024454E090909002D1
:1011A000445460909060014555E090E08080014596
:1011B000557090701010024454A0D08080123454A6
:1011C00060C020C00246564040E0405020024454D7
:1011D00090909070123454A0A0A04002545488A85B
:1011E000A8500244549060609001455590907090D2
:1011F00060024454F02040F0024757304020C020A5
:101200004030221656808080808080024757C02060
:1012100040304020C006425250A0FFFFFFFFFFFFBA
:10122000FFFFFFFFFFFFFFFFFFFFFFFFFFFFFFFFCE
:10123000FFFFFFFFFFFFFFFFFFFFFF090050221628
:10124000568000808080800146562070A0A07020CB
:101250000246562050E04050A0025555887050700C
:10126000880256568850F820F82022175780808030
:10127000008080800247577080E0907010E0173146
:1012800051A002565670A8C8C8A87014355560A061
:101290006000E003435350A050123353E020201469
:1012A0003151E002565670E8D8E8D870173151E055
:1012B00015335340A04012355540E04000E014354E
:1012C0005540A02040E0143555C020C020C0162253
:1012D000524080014555909090E08002565678E843
:1012E000E868282824115180112252408014355575
:1012F00040C04040E014355540A04000E003435357
:10130000A050A0024757808080A060F0200247577D
:101310008080A0D010207002475780408060A0F0ED
:101320002012365640004080A040024757402060BF
:1013300090F0909002475720406090F090900247C4
:101340005760906090F0909002475750A06090F0E6
:10135000909002475790006090F09090024757603D
:10136000906090F0909002465670A0A0F0A0B0015E
:101370004757609080809060400247574020F0803F
:10138000E080F00247572040F080E080F0024757AD
:101390006090F080E080F00247579000F080E0809D
:1013A000F01237578040E0404040E012375720406D
:1013B000E0404040E012375740A0E0404040E0129B
:1013C0003757A000E0404040E00256567048E848D9
:1013D000487002475750A090D0B0909002475740B5
:1013E00020609090906002475720406090909060FD
:1013F0000247576090609090906002475750A060FD
:1014000090909060024757900060909090601233E7
:1014100053A040A002465670B0B0D0D0E00247576B
:10142000402090909090600247572040909090907C
:1014300060024757609090909090600247579000EC
:1014400090909090600257571020885020202002E2
:10145000465680E09090E0800246566090A0A090B2
:10146000A0024757402000709090700247572040DC
:10147000007090907002475720500070909070025A
:10148000475750A0007090907002465650007090E0
:10149000907002475760906070909070025454F0C2
:1014A00068B0781135556080806040024757402011
:1014B0000060B0C06002475720400060B0C06002CA
:1014C000475760900060B0C060024656500060B060
:1014D000C060123757804000C04040E012375720AC
:1014E0004000C04040E012375740A000C04040E0FC
:1014F000123656A000C04040E0024757A040A0105E
:1015000070906002475750A000E0909090024757BB
:10151000402000609090600247572040006090900B
:10152000600247576090006090906002475750A05B
:101530000060909060024656900060909060123576
:10154000554000E0004002445470B0D0E0024757DC
:10155000402000909090700247572040009090905B
:10156000700247576090009090907002465690002D
:1015700090909070014858204000909070906001C9
:1015800047578080E090E08080014757900090901E
:10159000709060202020200020202020202020008B
:1015A00025753A2530327500253032753A253032AE
:1015B000750025756420253032753A253032750066
:1015C0003FFFF03800703186302387102787902F37
:1015D00087D02F03D02030102078102078102030B2
:1015E000102F03D02F87D027879023871031863084
:1015F0003800703FFFF03FFFF038007030FC3020C3
:10160000FC102078102030102C00D02E31D02F7BF1
:10161000D02F7BD02E31D02C00D02030102078104D
:1016200020FC1030FC303800703FFFF00410400206
:1016300008200208200410400820801041001041BA
:10164000000820800410400000001FFFF81FFFF872
:101650001FFFF81FFFF81FE020102010201010209F
:1016600010202010201030300840048003001FE0BC
:101670003FF03FF03FF01FE01FE03FF03FF03FF052
:101680000FC0078003004572723A207574663820D7
:10169000666F6E74206E6F7420696E697469616C18
:1016A000697A65642E004572723A20757466382036
:1016B000666F6E74206E6F7420696E697469616CF8
:1016C000697A65642E004572723A20757466382016
:1016D000666F6E74206E6F7420696E697469616CD8
:1016E000697A65642E00506C65617365207265735C
:1016F0006574005052494E5445522048414C54455F
:1017000044007F80FFC0FFC0FFC07F807F80FFC09C
:10171000FFC0FFC03F001E000C00FFFFFF0E000EC9
:10172000000E000E000E000E000E000E007FC03FE7
:10173000801F000E00040004000E001F003F807F89
:10174000C00E000E000E000E000E000E000E000E69
:101750000000FE0003FF800783C00E01C00E00E002
:101760001C00E07F00E03E00E01C00E00800E0001C
:1017700000E00001C00E01C00F078007FF0001FC60
:101780000001FC0007FF000F07800E01C00001C030
:101790000000E00800E01C00E03E00E07F00E01CEC
:1017A00000E00E00E00E01C00783C003FF8000FED2
:1017B0000000060C00FE07022603BC017FFE08FEA7
:1017C00008FE05080806000040F0C88888987810D0
:1017D000050808060000C0F88888888888F805058C
:1017E000050600012030F83020050808060000201A
:1017F00070F820202020E00509090600FF2070A8CD
:10180000A8B888887020050606060001E08CEA8CDE
:101810008A0A0509090600FFF8A88888888888A828
:10182000F8050A0A0600FE205050505088A8A888E3
:101830007003030306000340A040FFFFFFFFFFFF0C
:10184000FFFFFFFFFFFFFFFFFFFFFFFFFFFFFFFFA8
:101850000000000605FF0107070602008080808067
:10186000800080030303060105A0A0A0050606066C
:10187000000050F85050F8500509090600FF20708C
:10188000A8A07028A87020050707060000C8C81087
:101890002040989805070706000040A0A040A890A7
:1018A000680103030602058080800309090601FF21
:1018B0002040408080804040200309090601FF80CD
:1018C000404020202040408005070706000020A857
:1018D000702070A8200505050600012020F82020B2
:1018E0000203030601FFC04080050101060003F862
:1018F000020202060100C0C005070706000008102A
:101900001020404080050707060000708898A8C88E
:10191000887003070706010040C040404040E005D2
:101920000707060000708808102040F80507070622
:101930000000F8081030088870050707060000103E
:10194000305090F81010050707060000F880F008E6
:10195000088870050707060000304080F08888700E
:10196000050707060000F8081010202020050707CB
:1019700006000070888870888870050707060000D8
:1019800070888878081060020505060100C0C00054
:10199000C0C00206060601FFC0C000C040800305AB
:1019A000050601012040804020050303060002F8DF
:1019B00000F8030505060101804020408005070767
:1019C0000600007088102020002005070706000090
:1019D0007088B8A8B880700507070600007088886E
:1019E000F8888888050707060000F04848704848CE
:1019F000F005070706000070888080808870050762
:101A000007060000F04848484848F0050707060068
:101A100000F88080F08080F8050707060000F88055
:101A200080F080808005070706000070888080981D
:101A30008870050707060000888888F8888888036A
:101A40000707060100E04040404040E00507070668
:101A5000000038101010109060050707060000887D
:101A600090A0C0A0908805070706000080808080B5
:101A70008080F805070706000088D8A8888888882D
:101A80000507070600008888C8A898888805070702
:101A9000060000708888888888700507070600009F
:101AA000F08888F08080800507070600007088882D
:101AB00088A89068050707060000F08888F0A090C5
:101AC0008805070706000070888070088870050781
:101AD00007060000F8202020202020050707060028
:101AE000008888888888887005070706000088882D
:101AF000888850502005070706000088888888A835
:101B0000A8500507070600008888502050888805DF
:101B100007070600008888502020202005070706B8
:101B20000000F80810204080F80309090601FFE0D2
:101B300080808080808080E005070706000080406C
:101B400040201010080309090601FFE02020202092
:101B5000202020E005030306000520508805010130
:101B60000600FEF803030306010580402005050575
:101B70000600007008788878050707060000808056
:101B8000F0888888F0050505060000708080887060
:101B90000507070600000808788888887805050585
:101BA0000600007088F080700507070600003048C6
:101BB00040E04040400507070600FE7088888878AE
:101BC00008700507070600008080F0888888880371
:101BD00007070601004000C0404040E00409090634
:101BE00001FE10003010101010906005070706006D
:101BF0000080808890E09088030707060100C040BD
:101C000040404040E0050505060000D0A8A8A8A86F
:101C1000050505060000B0C888888805050506008A
:101C20000070888888700507070600FEF08888889D
:101C3000F080800507070600FE7888888878080805
:101C4000050505060000B0C8808080050505060072
:101C50000078807008F00507070600002020F820B3
:101C60002020180505050600008888889868050565
:101C700005060000888888502005050506000088B4
:101C800088A8A85005050506000088502050880542
:101C900007070600FE888888502040800505050655
:101CA0000000F8102040F80309090601FF20404019
:101CB0004080404040200109090602FF808080806A
:101CC00080808080800309090601FF804040402019
:101CD0004040408005030306000248A890FF1FFF14
:101CE000FFFFFFFFFF600000000001FF4000000059
:101CF0000000FF8000000000007F83CF00000C3058
:101D00003F87FF80000C301F867980000C000F8C0D
:101D100030C7838C30E78C30CFC7CC31F38C30DCCC
:101D2000ECEC33B98C30D86C6C33198C30D06C0C33
:101D300033198C30D86C0C33198C30DC6C0E3B1999
:101D40008C30CF7C079F198C30C77C038F194000E3
:101D50000000000002600000000000061FFFFFFFFF
:101D6000FFFFF800060900FE06018902FE20FFFEC3
:101D700007FE06FE00000006000701060606020038
:101D8000808080800080030303060103A0A0A005DB
:101D900007070600FF5050F850F850500509090693
:101DA00000FE2070A8A07028A87020060808060071
:101DB000FF40A84810204854080507070600FF60A8
:101DC000909060989068010303060203808080026F
:101DD00007070602FF4080808080804002070706D8
:101DE00002FF804040404040800505050600008815
:101DF00050F850880505050600002020F820200234
:101E000004040602FEC0404080050101060002F8FD
:101E1000020202060200C0C00406060601001010FD
:101E2000204080800406060601006090909090603B
:101E300003060606010040C0404040E004060606D6
:101E400001006090102040F0040606060100F0201A
:101E5000601010E005060606000010305090F810E3
:101E6000040606060100F080E01010E004060606F5
:101E700001006080E0909060040606060100F0100A
:101E800010204040040606060100609060909060BB
:101E900004060606010060909070106002050506B9
:101EA0000200C0C000C0C00207070602FEC0C0009A
:101EB000C0404080050505060000186080601805D8
:101EC0000303060001F800F8050505060000C03010
:101ED0000830C00407070601006090106040004011
:101EE0000506060600007090A8B08070050606067C
:101EF0000000205088F88888050606060000F08853
:101F0000F08888F0040606060100609080809060EA
:101F1000040606060100E090909090E00406060694
:101F20000100F080E08080F0040606060100F080E9
:101F3000E0808080040606060100609080B090601A
:101F40000406060601009090F090909003060606A5
:101F50000100E040404040E0050606060000381061
:101F60001010906004060606010090A0C0A090909A
:101F70000406060601008080808080F005060606C3
:101F8000000088D8A8A8888804060606010090D01A
:101F9000B0909090050606060000708888888870CA
:101FA000040606060100E09090E080800407070622
:101FB00001FF609090D0B06010040606060100E0BA
:101FC0009090E090900406060601006090402090FA
:101FD00060050606060000F82020202020040606E2
:101FE0000601009090909090600406060601009013
:101FF0009090F060600506060600008888A8A8D8C2
:102000008805060606000088502020508805060630
:10201000060000888850202020040606060100F0F3
:1020200010204080F0030606060100E080808080DA
:10203000E00406060601008080402010100306061A
:10204000060100E020202020E00503030600032015
:1020500050880501010600FEF80202020602048013
:102060004004040406010070909070040606060106
:10207000008080E09090E0040404060100708080FD
:10208000700406060601001010709090700404049D
:1020900006010060B0C07004060606010020504032
:1020A000E040400406060601FE6090907010600457
:1020B00006060601008080E0909090030606060167
:1020C000004000C04040E00308080601FE20006018
:1020D000202020A0400406060601008080A0C0A0A9
:1020E00090030606060100C040404040E00504049D
:1020F000060000D0A8A888040404060100E090901F
:102100009004040406010060909060040606060135
:10211000FEE09090E080800406060601FE7090903C
:10212000701010040404060100A0D0808004040490
:1021300006010070C030E00406060601004040E0E1
:1021400040502004040406010090909070040404A0
:102150000601009090606005040406000088A8A8AD
:102160005004040406010090606090040606060115
:10217000FE909090709060040404060100F02040EE
:10218000F00307070601002040408040402001077F
:10219000070602FF80808080808080030707060199
:1021A000008040402040408004020206010350A00D
:1021B000FFFFFFFFFFFFFFFFFFFFFFFFFFFFFFFF2F
:1021C000FFFFFFFFFFFFFFFFFFFFFFFFFFFFFFFF1F
:1021D000FF000000060007010606060200800080DE
:1021E0008080800406060601FF2070A0A0702005F4
:1021F00007070600FF304840F04040F80505050697
:102200000000A8508850A80506060600008850F86F
:1022100020F8200107070602FF8080800080808070
:102220000407070601FF708060906010E003010161
:10223000060105A0060707060000788494A494848C
:102240007803050506010160A06000E005050506AC
:1022500000002850A05028040303060100F01010CD
:10226000040101060102F00607070600007884B4A5
:10227000A4A48478040101060105F0040303060107
:10228000026090600507070600FF2020F82020006C
:10229000F803050506010140A02040E003050506FE
:1022A0000101C0204020C002020206020440800456
:1022B00005050601FF9090B0D080050606060000D7
:1022C00078E8E8682828010101060202800202027B
:1022D0000602FE408003050506010140C04040E0C3
:1022E00003050506010140A04000E00505050600C4
:1022F00000A0502850A00508080600FF40C040502C
:10230000703078100508080600FF40C0405068088B
:1023100010380508080600FFC0204030F030781063
:102320000407070601002000206080906005070771
:10233000060000402020507088880507070600002E
:1023400010202050708888050707060000205020C4
:1023500050708888050707060000285020507088B4
:102360008805070706000050002050708888050780
:1023700007060000205020507088880506060600D9
:102380000078A0F0A0A0B80408080601FE609080C4
:1023900080906020400407070601004020F080E0A4
:1023A00080F00407070601002040F080E080F00480
:1023B00007070601002050F080E080F004070706C0
:1023C00001005000F080E080F00307070601008064
:1023D00040E0404040E00307070601002040E040A5
:1023E0004040E003070706010040A0E0404040E015
:1023F000030707060100A000E0404040E005060694
:102400000600007048E848487004070706010050BD
:10241000A090D0B090900407070601004020609083
:102420009090600407070601002040609090906043
:102430000407070601002050609090906004070791
:1024400006010050A060909090600407070601000C
:1024500050006090909060050505060000885020AF
:1024600050880408080601FF1070B0B0D0D0E0809A
:102470000407070601004020909090906004070731
:10248000060100204090909090600407070601002C
:102490002050909090906004070706010050009033
:1024A00090909060050707060000102088502020BB
:1024B0002004060606010080E09090E080040606F5
:1024C0000601006090A0A090A0040707060100404C
:1024D00020007090907004070706010020400070F3
:1024E00090907004070706010020500070909070D3
:1024F00004070706010050A00070909070040606C3
:10250000060100500070909070040707060100203B
:1025100050207090907005040406000070A8B078F8
:102520000406060601FE708080702040040707063E
:10253000010040200060B0C07004070706010020C1
:10254000400060B0C0700407070601002050006022
:10255000B0C070040606060100500060B0C07003F1
:102560000707060100804000C04040E0030707065F
:102570000100204000C04040E00307070601004082
:10258000A000C04040E0030606060100A000C040D5
:1025900040E004070706010030601070909060046E
:1025A000070706010050A000E0909090040707067E
:1025B00001004020006090906004070706010020A1
:1025C0004000609090600407070601002050006002
:1025D00090906004070706010050A0006090906092
:1025E000040606060100500060909060050505068F
:1025F00000002000F8002004040406010070B0D0A0
:10260000E004070706010040200090909070040746
:102610000706010020400090909070040707060113
:1026200000205000909090700406060601005000B3
:10263000909090700409090601FE2040009090904F
:102640007090600408080601FE8080E09090E080B1
:10265000800408080601FE5000909090709060532E
:102660006E346B3300496E7661646572730042723A
:1026700069636B6F7574004D61696E005072696EAD
:10268000742066726F6D205344005072696E74201E
:1026900066726F6D20534400022E2E004D61696EEC
:1026A000005072696E740043616E63656C00537410
:1026B000617274207072696E7420003F00536D6FF8
:1026C0006F7468696E6700536D6F6F7468696E67C9
:1026D000005A005A005900590058005800436F72C0
:1026E00072656374696F6E00436F727265637469BB
:1026F0006F6E004D61696E0046696C616D656E7448
:102700000054656D7065726174757265004472691C
:10271000766520537472656E677468004261636BFE
:102720006C6173680053746570732F6D6D004A653A
:10273000726B00416363656C65726174696F6E00F2
:1027400056656C6F6369747900436F6E666967756F
:10275000726174696F6E004573746570732F6D6D6F
:10276000004573746570732F6D6D005A73746570D6
:10277000732F6D6D005A73746570732F6D6D0059F2
:1027800073746570732F6D6D005973746570732F5A
:102790006D6D005873746570732F6D6D0058737490
:1027A0006570732F6D6D00416476616E63656420A2
:1027B00053657474696E67730056652D6A65726B34
:1027C0000056652D6A65726B00567A2D6A65726BCC
:1027D00000567A2D6A65726B0056792D6A65726BA8
:1027E0000056792D6A65726B0056782D6A65726B9A
:1027F0000056782D6A65726B00416476616E636580
:10280000642053657474696E677300416D6178204C
:102810004500416D6178204500416D6178205A0086
:10282000416D6178205A00416D6178205900416DF9
:102830006178205900416D6178205800416D6178C0
:10284000205800412D74726176656C00412D7472C0
:102850006176656C00412D7265747261637400412C
:102860002D7265747261637400416363656C00412D
:102870006363656C00416476616E636564205365D3
:102880007474696E6773005654726176206D696E58
:10289000005654726176206D696E00566D696E0047
:1028A000566D696E00566D6178204500566D6178F1
:1028B000204500566D6178205A00566D6178205A87
:1028C00000566D6178205900566D61782059005688
:1028D0006D6178205800566D61782058004164760B
:1028E000616E6365642053657474696E677300205C
:1028F000082046616374002008204661637400204C
:1029000008204D6178002008204D617800200820C3
:102910004D696E002008204D696E004175746F741A
:10292000656D70004F6666004F6E004175746F7480
:10293000656D7000416476616E63656420536574F3
:1029400074696E6773004C6F6164206D6D004C6F2D
:102950006164206D6D00556E6C6F6164206D6D005B
:10296000556E6C6F6164206D6D00416476616E63BD
:1029700065204B00416476616E6365204B004164C5
:1029800076616E6365642053657474696E67730065
:10299000450045005A005A005859005859004164F2
:1029A00076616E6365642053657474696E67730045
:1029B00044697361626C65207374657070657273CD
:1029C000004D3834004175746F20686F6D650047A5
:1029D0003238004D6F76652061786973004D61690A
:1029E0006E004578747275646572004175746F206D
:1029F000686F6D6500473238004D6F7665205A006C
:102A00004D6F76652059004D6F76652058004D6FEB
:102A100074696F6E004578747275646572004D6FED
:102A2000766520302E3032356D6D004D6F76652025
:102A3000302E316D6D004D6F766520316D6D004D1E
:102A40006F76652031306D6D004D6F766520617851
:102A5000697300486F74656E6420746F6F20636FD4
:102A60006C64004578747275646572004D6F7665AC
:102A7000205A004D6F76652059004D6F76652058BD
:102A8000004D6F7665205A004D6F76652059004DD8
:102A90006F76652058005761697420666F72006612
:102AA000696C616D656E7420707572676500576141
:102AB000697420666F72207072696E7400746F2082
:102AC000726573756D652E2E2E00507265737320BE
:102AD000627574746F6E00746F20726573756D65C6
:102AE000207072696E74005761697420666F72009D
:102AF00066696C616D656E74206C6F616400496E0F
:102B0000736572742066696C616D656E7400616EC8
:102B10006420707265737320627574746F6E0074D4
:102B20006F20636F6E74696E7565005072657373A4
:102B300020627574746F6E00746F20686561742014
:102B40006E6F7A7A6C65004E6F7A7A6C6520686574
:102B50006174696E6700506C6561736520776169A7
:102B6000742E2E2E005761697420666F720066699C
:102B70006C616D656E7420756E6C6F616400576179
:102B8000697420666F720066696C616D656E742091
:102B90006368616E676500746F207374617274009E
:102BA0005061726B696E672E2E2E005052494E5442
:102BB0002050415553454400554E4C4F414420460A
:102BC000494C414D454E54004C4F41442046494CE0
:102BD000414D454E540020204E6F7A7A6C653A2064
:102BE000002000436F6E74696E75650050757267E2
:102BF00065206D6F726500524553554D45204F500D
:102C000054494F4E533A004368616E6765206669C8
:102C10006C616D656E7400556E6C6F6164206669E1
:102C20006C616D656E74004C6F61642066696C61E7
:102C30006D656E74004D363030204230205425646E
:102C4000004D373032203B2564004D373032205460
:102C50002564004D3730312054256400507265687A
:102C600065617420437573746F6D0050726568659B
:102C7000617420437573746F6D005072656865618F
:102C80007420414253005072656865617420504C55
:102C900041004261636B004E6F20534420636172B8
:102CA00064005072696E742066726F6D2053440028
:102CB0004368616E67652053442063617264004D10
:102CC00032310041626F7574205072696E746572A2
:102CD000004368616E67652066696C616D656E743E
:102CE000004368616E67652066696C616D656E742E
:102CF000004D36303020423000436F6E6669677594
:102D0000726174696F6E0054656D7065726174757F
:102D10007265004D6F74696F6E00526573756D65F5
:102D2000207072696E740054756E650053746F7014
:102D3000207072696E7400506175736520707269DD
:102D40006E7400496E666F2073637265656E005322
:102D5000746F70004261636B0053746F7020707207
:102D6000696E74003F0050726F6265205A204F6692
:102D700066736574004261627973746570205900EE
:102D80004261627973746570205800466C6F7700F9
:102D9000466C6F770046616E20737065656400460F
:102DA000616E20737065656400426564004265640D
:102DB000004E6F7A7A6C65004E6F7A7A6C650053BC
:102DC00070656564005370656564004D61696E00EF
:102DD000426162797374657020590042616279734F
:102DE00074657020580047616D6573005072696E9C
:102DF00074657220496E666F004D61696E00436FA5
:102E00006F6C646F776E0046616E207370656564E9
:102E10000046616E2073706565640042656400421F
:102E20006564004E6F7A7A6C65004E6F7A7A6C65D5
:102E3000004D61696E006F6F6F0000001FC07FF072
:102E4000DDD8FFF87FF0444024800000318000008E
:102E500024804440107CFEFEFE04000E000E007F25
:102E6000C0FFE0FFE0FFE0FFE006000F001F80363C
:102E7000C03FC009001680294006000F001F8036A1
:102E8000C03FC0168020401080104008801FC0370F
:102E9000607FF05FD050500D80104048905FD07739
:102EA000707FF01FC0104020200F007FE0FFF0E691
:102EB00070FFF0198036C0C0300F007FE0FFF0E6F1
:102EC00070FFF0198036C0198047414D45204F569C
:102ED000455200526573746F7265206661696C7348
:102EE000616665004C6F61642073657474696E6718
:102EF000730053746F72652073657474696E6773C1
:102F00000050726F6265205A204F666673657400C8
:102F1000416476616E6365642053657474696E679D
:102F200073004D61696E0050726F6265205A204FC8
:102F30006666736574004D6F76696E672E2E2E007F
:102F40004D3234004D323520500A4D32340050722B
:102F5000696E742070617573656400506175736586
:102F6000207072696E74005072696E742061626FB5
:102F700072746564004C756C7A426F74204D696E92
:102F800069204C43442052656164792E0050726977
:102F90006E74696E672E2E2E005072696E742070EA
:102FA000617573656400436172642072656D6F764C
:102FB0006564004361726420696E73657274656450
:102FC000004D313137004D33310043616E6E6F7407
:102FD00020656E746572207375626469723A2000B0
:102FE0002E0A006F70656E206661696C65642C2026
:102FF00046696C653A20006175746F25632E670021
:103000006572726F722077726974696E6720746F6F
:103010002066696C650A004E6F74205344207072FC
:10302000696E74696E670A005344207072696E7429
:10303000696E67206279746520002E0A0044656C11
:103040006574696F6E206661696C65642C204669E1
:103050006C653A200046696C652064656C65746532
:10306000643A0057726974696E6720746F206669EC
:103070006C653A20002E0A006F70656E20666169EB
:103080006C65642C2046696C653A20002E0A006F3E
:1030900070656E206661696C65642C2046696C659C
:1030A0003A200046696C652073656C6563746564DD
:1030B0000A002053697A653A200046696C65206FE2
:1030C00070656E65643A20002066696C653A200080
:1030D000667265736800646F696E67004E6F772073
:1030E00000454E4420535542524F5554494E450ACF
:1030F000002220706F73002220706172656E743A36
:103100002200535542524F5554494E452043414C9D
:103110004C207461726765743A2200747279696E2A
:103120006720746F2063616C6C207375622D676318
:103130006F64652066696C657320776974682074B4
:103140006F6F206D616E79206C6576656C732E20D3
:103150004D4158206C6576656C2069733A310A00E0
:103160004D3234004D3233202573005344206361C7
:103170007264206F6B0A006F70656E526F6F7420FF
:103180006661696C65640A00766F6C756D652E69A1
:103190006E6974206661696C65640A005344206935
:1031A0006E6974206661696C0A00286E6F2066691A
:1031B0006C65290043616E6E6F74206F70656E20C0
:1031C00073756264697220007C3C3E5E2B3D3F2F2C
:1031D0005B5D3B2C2A225C00000000000000000028
:1031E00000000000000000000000000000000000DF
:1031F00000000000000000000000000C00000000C3
:103200000000000C000000000000001200000000A0
:10321000000000230000000000000021000000006A
:103220000000004C800000000000005E80000000F4
:103230000000009240000000000000A140000000DB
:1032400000000121200000000000027F900000002B
:103250000000020010000000000007FFF80000005E
:103260000000040008000000000008000400000046
:10327000000008000600000000001000020000002E
:103280000000301E010000000000207F81000000CF
:10329000000041FFE0800000000043FCF0800000DF
:1032A0000000873B7840000000018EDBFC600000DE
:1032B00000010FEBCC20000000021FEDB610000053
:1032C00000021FDEB6100000000439CD7F080000A8
:1032D000000436E0FF08000000087EC0BB84000048
:1032E00000187F005D86000000107FC0ED820000A6
:1032F00000203CC07301000000203B337F01000030
:1033000000701BE77E03800000C81DEEDE04C000D5
:1033100000880FDEDC04400001240FDF3C092000A0
:10332000012607DBF8192000027203E7F013900072
:10333000025101FFE02290000489007F80244800B0
:103340000904801E004824000BFE400000DFF4004A
:1033500010004000008002001FFFFFFFFFFFFE0083
:10336000000000000000000000000000000000005D
:1033700000000000000000001022103C3C0E1F0066
:10338000102210042211040010221008221104003F
:10339000102210083C110400102210102211040009
:1033A00010221020221104001E1C1E3C3C0E0400A2
:1033B000000000000000000000000000000000000D
:1033C00000000000000000000000000000000000FD
:1033D00000000000000000000000000000000000ED
:1033E00000000000000000000000000000000000DD
:1033F00000000000000000000000000000000000CD
:1034000000000000000000000000000000000000BC
:1034100000000000000000060C00FE07022603BCAE
:10342000017FFE08FE08FE05080806000040F0C8FF
:103430008888987810050808060000C0F8888888F1
:103440008888F80505050600012030F830200508B9
:10345000080600002070F820202020E00509090659
:1034600000FF2070A8A8B88888702005060606000E
:1034700001E08CEA8C8A0A0509090600FFF8A88891
:1034800088888888A8F8050A0A0600FE205050504F
:103490005088A8A8887003030306000340A040FFDB
:1034A000FFFFFFFFFFFFFFFFFFFFFFFFFFFFFFFF2C
:1034B000FFFFFFFFFF0000000605FF0107070602F0
:1034C0000080808080800080030303060105A0A0A7
:1034D000A005060606000050F85050F850050909EE
:1034E0000600FF2070A8A07028A870200507070616
:1034F0000000C8C810204098980507070600004043
:10350000A0A040A890680103030602058080800304
:1035100009090601FF2040408080804040200309C7
:10352000090601FF80404020202040408005070719
:1035300006000020A8702070A820050505060001DF
:103540002020F820200203030601FFC0408005016F
:1035500001060003F8020202060100C0C0050707C9
:1035600006000008101020404080050707060000F4
:10357000708898A8C8887003070706010040C040FB
:10358000404040E005070706000070880810204012
:10359000F8050707060000F80810300888700507CE
:1035A0000706000010305090F810100507070600BD
:1035B00000F880F008088870050707060000304012
:1035C00080F0888870050707060000F808101020B2
:1035D000202005070706000070888870888870051D
:1035E0000707060000708888780810600205050645
:1035F0000100C0C000C0C00206060601FFC0C00036
:10360000C0408003050506010120408040200503DD
:1036100003060002F800F8030505060101804020BA
:103620004080050707060000708810202000200554
:1036300007070600007088B8A8B88070050707065D
:103640000000708888F8888888050707060000F061
:103650004848704848F005070706000070888080D9
:10366000808870050707060000F04848484848F081
:10367000050707060000F88080F08080F80507073E
:10368000060000F88080F0808080050707060000B3
:1036900070888080988870050707060000888888F1
:1036A000F8888888030707060100E0404040404052
:1036B000E00507070600003810101010906005079D
:1036C000070600008890A0C0A090880507070600A4
:1036D00000808080808080F805070706000088D879
:1036E000A8888888880507070600008888C8A898E1
:1036F0008888050707060000708888888888700514
:103700000707060000F08888F0808080050707061C
:10371000000070888888A89068050707060000F0F8
:103720008888F0A0908805070706000070888070E0
:10373000088870050707060000F8202020202020B8
:1037400005070706000088888888888870050707AD
:10375000060000888888885050200507070600006A
:1037600088888888A8A85005070706000088885020
:1037700020508888050707060000888850202020F0
:1037800020050707060000F80810204080F803090C
:10379000090601FFE080808080808080E0050707C7
:1037A000060000804040201010080309090601FFB0
:1037B000E020202020202020E00503030600052033
:1037C00050880501010600FEF80303030601058089
:1037D0004020050505060000700878887805070771
:1037E0000600008080F0888888F005050506000046
:1037F00070808088700507070600000808788888B0
:1038000088780505050600007088F08070050707B8
:10381000060000304840E04040400507070600FE33
:10382000708888887808700507070600008080F097
:10383000888888880307070601004000C040404090
:10384000E00409090601FE1000301010101090600D
:1038500005070706000080808890E090880307072E
:10386000060100C04040404040E00505050600005C
:10387000D0A8A8A8A8050505060000B0C8888888B3
:103880000505050600007088888870050707060092
:10389000FEF0888888F080800507070600FE78889B
:1038A0008888780808050505060000B0C880808073
:1038B00005050506000078807008F005070706007A
:1038C000002020F820202018050505060000888823
:1038D0008898680505050600008888885020050539
:1038E000050600008888A8A8500505050600008880
:1038F000502050880507070600FE88888850204021
:1039000080050505060000F8102040F803090906A7
:1039100001FF20404040804040402001090906024C
:10392000FF8080808080808080800309090601FFFD
:10393000804040402040404080050303060002488C
:10394000A890FF4F4646004F4E006563686F3A00EF
:103950004572726F723A004572726F7220777269A7
:1039600074696E6720746F20454550524F4D210A8F
:1039700000507265737320627574746F6E20286FC7
:1039800072204D3130382920746F206865617420B1
:103990006E6F7A7A6C650A00507265737320627577
:1039A00074746F6E20286F72204D31303829207466
:1039B0006F20726573756D650A00496E7365727468
:1039C0002066696C616D656E7420616E6420707232
:1039D00065737320627574746F6E20286F72204D4A
:1039E000313038290A004D3630303A20546F6F207C
:1039F000636F6C6400486F74656E6420746F6F2031
:103A0000636F6C640A00486F74656E6420746F6F36
:103A100020636F6C640A00496E7365727420666976
:103A20006C616D656E7420616E6420707265737375
:103A300020627574746F6E20286F72204D3130389B
:103A4000290A0063616E63656C00726573756D654C
:103A50006400726573756D650070617573656400EF
:103A6000706F7765726F6666002F2F616374696F80
:103A70006E3A0020573A0020573A00486F74656E3E
:103A80006420436F6F6C696E672E2E2E00486F7432
:103A9000656E642048656174696E672E2E2E002065
:103AA0002F002042403A0020403A004D3834205840
:103AB0002059205A204500546865726D616C20526F
:103AC000756E6177617900486F74656E6420544843
:103AD00045524D414C2052554E41574159004245A7
:103AE0004420544845524D414C2052554E41574177
:103AF0005900202D20496E76616C696420657874C8
:103B00007275646572206E756D62657220210A009F
:103B100048656174696E67206661696C656400421E
:103B200065642068656174696E67206661696C65AB
:103B30006400546865726D616C2052756E617761C6
:103B4000790042454420544845524D414C2052553D
:103B50004E415741590048656174696E672066613E
:103B6000696C656400486F74656E642048656174B3
:103B7000696E67206661696C656400546865726D82
:103B8000616C2052756E6177617900486F74656E63
:103B90006420544845524D414C2052554E415741A6
:103BA00059004D494E54454D502074726967676500
:103BB00072656400486F74656E64204572723A20C5
:103BC0004D494E54454D50004572723A204D494E74
:103BD00054454D5020424544004D415854454D50A8
:103BE0002074726967676572656400486F74656EFA
:103BF00064204572723A204D415854454D5000455D
:103C000072723A204D415854454D5020424544006F
:103C1000626564002C2073797374656D2073746F12
:103C20007070656421204865617465725F49443A2B
:103C3000200023646566696E652044454641554C05
:103C4000545F004B6420004B6920004B7020000043
:103C500062656400504944204175746F74756E65E7
:103C60002066696E697368656421205075742074DC
:103C70006865206C617374204B702C204B69206147
:103C80006E64204B6420636F6E7374616E74732076
:103C900066726F6D2062656C6F7720696E746F203D
:103CA000436F6E66696775726174696F6E2E680A1C
:103CB00000504944204175746F74756E65206661CB
:103CC000696C6564212074696D656F75740A0054B0
:103CD0006865726D616C2052756E6177617900481C
:103CE0006F74656E6420544845524D414C205255C6
:103CF0004E415741590042454420544845524D4198
:103D00004C2052554E415741590048656174696EC7
:103D100067206661696C656400486F74656E642035
:103D200048656174696E67206661696C656400420C
:103D300065642068656174696E67206661696C6599
:103D40006400504944204175746F74756E65206637
:103D500061696C6564212054656D7065726174756C
:103D6000726520746F6F20686967680A00204B6471
:103D70003A2000204B693A2000204B703A20000A7C
:103D800020436C617373696320504944200A00200A
:103D90004B643A2000204B693A2000204B703A20B7
:103DA000000A204E6F206F76657273686F6F740A19
:103DB000002054753A2000204B753A2000206D6198
:103DC000783A2000206D696E3A200020643A200085
:103DD00020626961733A2000504944204175746F34
:103DE00074756E652073746172740A0050494420C2
:103DF0004175746F74756E65206661696C656421C8
:103E00002054656D706572617475726520746F6F92
:103E100020686967680A001000AD0330016A01502C
:103E2000022B0170030A019004F500B005E500D0F3
:103E300006D800F007CE001009C500300ABE0050B9
:103E40000BB700700CB100900DAB00B00EA600D007
:103E50000FA200F0109D0010129900301395005031
:103E600014920070158E0090168B00B0178700D04A
:103E7000188400F0198100101B7E00301C7B00505C
:103E80001D7900701E7600901F7300B0207000D066
:103E9000216E00F0226B001024690030256600506E
:103EA0002663007027610090285E00B0295C00D076
:103EB0002A5900F02B5600102D5400302E5100507E
:103EC0002F4E0070304B0090314800B0324500D08A
:103ED000334200F0343E0010363B0030373700509C
:103EE00038330070392E00903A2900B03B2300D0BF
:103EF0003C1B00F03D1100103F0100F03F0000109E
:103F000000C90210012C014001220170011801B00A
:103F1000010E01F00104015002FA00B002F000307D
:103F200003E600D003DC009004D2007005C800A0B6
:103F300006BE000008B400B009AA00D00BA00060C3
:103F40000E960060118C000015820020197800C0C8
:103F50001D6E00A0226400B0275A00902C50000073
:103F6000314600E0343C0010383200903A280060BE
:103F70003C1E00A03D1400803E0A00203F00006F60
:103F800070656E00545249474745524544003A20F7
:103F9000007A5F6D6178007A5F6D696E00795F6DA0
:103FA000617800795F6D696E00785F6D6178007887
:103FB0005F6D696E005265706F7274696E6720651F
:103FC0006E6473746F70207374617475730A004546
:103FD0006E6473746F7073202563202563202563DE
:103FE00020256300205A3A0020593A0020583A0010
:103FF000656E6473746F7073206869743A2000484A
:104000006F6D696E67206661696C656400496E76E4
:10401000616C69642065787472756465720A004524
:10402000303A20005A3A2000593A20004D53312CA2
:104030004D53322C4D53332050696E730A583A2039
:10404000004D6963726F737465707320756E61766D
:1040500061696C61626C650A00205A3A0020593A25
:104060000020436F756E7420583A00C23100001C66
:10407000260000F4190000D80F0000EB080000C073
:10408000040000750200004001000024F4D4305008
:10409000C38E20C2A24017828B7011127A910D81BB
:1040A0006CD90AA861E108C7586607615143061E2A
:1040B0004B5D05C145A7041A411104093D980371E0
:1040C0003931034036DB0265339102D4305402802B
:1040D0002E1D02632CEE01752AC501B028A0011027
:1040E0002781018F2564012B244B01E0223401AC90
:1040F000211F018D200D01801FFC00841EED009703
:104100001DDF00B81CD200E61BC600201BBC0064EB
:104110001AB200B219A8000A19A0006A189900D1B1
:1041200017910040178B00B516840031167E00B33E
:104130001579003A157300C7146F0058146A00EE21
:104140001366008813630025135E00C7125B006CC2
:1041500012570015125400C111510070114F002167
:10416000114B00D61049008D104700461044000244
:10417000104200C00F4000800F3E00420F3C00067E
:104180000F3B00CB0E3800930E37005C0E35002736
:104190000E3400F30D3200C10D3100900D3000607F
:1041A0000D2E00320D2D00050D2C00D90C2B00AE6C
:1041B0000C2900850C29005C0C2700350C27000E0B
:1041C0000C2600E80B2400C40B2400A00B23007D68
:1041D0000B23005A0B2100390B2100180B2000F88B
:1041E0000A1F00D90A1E00BB0A1E009D0A1D00807E
:1041F0000A1D00630A1C00470A1B002C0A1B001141
:104200000A1A00F7091A00DD091900C4091900ABE0
:10421000091900920917007B091800630917004C5F
:1042200009160036091600200916000A091500F5BE
:10423000081500E0081400CC081400B8081400A405
:10424000081400900813007D0812006B0813005832
:104250000812004608120034081100230811001249
:1042600008110001081100F0071000E0071000D04D
:10427000071000C0071000B0070F00A10710009141
:10428000070E0083070F0074070F0065070E005725
:10429000070E0049070E003B070D002E070E0020F9
:1042A000070D0013070D0006070D00F9060C00EDC1
:1042B000060D00E0060C00D4060C00C8060C00BC7D
:1042C000060C00B0060C00A4060B0099060C008D2D
:1042D000060B0082060B0077060B006C060B0061D4
:1042E000060A0057060B004C060A0042060A003870
:1042F000060A002E060A0024060A001A060A001002
:1043000006090007060A00FD050900F4050900EB8F
:10431000050900E2050900D9050900D0050900C713
:10432000050900BE050900B5050800AD050800A592
:104330000509009C050800940508008C0508008408
:104340000508007C050800740508006C0507006579
:104350000508005D050700560508004E05070047E3
:104360000507004005080038050700310507002A49
:10437000050700230507001C050600160507000FAA
:104380000507000805060002050700FB040600F506
:10439000040700EE040600E8040600E2040700DB60
:1043A000040600D5040600CF040600C9040600C3B5
:1043B000040600BD040600B7040600B1040500AC05
:1043C000040600A6040600A00405009B0406009550
:1043D000040500900406008A040500850405008099
:1043E0000406007A04050075040500700405006BDE
:1043F00004050066040500610405005C040500571F
:10440000040500520405004D04050048040500435E
:104410000405003E0404003A04050035040500309C
:104420000404002C04050027040400230405001ED6
:104430000404001A04040016040500110404000D0D
:10444000040400090405000404040000040400FC42
:10445000030400F8030400F4030400F0030400EC78
:10446000030400E8030400E4030400E0030400DCA8
:10447000030400D8030400D4030400D0030400CCD8
:10448000030400C8030300C503030024F404D92077
:104490001BC40C5C0E9804C4095F0265077101F42B
:1044A00005F900FB04B30048048700C10369005804
:1044B00003550003034500BE023A00840231005355
:1044C000022A002902250004022000E4011C00C881
:1044D000011900AF01170098011400840113007145
:1044E0000110006101100051010E0043010D003662
:1044F000010B002B010B0020010B00150109000C22
:1045000001090003010800FB000800F3000800EBAC
:10451000000700E4000600DE000600D8000600D216
:10452000000600CC000500C7000500C2000500BD64
:10453000000400B9000400B5000400B1000400AD9F
:10454000000400A9000400A5000300A20003009FCE
:104550000004009B000300980003009500020093F4
:10456000000300900003008D0002008B0003008810
:104570000002008600020084000300810002007F28
:104580000002007D0002007B00020079000200773B
:104590000001007600020074000200720001007148
:1045A0000002006F0002006D0001006C0002006A52
:1045B000000100690002006700010066000100655B
:1045C000000100640002006200010061000100605F
:1045D0000001005F0002005D0001005C0001005B63
:1045E0000001005A00010059000100580001005765
:1045F0000001005600010055000100540001005365
:104600000000005300010052000100510001005061
:104610000001004F0001004E0000004E0001004D5F
:104620000001004C0001004B0000004B0001004A5B
:104630000001004900010048000000480001004757
:104640000001004600000046000100450000004552
:10465000000100440001004300000043000100424B
:104660000000004200010041000000410001004044
:104670000001003F0000003F0001003E0000003E3E
:104680000001003D0000003D0001003C0000003C36
:104690000000003C0001003B0000003B0001003A2C
:1046A0000000003A00010039000000390001003824
:1046B000000000380000003800010037000000371B
:1046C0000001003600000036000000360001003511
:1046D0000000003500000035000100340000003407
:1046E00000000034000100330000003300000033FC
:1046F00000010032000000320000003200010031F1
:1047000000000031000000310001003000000030E6
:10471000000000300001002F0000002F0000002FDB
:104720000000002F0001002E0000002E0000002ECF
:104730000001002D0000002D0000002D0000002DC4
:104740000001002C0000002C0000002C0000002CB8
:104750000001002B0000002B0000002B0000002BAC
:104760000001002A0000002A0000002A0000002AA0
:104770000001002900000029000000290000002994
:104780000000002900010028000000280000002887
:10479000000000280000002800010027000000277A
:1047A000000000270000002700000027000100266D
:1047B0000000002600000026000000260000002661
:1047C0000001002500000025000000250000002554
:1047D0000000002500000025000100240000002446
:1047E0000000002400000024000000240001002339
:1047F000000000230000002300000023000000232D
:10480000000000230000002300010022000000221D
:104810000000002200000022000000220000002210
:104820000001002100000021000000210000002103
:1048300000000021000000210000002100010020F4
:1048400000000020000000200000002000000020E8
:104850000000002000000020000000200001001FD8
:104860000000001F0000001F0000001F0000001FCC
:104870000000001F0000001F0001001E0000001EBD
:104880000000001E0000001E00000020204D3630F9
:104890003320003A0A0020286D6D290020530020A3
:1048A0005A0020590020580020204D34323520462F
:1048B000004261636B6C61736820636F6D70656E3D
:1048C000736174696F6E3A0A002055004C004669A6
:1048D0006C616D656E74206C6F61642F756E6C6FAA
:1048E0006164206C656E677468733A0A0020450045
:1048F000205A0020204D39303720580053746570FD
:10490000706572206D6F746F722063757272656E60
:1049100074733A0A0020204D393030204B004C6926
:104920006E65617220416476616E63653A0A0020AB
:10493000204D383531205A005A2D50726F62652053
:104940004F66667365740020440020490020204DA6
:1049500033303420500020440020490020204D33C3
:1049600030312050005049442073657474696E677B
:10497000733A0A0020460020420020480020204DC3
:104980003134352053004D6174657269616C206863
:10499000656174757020706172616D6574657273A4
:1049A0003A0A0020204D3432302053004175746F94
:1049B00020426564204C6576656C696E673A0A0032
:1049C000204500205A002059002058002054002083
:1049D000530020204D32303520420020453C6D618F
:1049E000785F655F6A65726B3E0020583C6D617848
:1049F0005F785F6A65726B3E20593C6D61785F79C4
:104A00005F6A65726B3E205A3C6D61785F7A5F6ABF
:104A100065726B3E00416476616E6365643A204264
:104A20003C6D696E5F7365676D656E745F74696D0B
:104A3000655F75733E20533C6D696E5F66656564A6
:104A4000726174653E20543C6D696E5F747261766C
:104A5000656C5F66656564726174653E0020540034
:104A600020520020204D32303420500041636365D5
:104A70006C65726174696F6E2028756E6974732F2E
:104A80007332293A20503C7072696E745F616363BF
:104A9000656C3E20523C726574726163745F616341
:104AA00063656C3E20543C74726176656C5F616333
:104AB00063656C3E0A00204500205A002059002002
:104AC000204D3230312058004D6178696D756D2070
:104AD000416363656C65726174696F6E2028756EE1
:104AE0006974732F7332293A0A00204500205A0056
:104AF00020590020204D3230332058004D61786914
:104B00006D756D20666565647261746573202875C6
:104B10006E6974732F73293A0A0053746570732099
:104B200070657220756E69743A0A0020204D313428
:104B3000392043203B20556E69747320696E2043F1
:104B4000656C736975730A0020204732312020207C
:104B5000203B20556E69747320696E206D6D00488E
:104B6000617264636F6465642044656661756C742A
:104B70002053657474696E6773204C6F616465645B
:104B80000A00282300002823000064000000E80336
:104B90000000000096430000964300000041000022
:104BA00020420000C9420000C9420000C844000081
:104BB000D243454550524F4D20496E697469616C2E
:104BC000697A65640A00290A002062797465733B7A
:104BD0002063726320002073746F726564207365B4
:104BE0007474696E67732072657472696576656442
:104BF000202800202863616C63756C6174656429EA
:104C0000210A0020213D2000454550524F4D2043B0
:104C10005243206D69736D61746368202D20287381
:104C2000746F7265642920002053697A653A200008
:104C3000496E6465783A2000204D61726C696E3D62
:104C4000563638290A00454550524F4D2076657238
:104C500073696F6E206D69736D6174636820284598
:104C60004550524F4D3D00290A002062797465730A
:104C70003B20637263200053657474696E67732010
:104C800053746F726564202800454550524F4D2083
:104C90006461746173697A65206572726F722E0A3D
:104CA0000050726F62696E67206661696C65640AA4
:104CB0000050726F62696E67206661696C6564009E
:104CC0005761726E696E673A20486F6D696E672032
:104CD00042756D702044697669736F72203C203193
:104CE0000A00020204486F6D652025732573257341
:104CF000206669727374002066697273740A0048D2
:104D00006F6D65200020746F6F206C6F6E6720657B
:104D10007874727573696F6E2070726576656E74E3
:104D200065640A0020636F6C642065787472757323
:104D3000696F6E2070726576656E7465640A002016
:104D4000453A00205A3A0020593A00583A000000EB
:104D5000F0410000F04100000041FF01010000A00F
:104D6000400000A040000000400000254300004B30
:104D7000430000244300000000CDCC3B4300001F53
:104D80004300002543CDCC3B4300001F43000000FF
:104D900000333373C10000A0C020746F6F206C6FAC
:104DA0006E6720657874727573696F6E20707265B6
:104DB00076656E7465640A0020636F6C64206578A4
:104DC00074727573696F6E2070726576656E746546
:104DD000640A00627573793A2070617573656420A6
:104DE000666F7220696E7075740A00627573793A25
:104DF0002070617573656420666F722075736572CB
:104E00000A00627573793A2070726F636573736913
:104E10006E670A004D3131372050726F6265207322
:104E200075636365737366756C0020496E76616C9B
:104E300069642065787472756465722000205A3A3E
:104E4000200020593A200042656420583A20005042
:104E5000726F6265205A204F66667365743A20004F
:104E60003F5A206F7574206F662072616E676520EF
:104E7000282D3220746F2035290A004D3134352019
:104E8000533C696E6465783E206F7574206F6620B0
:104E900072616E67652028302D31290A00436C69E4
:104EA000636B20746F20726573756D652E2E2E00F6
:104EB000220A00556E6B6E6F776E20636F6D6D61A9
:104EC0006E643A202200454550524F4D204F4B0A08
:104ED000004E6F206D6F76652E004543484F0049A8
:104EE0004E464F004552524F52530044525952556C
:104EF0004E00434F4D4D554E49434154494F4E008E
:104F00006F666600DA4EDF4EE44EEB4EF24E4445DD
:104F10004255473A004C756C7A426F74204D696E69
:104F200069204C4344204F46462E00205A00205909
:104F300000580020204D61783A2000205A00205966
:104F400000580020204D696E3A2000536F6674208F
:104F5000656E6473746F70733A2000256973002561
:104F6000696D20256973002569682025696D2025F4
:104F7000697300256964202569682025696D2025ED
:104F800069730025697920256964202569682025D1
:104F9000696D20256973005072696E742074696DA3
:104FA000653A20004D3131332053002F2F2000432C
:104FB00061703A004348414D4245525F54454D505F
:104FC00045524154555245004D4F54494F4E5F4D47
:104FD0004F44455300544845524D414C5F50524F49
:104FE00054454354494F4E004155544F5245504F3C
:104FF00052545F53445F5354415455530050524FE1
:105000004D50545F535550504F525400454D4552EA
:1050100047454E43595F5041525345520043415317
:10502000455F4C494748545F4252494748544E45B2
:10503000535300544F47474C455F4C4947485453DE
:1050400000534F4654574152455F504F5745520009
:105050004255494C445F50455243454E54004C45DF
:1050600056454C494E475F44415441005A5F5052A7
:105070004F4245004155544F4C4556454C00505207
:10508000494E545F4A4F420050524F475245535386
:10509000004155544F5245504F52545F54454D5066
:1050A00000564F4C554D45545249430045455052CA
:1050B0004F4D0042494E4152595F46494C455F545D
:1050C00052414E534645520053455249414C5F5858
:1050D0004F4E5F584F4646004649524D5741524544
:1050E0005F4E414D453A4D61726C696E20204649D4
:1050F000524D574152455F56455253494F4E3A32F1
:105100002E302E302E3135322045585452554445DC
:10511000525F545950453A53696E676C65457874CF
:1051200072756465724165726F563220534F5552E5
:1051300043455F434F44455F55524C3A6874747021
:10514000733A2F2F636F64652E616C6570686F62B0
:105150006A656374732E636F6D2F64696666757319
:10516000696F6E2F4D41524C494E2050524F544F53
:10517000434F4C5F56455253494F4E3A312E3020E3
:105180004D414348494E455F545950453A4C756C22
:105190007A426F74204D696E69204C434420455813
:1051A0005452554445525F434F554E543A31205561
:1051B0005549443A30383366363866312D30323806
:1051C000652D343934632D393865312D66326530BB
:1051D00064666165653961350A0020284E6F742068
:1051E000796574206D65617375726564290020208E
:1051F00041766572616765206D656173757265647E
:10520000206261636B6C61736820286D6D293A00C0
:105210002020536D6F6F7468696E6720286D6D294B
:105220003A20202020202020202020202020202064
:105230002020530020204261636B6C61736820441E
:10524000697374616E636520286D6D293A20202092
:10525000202020202000202846312E30203D2066AE
:10526000756C6C2C2046302E30203D206E6F6E65A4
:10527000290A002020436F7272656374696F6E2083
:10528000416D6F756E742F466164652D6F75743A4C
:10529000202020202046006163746976653A0A0068
:1052A000696E004261636B6C61736820436F727258
:1052B000656374696F6E2000205A002059002058E1
:1052C0000020506F736974696F6E616C2045727253
:1052D0006F723A0A002059002058004E6F7A7A6C9B
:1052E0006520546970204F757465722044696D653E
:1052F0006E73696F6E733A0A002020546F703A2003
:105300000020204261636B3A2000202046726F6EBD
:10531000743A2000202052696768743A20002020E7
:105320004C6566743A20004261636B6C6173683A45
:105330000A00205A0020590020580043656E746509
:10534000723A0A0020204261636B3A200020204616
:10535000726F6E743A2000202052696768743A2098
:105360000020204C6566743A20002020546F703A6B
:10537000200053696465733A0A00426564204C65F5
:1053800076656C696E6720004661696C656420749F
:105390006F20656E61626C6520426564204C6576A5
:1053A000656C696E670A00426564204C6576656CC1
:1053B00020436F7272656374696F6E204D61747201
:1053C00069783A000A0A426564204C6576656C206B
:1053D000436F7272656374696F6E204D6174726998
:1053E000783A00202B000A436F727265637465641B
:1053F00020426564204865696768742076732E20B2
:1054000042656420546F706F6C6F67793A0A0020B0
:105410002B000A4265642048656967687420546FF0
:10542000706F6772617068793A0A2020202B2D2DE9
:105430002D204241434B202D2D2B0A2020207C2063
:10544000202020202020202020207C0A204C207C8E
:1054500020202020282B29202020207C20520A20B8
:1054600045207C20202020202020202020207C205F
:10547000490A2046207C20282D29204E20282B292F
:10548000207C20470A2054207C202020202020201F
:10549000202020207C20480A2020207C2020202042
:1054A000282D29202020207C20540A2020207C2008
:1054B000202020202020202020207C0A2020204F77
:1054C0002D2D2046524F4E54202D2D2B0A202830B2
:1054D0002C30290A00202844525952554E290047A1
:1054E0003239204175746F20426564204C657665C1
:1054F0006C696E67003F20284C2C522C462C4229A8
:10550000206F7574206F6620626F756E64732E0A4B
:10551000003F50726F626520706F696E747320284F
:10552000592920697320696D706C61757369626CAB
:10553000652028322D32292E0A003F50726F626595
:1055400020706F696E747320285829206973206950
:105550006D706C61757369626C652028322D32291B
:105560002E0A003F2856296572626F7365206C65AC
:1055700076656C20697320696D706C617573696202
:105580006C652028302D34292E0A0043757272650F
:105590006E742066696C653A2000456E6420666909
:1055A0006C65206C6973740A00426567696E2066D9
:1055B000696C65206C6973740A00416476616E637E
:1055C00065204B3D003F4B2076616C7565206F7503
:1055D00074206F662072616E67652028302D31302F
:1055E000292E0A004D31313720486F7420456E64F2
:1055F0002048656174696E672E2E2E0A4D31303455
:1056000020533137302054300A473238204F310A86
:10561000473120593235205A31302046353030302C
:105620000A4D313137205265776970696E67206E97
:105630006F7A7A6C650A54300A4731205831313517
:1056400020593131352046353030300A4D3130392E
:1056500020523137302054300A4731205A310A471E
:1056600031205831313520593131352046343030F0
:10567000300A4731205834352059313734204634E8
:105680003030300A473120583131352059313135E9
:105690002046343030300A473120583435205931D3
:1056A00037342046343030300A47312058313135D4
:1056B00020593131352046343030300A47312058B6
:1056C000343520593137342046343030300A4731B0
:1056D0002058313135205931313520463430303081
:1056E0000A47312058343520593137342046343078
:1056F00030300A4731205831313520593131352089
:1057000046343030300A473120583435205931374B
:10571000342046343030300A47312058313135207A
:10572000593131352046343030300A473120583431
:105730003520593137342046343030300A47312053
:105740005A31350A4D31303620533235350A47301B
:105750002058302059300A4D3130392052313630FE
:105760002054300A4D313037004732380020466C23
:105770006F773A200020643A0020693A0020703A9E
:1057800000204500205A00205900204D3932205871
:105790000043290A0061626C656420286D696E20EF
:1057A00074656D70200064697300656E00436F6CF2
:1057B0006420657874727564657320617265200079
:1057C000205400205200416363656C657261746906
:1057D0006F6E3A205000496E76616C69642065787E
:1057E0007472756465720A0020643A0020693A0098
:1057F00020703A00536C6565702E2E2E0047322FB4
:1058000047332062616420706172616D65746572F6
:10581000730A0050726F6265205A204F6666736586
:10582000743A2000446F6E6520736176696E67205C
:1058300066696C652E0A00534420726561642065B8
:1058400072726F720A00446F6E65207072696E74B6
:10585000696E672066696C650A004D3239005354E1
:105860004F505045442E20005072696E746572206E
:1058700073746F707065642064756520746F206543
:1058800072726F72732E2046697820746865206585
:1058900072726F7220616E6420757365204D3939A4
:1058A0003920746F20726573746172742E202854CD
:1058B000656D7065726174757265206973207265BB
:1058C0007365742E20536574206974206166746555
:1058D000722072657374617274696E67290A004E72
:1058E0006F20436865636B73756D207769746820FA
:1058F0006C696E65206E756D6265722C204C6173EB
:1059000074204C696E653A20004E6F2043686563D1
:105910006B73756D2077697468206C696E65206E95
:10592000756D6265722C204C617374204C696E65D4
:105930003A2000636865636B73756D206D69736DE4
:10594000617463682C204C617374204C696E653AF5
:1059500020004C696E65204E756D6265722069731A
:10596000206E6F74204C617374204C696E65204EFC
:10597000756D6265722B312C204C617374204C69FB
:105980006E653A20004D31313000526573656E64AA
:105990003A20002042002050006F6B00220A006570
:1059A0006E7175657565696E6720220050494420E7
:1059B0004175746F74756E65206661696C656421EC
:1059C00020426164206578747275646572206E751A
:1059D0006D6265720A0042656420636F6F6C696E68
:1059E000672E2E2E004265642068656174696E67BB
:1059F0002E2E2E006F6B0047323858590020205051
:105A00006C616E6E65724275666665724279746528
:105A1000733A20002046726565204D656D6F72797E
:105A20003A2000436F6D70696C65643A2041756778
:105A300020203920323031390A00207C2041757411
:105A4000686F723A2028416C657068204F626A6501
:105A500063747320496E632E2C204C756C7A426FF0
:105A60007420476974205265706F7369746F72791E
:105A7000290A004175672020392032303139313010
:105A80003A32333A313200204C61737420557064DD
:105A9000617465643A2000322E302E302E3135325A
:105AA0000A004D61726C696E0020536F66747761F5
:105AB00072652052657365740A00205761746368CB
:105AC000646F672052657365740A002042726F77B5
:105AD0006E206F75742052657365740A00204578D6
:105AE0007465726E616C2052657365740A00506F44
:105AF00077657255700A0073746172740A004B49BD
:105B00004C4C45442E20005072696E7465722068BA
:105B1000616C7465642E206B696C6C28292063614C
:105B20006C6C6564210A004B494C4C2063617573B1
:105B30006564206279204B494C4C20627574746F07
:105B40006E2F70696E0A004B494C4C20636175736F
:105B5000656420627920746F6F206D7563682069B9
:105B60006E6163746976652074696D65202D2063AC
:105B7000757272656E7420636F6D6D616E643A202C
:105B8000004D3132310A4730205A31300A4732381D
:105B90002058302059300A4731320A4D31303920EF
:105BA000523136300A4D3131372050726F62696E92
:105BB00067206265640070726F62655F7265776905
:105BC00070650050726F62696E67206661696C650E
:105BD00064004D31313720426564206C6576656C18
:105BE000696E67206661696C65642E0A4730205AC9
:105BF00031300A47302045300A4D333030205032A2
:105C00003520533838300A4D33303020503530206D
:105C100053300A4D3330302050323520533838302D
:105C20000A4D333030205035302053300A4D333058
:105C3000302050323520533838300A473420533121
:105C40000070726F62655F6661696C6564005072B6
:105C50006F7465637465642050696E0A0025301D99
:105C60000C1E282924311C0B184527232F1B0A172B
:105C70004443222B1A4142043803FF360408060627
:105C800000017B4659877C9168A7B3C2E000E2001F
:105C9000E400E6009C9111241FBECFEFD1E2DEBFED
:105CA000CDBF00E00CBF14E0A0E0B2E0E6ECFBEBFF
:105CB00002E00BBF02C007900D92AE33B107D9F7D7
:105CC00027E1AEE3B4E001C01D92A330B207E1F7D3
:105CD0001EE2CAE4DEE200E006C021970109802F3F
:105CE000FE010F949755C134D10780E00807A9F74A
:105CF0000E94B73A0D94D15D0C9400001F920F9250
:105D00000FB60F9211242F933F938F939F93AF93CE
:105D1000BF9380913F0490914004A0914104B091C1
:105D2000420430913E0423E0230F2D3720F40196E6
:105D3000A11DB11D05C026E8230F0296A11DB11DAE
:105D400020933E0480933F0490934004A093410429
:105D5000B09342048091430490914404A09145047F
:105D6000B09146040196A11DB11D80934304909308
:105D70004404A0934504B0934604BF91AF919F9112
:105D80008F913F912F910F900FBE0F901F901895FC
:105D90002FB7F89460913F047091400480914104C2
:105DA000909142042FBF08953FB7F8948091430427
:105DB00090914404A0914504B091460426B5A89B57
:105DC00005C02F3F19F00196A11DB11D3FBFBA2F8D
:105DD000A92F982F8827820F911DA11DB11DBC01ED
:105DE000CD0142E0660F771F881F991F4A95D1F7B2
:105DF00008958F929F92AF92BF92CF92DF92EF92CF
:105E0000FF926B017C01D0DF4B015C01C114D10416
:105E1000E104F104F1F09CD3C7DFDC01CB01881968
:105E20009909AA09BB09883E9340A105B10570F301
:105E300021E0C21AD108E108F10888EE880E83E05B
:105E4000981EA11CB11CC114D104E104F10421F776
:105E5000DDCFFF90EF90DF90CF90BF90AF909F90FD
:105E60008F9008958230910538F0880F991F880F20
:105E7000991F05970197F1F70895789484B582608A
:105E800084BD84B5816084BD85B5826085BD85B5DE
:105E9000816085BDEEE6F0E0808181608083E1E88D
:105EA000F0E01082808182608083808181608083C5
:105EB000E0E8F0E0808181608083E1EBF0E08081C8
:105EC00084608083E0EBF0E0808181608083E1E9A1
:105ED000F0E0808182608083808181608083E0E95E
:105EE000F0E0808181608083E1EAF0E0808182607F
:105EF0008083808181608083E0EAF0E0808181603E
:105F00008083E1E2F1E08081826080838081816032
:105F10008083E0E2F1E0808181608083EAE7F0E065
:105F200080818460808380818260808380818160C1
:105F300080838081806880831092C10008951F93C0
:105F4000CF93DF93182FEB0161E016D1209711F466
:105F500060E004C0CF3FD10531F461E0812FDF91D3
:105F6000CF911F9145C1E12FF0E0E55FFD4FE49136
:105F70004E2F50E0FA013197E231F10508F09DC053
:105F80008827EE58FF4F8F4F0D94975584B5806842
:105F900084BDC7BD97C084B5806284BDC8BD92C0B2
:105FA00080918000806880938000D0938900C093A6
:105FB000880088C080918000806280938000D093A8
:105FC0008B00C0938A007EC080918000886080939F
:105FD0008000D0938D00C0938C0074C08091B0007D
:105FE00080688093B000C093B3006CC08091B00013
:105FF00080628093B000C093B40064C08091900030
:10600000806880939000D0939900C09398005AC004
:1060100080919000806280939000D0939B00C09309
:106020009A0050C080919000886080939000D09337
:106030009D00C0939C0046C08091A0008068809322
:10604000A0008091A0008F7B8093A000D093A90036
:10605000C093A80037C08091A00080628093A00008
:10606000D093AB00C093AA002DC08091A00088609F
:106070008093A000D093AD00C093AC0023C080916A
:106080002001806880932001D0932901C0932801CA
:1060900019C080912001806280932001D0932B0150
:1060A000C0932A010FC08091200188608093200155
:1060B000D0932D01C0932C0105C0C038D1050CF040
:1060C0004CCF46CFDF91CF911F91089590E0FC0116
:1060D0003197E231F10508F04EC08827EC57FF4FA9
:1060E0008F4F0D949755809180008F7703C08091DA
:1060F00080008F7D80938000089580918000877F4D
:10610000F9CF84B58F7702C084B58F7D84BD0895A3
:106110008091B0008F7703C08091B0008F7D809315
:10612000B0000895809190008F7707C08091900013
:106130008F7D03C080919000877F809390000895A9
:106140008091A0008F7707C08091A0008F7D03C051
:106150008091A000877F8093A00008958091200106
:106160008F7707C0809120018F7D03C0809120012F
:10617000877F809320010895CF93DF9390E0FC0107
:10618000EF5AFD4F2491FC01E956FD4F849188237D
:1061900061F190E0880F991FFC01EF5EFC4FC59103
:1061A000D491FC01E950FD4FA591B491611109C052
:1061B0009FB7F8948881209582238883EC912E23C1
:1061C0000BC0623061F49FB7F8943881822F8095BC
:1061D00083238883EC912E2B2C939FBF06C08FB70F
:1061E000F894E8812E2B28838FBFDF91CF910895FB
:1061F0001F93CF93DF93282F30E0F901E55FFD4F28
:106200008491F901EF5AFD4FD491F901E956FD4F00
:10621000C491CC23C1F0162F811158DFEC2FF0E090
:10622000EE0FFF1FE950FD4FA591B4918FB7F89481
:10623000111105C09C91ED2FE095E92302C0EC916E
:10624000ED2BEC938FBFDF91CF911F910895CF93EA
:10625000DF93282F30E0F901E55FFD4F8491F901CC
:10626000EF5AFD4FD491F901E956FD4FC491CC236B
:1062700089F081112BDFEC2FF0E0EE0FFF1FE352CE
:10628000FD4FA591B491EC91ED2381E090E021F4D4
:1062900080E002C080E090E0DF91CF910895089502
:1062A0001F920F920FB60F9211240BB60F922F93DD
:1062B0003F934F935F936F937F938F939F93AF938E
:1062C000BF93EF93FF93E0910802F09109021995B3
:1062D000FF91EF91BF91AF919F918F917F916F91BE
:1062E0005F914F913F912F910F900BBE0F900FBE7A
:1062F0000F901F9018951F920F920FB60F921124B6
:106300000BB60F922F933F934F935F936F937F93AF
:106310008F939F93AF93BF93EF93FF93E0910A0204
:10632000F0910B021995FF91EF91BF91AF919F9161
:106330008F917F916F915F914F913F912F910F902E
:106340000BBE0F900FBE0F901F9018951F920F92CB
:106350000FB60F9211240BB60F922F933F934F93CA
:106360005F936F937F938F939F93AF93BF93EF93BD
:10637000FF93E0910C02F0910D021995FF91EF91BE
:10638000BF91AF919F918F917F916F915F914F914D
:106390003F912F910F900BBE0F900FBE0F901F904B
:1063A00018951F920F920FB60F9211240BB60F92F1
:1063B0002F933F934F935F936F937F938F939F930D
:1063C000AF93BF93EF93FF93E0910E02F0910F0212
:1063D0001995FF91EF91BF91AF919F918F917F910F
:1063E0006F915F914F913F912F910F900BBE0F9046
:1063F0000FBE0F901F9018951F920F920FB60F921D
:1064000011240BB60F922F933F934F935F936F938B
:106410007F938F939F93AF93BF93EF93FF93E091FD
:106420000402F09105021995FF91EF91BF91AF9190
:106430009F918F917F916F915F914F913F912F919C
:106440000F900BBE0F900FBE0F901F9018951F92CC
:106450000F920FB60F9211240BB60F922F933F930A
:106460004F935F936F937F938F939F93AF93BF935C
:10647000EF93FF93E0910602F09107021995FF91C7
:10648000EF91BF91AF919F918F917F916F915F91AC
:106490004F913F912F910F900BBE0F900FBE0F9019
:1064A0001F9018951F920F920FB60F9211240BB6E2
:1064B0000F922F933F934F935F936F937F938F939D
:1064C0009F93AF93BF93EF93FF93E0911002F091EE
:1064D00011021995FF91EF91BF91AF919F918F910B
:1064E0007F916F915F914F913F912F910F900BBED4
:1064F0000F900FBE0F901F9018951F920F920FB61E
:106500000F9211240BB60F922F933F934F935F93EB
:106510006F937F938F939F93AF93BF93EF93FF936B
:10652000E0911202F09113021995FF91EF91BF9142
:10653000AF919F918F917F916F915F914F913F911B
:106540002F910F900BBE0F900FBE0F901F901895BC
:1065500008951F93CF93DF93EC011D821C821F824D
:106560001E82198681E0888782E28A871F861E86BE
:10657000FE01B396CE01C1962FEF2193E817F907DC
:10658000E1F711E018A3CE0122D61F8B188E198EC9
:1065900080E48A8F1B8E88EB96E39AAB89ABDF9100
:1065A000CF911F910895DB01ED91FC911994EF9229
:1065B000FF921F93CF93DF931F921F92CDB7DEB749
:1065C0007C01DC01D196ED91FC91D29782E0698348
:1065D0007A83199520E030E04AE069817A81C70129
:1065E000E2DF182FD701D196ED91FC91D29783E08D
:1065F0001995D701D196ED91FC91D29780E019952C
:10660000812F0F900F90DF91CF911F91FF90EF900E
:1066100008950F931F93CF93DF93EC018B01E9A9AA
:10662000FAA982E01995E9A9FAA981E0199520E073
:1066300030E044E1B801CE01B6DF9E012D5C3F4F52
:1066400047E1B801CE01AFDFE9A9FAA980E0DF9107
:10665000CF911F910F911994EF92FF921F93CF93B7
:10666000DF93EC017B01E9A9FAA982E01995E9A978
:10667000FAA981E0199520E030E045E1B701CE01AB
:1066800092DF182F882339F09E012D5C3F4F47E1A0
:10669000B701CE0188DFE9A9FAA980E01995812F19
:1066A000DF91CF911F91FF90EF900895FC01448FEF
:1066B000258F9C01245E3F4F42E375CFCF93DF933C
:1066C0001F92CDB7DEB79E012F5F3F4F46E46BDFD1
:1066D00089810F90DF91CF910895CF93DF931F921F
:1066E000CDB7DEB79E012F5F3F4F47E45CDF898166
:1066F0000F90DF91CF91089520E030E048E453CF30
:10670000CF93DF93EC016A817B81D8DF88836A8134
:106710007B81CE01E2DF89836A817B81CE01ECDF60
:106720008B879E012D5C3F4F6A817B8147E1CE01C3
:10673000DF91CF9138CFCF93DF93EC016A817B81DA
:1067400036DF882319F0CE01DBDF81E0DF91CF91C6
:1067500008958F929F92AF92BF92CF92EF920F9334
:10676000CF93DF931F921F92CDB7DEB74C015B0131
:106770002A834983EEDEF401B382A282498147A3D2
:106780002A8120A705A3E4A2C3A2C4010F900F9001
:10679000DF91CF910F91EF90CF90BF90AF909F90EE
:1067A0008F90C9CFFC016281738133CFCF93DF9388
:1067B000EC01EE85FF85309709F019956A817B81A0
:1067C000CE01DF91CF9148CF362F242FFC0162817B
:1067D0007381432F6BCF0F93FC0182819381648F70
:1067E000458F278F068F9F01245E3F4F4BE3BC01EF
:1067F000CF010F91D8CEFC0160A30895BF92CF9234
:10680000DF92EF92FF920F931F93CF93DF936C0170
:10681000D62FB42EC22F7801CC2369F0F701049152
:1068200020E04B2D6D2FC601D6DFFFEFEF1AFF0AD8
:10683000C150D85FF1CFDF91CF911F910F91FF90A1
:10684000EF90DF90CF90BF9008958F929F92AF927C
:10685000BF92CF92DF92EF92FF920F931F93CF934D
:10686000DF935C01C62EC42FD22ED02F220F220F11
:10687000220F1ED0882379F0DC0F8D2C912CCD17A0
:1068800051F087012D2D4C2F6C2DC501B7DFE80C81
:10689000F91CCF5FF4CFDF91CF911F910F91FF9043
:1068A000EF90DF90CF90BF90AF909F908F90089522
:1068B0000F93FC010150040F84A996A9941718F0B6
:1068C000081728F402C0081750F0041740F42150AC
:1068D000260F83A995A9961720F4281720F480E0A5
:1068E00007C0281720F481E0261710F0F8CF81E0C8
:1068F0000F91089581E008952EE93FE0009729F077
:10690000F9013197F1F70197F9CF0895FC0112824F
:1069100080818150838314820895FC01808192815B
:10692000980F92832181921760F494819F5F9483E2
:106930009381890F821710F08FEF820F838381E09C
:10694000089580E00895FC0191E08381861708F4A2
:1069500090E031E0461708F030E0832F892B21E0EA
:106960005281451708F420E02823832F8923822BA6
:106970000895DC01FB01108212968C91129781839D
:1069800015968C9115978150828313968C918383F1
:106990000895FB0141812381213029F0233031F416
:1069A00068EF640F04C0642F485F01C0642FCBCF31
:1069B000DC0115962C9115971696ED91FC91179781
:1069C000CF01820F911D820F911D1192E817F907D7
:1069D000E1F70895FC01A681B7818281481B85817A
:1069E000483018F0A80FB11D4770382F36953695EE
:1069F0003695562F577080E890E002C095958795A0
:106A00005A95E2F7439F402D112466956695669549
:106A1000E62FF0E0E40FF11DEA0FFB1F3081222387
:106A200011F0832B02C08095832380830895FB019E
:106A30004181DC0112962C911297421760F0139657
:106A40002C911397241738F0608115962C916217BA
:106A500010F42481BFCF0895CF92DF92FF920F935D
:106A60001F93CF93DF936C01EB01FA809B819130F0
:106A700051F030F0923049F0933051F41FEF09C0DB
:106A800010E001E007C011E004C010E00FEF02C009
:106A900010E000E0F7FE03C0BE01C601C8DF988128
:106AA000900F98839981910F9983FF0C99F7DF914B
:106AB000CF911F910F91FF90DF90CF9008950F938A
:106AC0001F93CF93DF938901FB01C281D3814233AE
:106AD000D9F058F44531E1F0473109F1443141F53D
:106AE000CE0166DFCE0112DF23C04634E1F0473429
:106AF000E1F04B33E9F4B901CE014BDF8823C1F05B
:106B0000B801CE01A9DF14C0B901CE0190DF10C0D9
:106B1000CE0103DF882369F0CE014ADF09C0B90145
:106B2000CE0127DF05C08D8101C08981F8018083F6
:106B300081E0DF91CF911F910F910895CF92DF9265
:106B4000EF92FF920F931F93CF93DF937C01D62F89
:106B5000D42EC22F122FC62EC20E6C2D611B1830E0
:106B600038F00FEF20E04D2DC70135DE1850F5CF7E
:106B70006C2F687F6D0F2C2F277071F097E02927FD
:106B80002F5F27700FEF10E001C0000F2A95EAF782
:106B900020E04D2DC7011FDEDF91CF911F910F9196
:106BA000FF90EF90DF90CF900895CF92DF92EF9219
:106BB000FF920F931F93CF93DF937C01D62ED42F98
:106BC000C22F122FC42EC20E4C2D411B183038F08C
:106BD0000FEF21E06D2DC701FEDD1850F5CF4C2FD2
:106BE000487F4D0F2C2F277071F097E029272F5FDA
:106BF00027700FEF10E001C0000F2A95EAF721E09F
:106C00006D2DC701E8DDDF91CF911F910F91FF90AE
:106C1000EF90DF90CF900895EF92FF920F931F9324
:106C2000CF93DF93EC01162FF42EE22E01E040DE2D
:106C3000882359F02E2D4F2D612FCE01DF91CF915A
:106C40001F910F91FF90EF9079CFDF91CF911F911E
:106C50000F91FF90EF900895EF92FF920F931F9383
:106C6000CF93DF93EC01162FF42EE22E022F21E0BA
:106C70001FDE882359F02E2D4F2D612FCE01DF917D
:106C8000CF911F910F91FF90EF908FCFDF91CF9118
:106C90001F910F91FF90EF900895DF92EF92FF9276
:106CA0000F931F93CF93DF937C01162FC42FD22E07
:106CB000D02FFEDD8823F9F02D2D4C2F612FC70139
:106CC0003DDF2D2F4C2F612FC7016FDF6FEF6D0D53
:106CD000610F2D2F4C2FC70168DF4FEF4D0F4C0F69
:106CE0002D2D612FC701DF91CF911F910F91FF9043
:106CF000EF90DF9023CFDF91CF911F910F91FF9005
:106D0000EF90DF900895EF92FF920F931F93CF9330
:106D1000DF937C01D62F122FC42F040F212F4C2F6D
:106D20006D2FC7010BDFCF5F0C13F8CFDF91CF9131
:106D30001F910F91FF90EF900895DF92EF92FF92D5
:106D40000F931F93CF93DF93EC01162FF42EE22EB7
:106D5000AFDD882329F02E2D4F2D612FCE01D3DFFB
:106D6000DF91CF911F910F91FF90EF90DF900895E9
:106D70000895FC01E60FF11D849190E0982F88277B
:106D80003196E4918E0F911D0895FC018491089530
:106D9000FCDF882321F0823011F083E0089586E043
:106DA000089580E00895FC018081089566E0E1CFB8
:106DB00068E0DFCF0A96FC01849108950B96FC01F0
:106DC00084910895DC011496ED91FC91159731960C
:106DD00084910895BF92CF92DF92EF92FF920F932A
:106DE0001F93CF93DF938C01E62EDC011496CD9197
:106DF000DC911597CE01C9DFF82EF80184819581C9
:106E0000C7DFC82EF1E0FF1203C02FE0B22E02C090
:106E1000BB24BA94D80114968D919C911597CADF22
:106E2000F82EF80184819581C9DFD82ED8011496F7
:106E30008D919C911597BCDFB0E6BE1538F4009794
:106E400029F0C80FD91F91E6F92E0FC0F8018481EF
:106E50009581ACDFF0E4FE1538F4009729F0C80FF7
:106E6000D91F81E4F82E01C06196DE1490F4D80198
:106E700050961C92509753961C92539754961C927E
:106E8000549751961C92519752961C9280E090E034
:106E900066C0DF1460F38C2D90E0FE0124912F3F3B
:106EA00011F4219657C0FE104CC0D80114968D9154
:106EB0009C9115976ADF9E012F5F3F4FFE0188234B
:106EC00011F08230E1F48491D80153968C9353975A
:106ED000F901249154962C935497FE013396E49132
:106EE0005096EC935097FE013496E4915196EC93B2
:106EF0005197FE013596E4915296EC9320C084910F
:106F0000982F9F709250D80152969C9352978295D9
:106F10008F7051968C935197F9012491822F8F7025
:106F200054968C93549722952F7053962C93539785
:106F3000FE013296E491E295EF705096EC93CE010B
:106F40000EC0FE013296E491EB219C012E0F311D03
:106F5000C20FD31FFD1409F48ACFF3949ECFDF91A3
:106F6000CF911F910F91FF90EF90DF90CF90BF9046
:106F700008954F925F926F927F929F92AF92BF92CD
:106F8000CF92DF92EF92FF920F931F93CF93DF93F5
:106F90001F92CDB7DEB72C01C62E942E622F1ADFBA
:106FA0007C01892B09F43AC0F20184819581F0DEDD
:106FB000B82EF201138904898189C80E8289981A32
:106FC000D92CD01A212F4D2D6C2DC20171DC8823B4
:106FD00011F1EB0CF11C195F169516951695612EA3
:106FE000712CD914C1F03C2D57018A2D8E198117AF
:106FF00070F4F501049120E04D2D632FC201398317
:10700000EADBFFEFAF1ABF0A3981385FEECFE60C3B
:10701000F71CD394E6CFF201808901C080E00F9085
:10702000DF91CF911F910F91FF90EF90DF90CF9064
:10703000BF90AF909F907F906F905F904F9008951A
:107040000F931F93CF93DF9300D0CDB7DEB78C01A2
:10705000DC015596ED91FC9156972B834A83698309
:1070600019954A81480F2B816981C8010F900F90B3
:107070000F90DF91CF911F910F917BCFAF92BF9275
:10708000DF92EF92FF920F931F93CF93DF931F92A4
:107090001F92CDB7DEB77C01D62E042FDC015596AA
:1070A000ED91FC91569729833A831995080F298110
:1070B000A22E3A81B32E10E0F50121915F01222327
:1070C00039F0402F6D2DC70154DFD80E180FF4CFC3
:1070D000812F0F900F90DF91CF911F910F91FF9013
:1070E000EF90DF90BF90AF900895DF92EF92FF9204
:1070F0000F931F93CF93DF937C01D62FD42E89015A
:10710000DC015596ED91FC9156971995D80EC0E08B
:10711000F8012491222349F04D2D6D2FC70129DF5D
:10712000D80FC80F0F5F1F4FF3CF8C2FDF91CF9178
:107130001F910F91FF90EF90DF900895DC0114965E
:107140002D913C9115972115310509F43FC05796B3
:107150008C915797F901811108C03596E4915896A2
:10716000EC935897F9013C9611C0813041F43F9659
:10717000E4915896EC935897F901709607C03D96A4
:10718000E4915896EC935897F9013E96E4915996FC
:10719000EC93599758968C915897082E000C990BA0
:1071A00059962C915997821B910927FD93955A96D0
:1071B0002C915A97203441F0829FC001112426E07F
:1071C000969587952A95E1F75B968C93089521ED26
:1071D00036E3FC01368B258B0895CF92DF92EF9238
:1071E000FF920F931F93CF93DF938C017B016A0172
:1071F000CB01FA011995D82F882311F1682FC80106
:10720000E9DDF801C189C195FFEFEF1AFF0AC70157
:10721000F6011995F801882351F08089C80FC7013C
:10722000F6011995D82F682FC801D4DDEDCFD032E3
:1072300021F091898389890F01C080898C0F01C059
:1072400080E0DF91CF911F910F91FF90EF90DF9041
:10725000CF90089543ED56E3C0CFCF93DF93FC0169
:10726000248135812617370741F0EC01758364834B
:1072700065DF81ED96E39E8B8D8BDF91CF91089535
:10728000CF93DF9300D01F92CDB7DEB761157105A4
:107290008105910579F09B01AC0169833A834B83A9
:1072A0005C830F940D5629813A814B815C810F9448
:1072B0007B5503C060E070E0CB010F900F900F9002
:1072C0000F90DF91CF910895CF92DF92EF92FF92CE
:1072D0000F931F9362177307840795077CF4890146
:1072E0009A016B017C01C901B8016C197D098E09F5
:1072F0009F09C6DF6C0D7D1D8E1D9F1D1F910F9177
:10730000FF90EF90DF90CF9008954F925F926F9231
:107310007F92AF92BF92CF92DF92EF92FF920F9344
:107320001F93CF93DF93CDB7DEB729013A019B01BD
:10733000AC0124193509460957098A899B89AC890A
:10734000BD89BC01CD016A197B098C099D090F9487
:107350001755A801970124193509460957090F94B3
:107360007B55CA01B9016A0D7B1D8C1D9D1DDF91E6
:10737000CF911F910F91FF90EF90DF90CF90BF9032
:10738000AF907F906F905F904F90089580E090E075
:1073900008950895CF92DF92EF92FF920F931F937B
:1073A000CF93DF936C017A018B01C0E0D0E0CE1562
:1073B000DF0589F0D8016D918D01D601ED91FC9129
:1073C0000190F081E02DC6011995892B11F47E0101
:1073D00002C02196ECCFC701DF91CF911F910F9191
:1073E000FF90EF90DF90CF9008956115710579F0CF
:1073F000FB0101900020E9F73197AF01461B570BC5
:10740000DC01ED91FC910280F381E02D199480E084
:1074100090E00895DC01ED91FC910190F081E02D68
:1074200019944F925F926F927F92EF92FF920F9317
:107430001F93CF93DF93CDB7DEB7A1970FB6F89424
:10744000DEBF0FBECDBF7C01FA01CB0119A22230F5
:1074500008F42AE08E010F5D1F4F422E512C612C43
:10746000712CBF01A30192010F945955F901CA0172
:10747000015011096A3014F4605D01C0695CD801E3
:107480006C93232B242B252B61F7B801C701ADDFAB
:10749000A1960FB6F894DEBF0FBECDBFDF91CF919E
:1074A0001F910F91FF90EF907F906F905F904F90A2
:1074B0000895CF92DF92EF92FF920F931F93CF9395
:1074C000DF93EC016A017B012115310579F4E88134
:1074D000F9810190F081E02D642FDF91CF911F9110
:1074E0000F91FF90EF90DF90CF9019942A303105E3
:1074F000D9F477FF18C06DE28DDF8C014427552742
:10750000BA014C195D096E097F092AE0CE0189DFB5
:10751000800F911FDF91CF911F910F91FF90EF90FE
:10752000DF90CF9008952AE0B701A601CE01DF9148
:10753000CF911F910F91FF90EF90DF90CF9071CF7F
:107540009A01AB01770F660B770BB3CFCF92EF9217
:107550000F93FC0113AE14AE15AE0496FAD80F913A
:10756000EF90CF90089580E090E0089508950E94F4
:107570003D2FFCDF0F947D50C0E0D0E00F940B5105
:107580002097E1F30E940000F9CFE8E6F4E083AF32
:1075900064AF08954AE050E0BC0188E694E0D0CFA3
:1075A000EF92FF920F931F93CF93DF937A016F3F78
:1075B00071058105910509F048F488E694E02ADF19
:1075C0008CE694E0FFDB282F30E014C0C091A304C8
:1075D000D091A4044D2F50E0EC2FF0E08B019C01E2
:1075E000BF018CE694E04CD6C80FC093A304D0939F
:1075F000A4049C01C901DF91CF911F910F91FF90CD
:10760000EF900895EF92FF920F931F93CF93DF9324
:107610008B01C8E6D4E0FBACECAC4E2D50E06F2DF6
:1076200070E09C018CE694E083D6F80EFBAEECAEE5
:10763000DF91CF911F910F91FF90EF900895EF92FE
:10764000FF920F931F93CF93DF938B01C8E6D4E093
:10765000FBACECAC4E2D50E06F2D70E09C018CE645
:1076600094E0B2D6F80EFBAEECAEDF91CF911F9155
:107670000F91FF90EF9008956FEF7FEFC3CF4FEF23
:107680005FEF8ECF0F931F93CF93DF931F92CDB7F2
:10769000DEB7082F84EA96E00E94C37F182F863158
:1076A00068F484EA96E0E8DF153109F43DC060E251
:1076B00070E080E090E0E3DF1F5FF6CFCE0101963F
:1076C0000E94788360E870E09DDF8981853120F534
:1076D0006EE270E080E090E0D2DF19811431E1F0D9
:1076E0006EE270E080E090E0CADF1331A9F089819A
:1076F0002EEF3FEF281B310986E0829FB001839F68
:10770000700D112460587F4F84EA96E07BDF60E2C1
:1077100070E080E090E0B3DF80914704801721F0B3
:10772000009347040E945A830F90DF91CF911F91DD
:107730000F9108954F925F926F927F928F929F92D6
:10774000AF92BF92CF92DF92EF92FF920F931F936F
:10775000CF93DF93CDB7DEB72D970FB6F894DEBF8A
:107760000FBECDBF80919A06882309F48AC060912C
:107770000F0D7091100D072E000C880B990B0F94B4
:10778000B15211E020910B0D30910C0D40910D0D77
:1077900050910E0D0F94125418160CF010E06091D9
:1077A000EB0C7091EC0C072E000C880B990B0F94CE
:1077B000B1522091E70C3091E80C4091E90C5091C6
:1077C000EA0C0F94125418160CF4106810935A0413
:1077D000C0906902D0906A02E0906B02F0906C0257
:1077E00020E030E0A901C701B6010F940F5287FDD8
:1077F00005C020E030E040E05FE304C020E030E07E
:1078000040E05FEBC701B6010F9436510F947E52F2
:10781000CB010F94C545BC0185E594E00F94885ACF
:10782000C0906D02D0906E02E0906F02F0907002F6
:1078300020E030E0A901C701B6010F940F5287FD87
:1078400005C020E030E040E05FE304C020E030E02D
:1078500040E05FEBC701B6010F9436510F947E52A2
:10786000CB010F94C545BC0180E594E00F94885A84
:1078700081E792E00F94D74ABC0188E494E00F942A
:10788000885A0E940282182F81E05FD620915A0404
:1078900027FF03C048E00CE002C042E102E0809113
:1078A000A00490E044977CF48091A204841758F0DF
:1078B00027FD37C180E596E17C0123E060E58CE699
:1078C00094E00E9425348091A0048431B8F4809122
:1078D000A204823098F0112309F426C18091060D8C
:1078E000882309F421C180EC95E17C0102E123E0C9
:1078F00042E068E68CE694E00E9425348091A00482
:107900008C31D0F590915A0480900B0D90900C0D15
:10791000A0900D0DB0900E0DC0900F0DD090100DD9
:10792000843128F48091A204883008F03AC2809112
:10793000A004883008F415C28091A0048C3108F4AA
:1079400017C28090E70C9090E80CA090E90CB090E2
:10795000EA0C8091EB0C9091EC0C2091A004283063
:1079600008F40CC28091A0048C3108F40EC28091FE
:10797000A0048C3108F40FC280917E0983FF27C0D8
:107980008091AE07882319F18091A0048433F8F424
:107990008091A2048A32D8F007E028E04AE26AE245
:1079A0008CE694E0CAD905E022E04CE262E38CE682
:1079B00094E0C3D904E02AE041E36AE28CE694E073
:1079C0006CD94BE262E38CE694E00E94E433809150
:1079D000A004853328F48091A204813308F0A7C065
:1079E0000E942787823048F09091A004943328F4B5
:1079F0009091A204923308F0A2C08091A0048F322B
:107A000008F05EC08091A204883208F459C00F9437
:107A10009E4C2B013C018CE3C82ED12CE12CF12C87
:107A2000C301B201A70196010F945955CA01B901CA
:107A3000A70196010F945955CA01062FD72E590157
:107A4000AE014F5F5F4F7A0150E8451651E555068C
:107A500051E06506710408F48CC0B90128E130E0FA
:107A600040E050E00F94595529013A01DF920F93FD
:107A7000C50168E170E00F9432559F938F935F9238
:107A80004F9282EB95E19F938F93FF92EF920F9429
:107A9000B75A0FB6F894DEBF0FBECDBF5AE04516F9
:107AA00051046104710408F08EC098E0892F880F9A
:107AB000980F892F81956FE2855A67DDC701DCDD5C
:107AC0008091A0048632A0F48091A2048E3180F0CF
:107AD00008E020E84EE160E08CE694E02ED9809149
:107AE000A004863228F48091A2048F3108F06DC082
:107AF0008091A004823328F48091A2048B3208F094
:107B000014C18091A004813408F040C28091A20485
:107B1000873308F43BC26EE380E037DD812FB2DDAE
:107B200035C28CE296E1C8CE86EF95E1DECE04E068
:107B30002AE441E366E38CE694E0AFD851CFF8E461
:107B40008F9FB0011124072E000C880B990B0F9406
:107B5000B1522AE037ED43E25CE30F944D540F94A9
:107B60008352262F02E042E367E38CE694E0E5D8F7
:107B700044CF84E6A816B10498F4DF920F933F93A4
:107B80002F9388EA95E19F938F93FF92EF920F9442
:107B9000B75A0FB6F894DEBF0FBECDBF95E086CFC3
:107BA000DF920F933F932F9380EA95E19F938F93FA
:107BB000FF92EF920F94B75A0FB6F894DEBF0FBE44
:107BC000CDBF96E073CF99E071CF60E08CE694E092
:107BD0000E94FB3365E283E0D8DC68E570E080E07A
:107BE00090E04DDD65E28BE0D0DC112321F085E5EE
:107BF00094E042DD24C08091D10D80FD17C035E5B1
:107C0000E32E34E0F32EF70161917F016623B9F092
:107C10006F3234F4062E000C770B880B990B04C0DE
:107C20006FE370E080E090E02ADDEDCF8091D00D31
:107C300080FDDDCF6FEF7FEF83E995E100DD65E249
:107C400088E2A3DC69E570E080E090E018DD65E2A1
:107C500080E39BDC112321F080E594E00DDD26C05C
:107C60008091D10D869580FD17C020E5E22E24E09D
:107C7000F22EF70161917F016623C1F06F3234F477
:107C8000062E000C770B880B990B04C06FE370E095
:107C900080E090E0F4DCEDCF8091D00D869580FD02
:107CA000DBCF6FEF7FEF83E995E1C9DC65E28DE41F
:107CB0006CDC6AE570E080E090E0E1DC65E285E59F
:107CC00064DC112321F088E494E0D6DC28C08091A4
:107CD000D10D8695869580FD17C098E4E92E94E035
:107CE000F92EF70161917F016623C9F06F3234F4F8
:107CF000062E000C770B880B990B04C06FE370E025
:107D000080E090E0BCDCEDCF8091D00D869586952B
:107D100080FDD9CF6FEF7FEF88E995E190DC61E0DE
:107D20008CE694E00E94FB33E3CE83E00ED462E362
:107D300083E02BDC66E070E080E090E0A0DC81E096
:107D400004D462E38CE021DC8091630290916402B0
:107D50000F948F4591DC65E270E080E090E08FDC6D
:107D6000D0CE8091FE0C11112DC08111E5CD2AC01D
:107D70008091A204853108F059C0E3CD2091DA0C3E
:107D8000111184C02111EECD81C08091A2048531F2
:107D900008F0B0C0ECCD8091A204853108F0DAC0C3
:107DA000EBCD90FD03C086E596E102C08EE696E13C
:107DB0007C010CE022E048E068E08CE694E00E9460
:107DC0002534B5CDB601DD0C880B990B0F94B1525B
:107DD00020E030E040E05FE30F9436510F947E5294
:107DE000CB010F948F457C01FC0180818032E1F44E
:107DF000F7018181803211F401E001C002E0902F8F
:107E0000990F900F892F819567E0815FBEDB83E03A
:107E100090E0801B91098E0D9F1D2EDC69E070E0C3
:107E200080E090E02CDC88CD03E0E9CF20E030E07A
:107E300040E05FE3C501B4010F9436510F947E52C8
:107E4000CB010F948F457C01FC0180818032E1F4ED
:107E5000F7018181803211F401E001C002E0902F2E
:107E6000990F900F892F81956CE1815F8EDB83E004
:107E700090E0801B91098E0D9F1DFEDB69E070E094
:107E800080E090E0FCDB5DCD03E0E9CFBC01990F21
:107E9000880B990B0F94B15220E030E040E05FE393
:107EA0000F9436510F947E52CB010F948F457C0175
:107EB000FC0180818032E1F4F7018181803211F48C
:107EC00001E001C002E0902F990F900F892F81955A
:107ED00067E0845A5ADB83E090E0801B91098E0DA5
:107EE0009F1DCADB69E070E080E090E0C8DB3ACD1E
:107EF00003E0E9CF20E030E040E05FE3C501B401FA
:107F00000F9436510F947E52CB010F948F457C0114
:107F1000FC0180818032E1F4F7018181803211F42B
:107F200001E001C002E0902F990F900F892F8195F9
:107F30006CE1845A2ADB83E090E0801B91098E0D6E
:107F40009F1D9ADB69E070E080E090E098DB0FCD48
:107F500003E0E9CF0091060D002309F40DCD6CE19B
:107F600087E613DBF4E60F9FC001112481589F4F71
:107F70006FEF70E00F944655CB010F948F457CDB7B
:107F800065E270E080E090E07ADBF6CC2D960FB6EB
:107F9000F894DEBF0FBECDBFDF91CF911F910F913F
:107FA000FF90EF90DF90CF90BF90AF909F908F9019
:107FB0007F906F905F904F9008950F931F93CF9392
:107FC000DF93CDB7DEB728970FB6F894DEBF0FBEAC
:107FD000CDBF8A0123E0660F771F2A95E1F7680F6E
:107FE000791F48E050E0CE0101960F94EB592981AA
:107FF0003A81F801808191812817390790F0821722
:10800000930760F09C818281981758F081E090E09E
:108010003B812381231738F080E005C081E090E0A8
:1080200002C08FEF9FEF28960FB6F894DEBF0FBE09
:10803000CDBFDF91CF911F910F910895EF92FF92E5
:108040000F931F93CF93DF93EC018B017A018A8505
:108050009B858617970729F088819981FED81B8711
:108060000A8788859985019681F00E811F81B70165
:1080700088819981EFD8080F111D8885998580170F
:10808000910718F481E090E011C06E818A81680F39
:1080900097014C81888199810E943E382E813F81D1
:1080A000280F311D3F832E8380E090E0DF91CF9138
:1080B0001F910F91FF90EF9008954F925F926F92F2
:1080C0007F928F929F92AF92BF92CF92DF92EF9268
:1080D000FF920F931F93CF93DF93CDB7DEB72D970A
:1080E0000FB6F894DEBF0FBECDBF6C012A013B0175
:1080F000490158011B861C86CE0101967C0188E04F
:10810000F70111928A95E9F7DB01CA0127E0B695DC
:10811000A795979587952A95D1F79A838983F42F08
:10812000FF77FD878F2F80588B838C831A86198663
:108130004F3F51056105710509F018F460E070E0EA
:1081400026C060915D0470915E048E01075F1F4F31
:1081500097014DED5FE380915B0490915C040E9478
:10816000147E97FDEBCF69857A8583E0660F771FD4
:108170008A95E1F780915B0490915C04680F791F08
:1081800048E050E0C7010F94EB596F817885611585
:10819000710519F44B86B60106C0C616D70619F04C
:1081A0008D8580688B87AE01455F5F4FC401F50107
:1081B00019952D960FB6F894DEBF0FBECDBFDF9197
:1081C000CF911F910F91FF90EF90DF90CF90BF90D4
:1081D000AF909F908F907F906F905F904F90089599
:1081E0006F927F928F929F92AF92BF92CF92DF92C7
:1081F000EF92FF920F931F93CF93DF9300D01F92C4
:10820000CDB7DEB76C017B013A01590148011982F3
:108210001A821B821C82AE014F5F5F4FB301C70100
:108220000E94747E7C0149815A816B817C81411559
:1082300051056105710529F084019501C6013DDFF5
:10824000E6CF0F900F900F900F90DF91CF911F917D
:108250000F91FF90EF90DF90CF90BF90AF909F90E5
:108260008F907F906F90089521E020935F04EBE55D
:10827000F4E0918380837383628380E090E00895CB
:108280007F92AF92BF92CF92DF92EF92FF920F93C5
:108290001F93CF93DF93CDB7DEB72C970FB6F8942B
:1082A000DEBF0FBECDBF6C01762EF72F842FE52FDA
:1082B000B901A801D6011496AD90BC901597909184
:1082C0005F0491110AC026EC36E1482F672DC601E4
:1082D0000E94753880E090E019C0DA82C9827B8202
:1082E000FC838D83EE8318861F82FA86E9861C86BE
:1082F0001B860EE110E49E012F5F3F4FC501DDDEBE
:10830000B501C6010E942D398F8198852C960FB634
:10831000F894DEBF0FBECDBFDF91CF911F910F91BB
:10832000FF90EF90DF90CF90BF90AF907F90089537
:10833000CF92DF92EF92FF920F931F93CF93DF9331
:10834000CDB7DEB72C970FB6F894DEBF0FBECDBF0A
:108350007C01C901F701C480D58020915F042111FF
:1083600008C026EA36E1C7010E94753880E090E037
:108370001CC0FA82E9826B837C834D835E831886FE
:108380001F821A8709871C861B860EE110E49E0156
:108390002F5F3F4F4EE05EE7BC01C60121DFB60113
:1083A000C7010E942D398F8198852C960FB6F894BD
:1083B000DEBF0FBECDBFDF91CF911F910F91FF9018
:1083C000EF90DF90CF900895CF92DF92EF92FF92DF
:1083D0000F931F93CF93DF93CDB7DEB72C970FB6D4
:1083E000F894DEBF0FBECDBF7C01C901F701C48088
:1083F000D58020915F04211108C026E836E1C7012D
:108400000E94753880E090E01CC0FA82E9826B839C
:108410007C834D835E8318861F821A8709871C869A
:108420001B860EE110E49E012F5F3F4F41E15EE7A6
:10843000BC01C601D5DEB601C7010E942D398F816E
:1084400098852C960FB6F894DEBF0FBECDBFDF9196
:10845000CF911F910F91FF90EF90DF90CF900895F3
:10846000CF93DF93EC01262F4CAD6BAD04960E94A9
:1084700020382BAD082E000C990B820F911D8BAF6D
:1084800081E090E0DF91CF9108950F939CE0899F68
:10849000802D112421E0280F20936704845F8093AE
:1084A000660490E002964091A00450E0841795077E
:1084B00014F480E033C0822F90E02091A20430E0D9
:1084C00082179307B4F76623A9F061E08CE694E085
:1084D0000E94FB33409167044E5F0BE020E860E0B0
:1084E0008CE694E00E949D3660E08CE694E00E9469
:1084F000FB3305C061E08CE694E00E94FB336091A1
:1085000066048091A0046817A0F29091670480919E
:10851000A204891770F280E038D881E00F910895A5
:10852000CF93DF93FC0185ADEF012496811105C047
:1085300081E085AFCE010E949B33CE01DF91CF91C8
:108540000C94D2336FEF7FEF7AC8482F50E0209120
:108550006504022E000C330B4217530781F0809301
:108560006504813031F463E67DE18CE694E00C949F
:108570002D3961EB77E18CE694E00C942D39089568
:1085800088E694E0CDDF80E00E944B9F8CE694E08B
:108590000E94D6338111F7CF64EC79E080E090E05F
:1085A0000C94A39FEF92FF920F938EEDE82E8CE137
:1085B000F82E03E127E047E064E28CE694E00E94B5
:1085C000253483E0C2DF22E533E04BE265E28CE64E
:1085D00094E00E943E382CE533E047E367E08CE608
:1085E00094E00F91FF90EF900C943E3888E694E071
:1085F00097DFD8DF8CE694E00E94D6338111F9CF63
:1086000064EC79E080E090E00C94A39FB9DFEECFBA
:1086100060E070E083E69DE127CE1F93CF93DF9368
:10862000C0916D04C695C69588E694E079DFDC2F8D
:10863000DD0F1D2F1C0F83E088DF6C2F80E00E9470
:10864000C53A84EA96E018D86D2F80E00E94C53ABA
:1086500083EF96E177DF612F80E00E94C53A86EED6
:1086600096E170DF8CE694E00E94D6338111E3CF6F
:10867000DF91CF911F9108950895CF93E62F6CE07D
:10868000869F602D112481E0860F80936704645FCC
:1086900060936604462F50E04E5F5F4F2091A00428
:1086A00030E0421753070CF44CC090E02091A20434
:1086B00030E0821793070CF044C0CE2F8EE30E9467
:1086C000C53A65E470E080E090E00E943F3B61E3E2
:1086D0006C0F062E000C770B880B990B0E943F3B0A
:1086E00060E270E080E090E00E943F3B60910B0D03
:1086F00070910C0D80910D0D90910E0D0F947E5286
:10870000CB010F948F450E943C3B6FE270E080E00C
:1087100090E00E943F3B0E940282811109C085E0E7
:10872000C89FF0011124E650F34F8481811109C0E4
:1087300080910F0D9091100D0F948F45CF910C9457
:108740003C3BCF910895CF92DF92EF92FF920F932F
:108750001F93CF93DF931F921F92CDB7DEB77B019C
:10876000622F498392DE4981882309F444C044235F
:1087700011F101151105F9F4C7010E94E47F25E10B
:1087800030E0281B310937FF02C02F5F3F4F35957E
:10879000279530E82158822F830F87FD0DC060E2B6
:1087A00070E080E090E02A8339830E943F3B39816A
:1087B00031502A81F0CF30E8C32ED12CB601C70149
:1087C0000E941F3B7601E81AF90A0115110511F400
:1087D0001E2D07C0FF24B701C8010E94023B1E2DB9
:1087E000181B173040F060E270E080E090E00E94DB
:1087F0003F3B181BF6CF0F900F90DF91CF911F9149
:108800000F91FF90EF90DF90CF9008950F93CF934B
:10881000DF93982F862FEA01692F37DE882331F105
:1088200062E770E0CE010E941F3BC2E7C81BC73061
:1088300040F060E270E080E090E00E943F3BC81BA7
:10884000F6CF609166048AE70E94C53A602F000F58
:10885000770B880B990B0E943F3B60E270E080E051
:1088600090E0DF91CF910F910C943F3BDF91CF913E
:108870000F910895CF92DF92EF92FF920F931F9383
:10888000CF93DF93982F862F6A017901692FFDDD41
:10889000882309F447C0C701002321F00E94E47F28
:1088A000182F03C00E94C37F182FC3E1D0E0C11B63
:1088B000D1098C2F880FC80FCC0FD0E0BE01C601A4
:1088C0000E941F3BC81B6AE370E080E090E00E94BA
:1088D0003F3BC73040F060E270E080E090E00E94F3
:1088E0003F3BC81BF6CF8AEF189F802D1124609163
:1088F000660480580E94C53AC701002349F0DF9101
:10890000CF911F910F91FF90EF90DF90CF901ACEF3
:10891000DF91CF911F910F91FF90EF90DF90CF905B
:108920000C943C3BDF91CF911F910F91FF90EF9002
:10893000DF90CF900895BF92CF92DF92EF92FF9297
:108940000F931F93CF93DF936C017B010E94E47F11
:10895000C82FC7010E94C37F03E110E0081B110963
:108960008C2F90E0BB24B394081719071CF0B12C8E
:10897000C5E201C0CFE12C2F30E0A9014E5F5F4F6F
:108980008091A00490E04817590744F0295031091C
:108990008091A20490E082179307BCF5D0E0E11427
:1089A000F104D9F16AE370E080E090E00E943F3B7F
:1089B000BB2081F0C45F8091A004C81770F12C2FF8
:1089C00030E0295031098091A20490E0821793078A
:1089D0001CF423C0DD2309F1802F880F800F6C2F3A
:1089E000880F0E94C53A60E270E080E090E00E944B
:1089F0003F3BC701DF91CF911F910F91FF90EF9007
:108A0000DF90CF90BF900C943C3B6C2F80E00E9495
:108A1000C53AC60197DDD1E0C2CFDF91CF911F915A
:108A20000F91FF90EF90DF90CF90BF900895CF927D
:108A3000DF92EF92FF920F931F93CF93DF931F92DA
:108A4000CDB7DEB7182F7A01D22ECA0169830E94F2
:108A5000E47F082F812F880F810FC82ECC0C1CE0DB
:108A60006981169F100D1124DD20C1F061E08CE6B4
:108A700094E00E94FB33202F220F200F220F2E5F45
:108A80000BE047EF410F6FEF6C0D8CE694E00E9416
:108A90009D3660E08CE694E00E94FB33612F8C2DC4
:108AA0000E94C53AC7014EDDDD2071F061E08CE621
:108AB00094E00F90DF91CF911F910F91FF90EF9075
:108AC000DF90CF900C94FB330F90DF91CF911F91EB
:108AD0000F91FF90EF90DF90CF900895AF92BF92EB
:108AE000DF92EF92FF920F931F93CF93DF93EC01EE
:108AF0005B01D42EC901B801A7010E94938191E0C6
:108B00002D2D2927A50164E081E091DFCE010E948F
:108B1000E47F2D2DAE0164E094E1981B892FDF9155
:108B2000CF911F910F91FF90EF90DF90BF90AF908A
:108B30007ECFEF92FF920F93CF93DF93D82FC62F64
:108B40007901682F8C2FA1DC8823F1F0002331F00C
:108B500062E070E080E090E00E943F3B2D2F4C2FC0
:108B600064E1C7010E946F8068E770E00E94023BE9
:108B7000C8E7C81BC73040F060E270E080E090E0DA
:108B80000E943F3BC81BF6CFDF91CF910F91FF9022
:108B9000EF9008958F929F92AF92BF92CF92DF9203
:108BA000EF92FF920F936B017C0180906104909093
:108BB0006204A0906304B0906404A50194010F9432
:108BC0000F52882301F120E030E0A901C701B6016E
:108BD0000F940F52882351F0A5019401C701B601EB
:108BE0000F940F5287FD04C081E003C080E001C0F4
:108BF0008FEF80936004C0926104D0926204E0928F
:108C00006304F09264048091A004813128F480917F
:108C1000A204833008F048C08091A004853128F474
:108C20008091A204843108F04FC08091A0048F335A
:108C300008F057C08091A2048F3208F452C080918E
:108C4000600440E3481B87E3E82E87E1F82E0DE03F
:108C500022E06AE58CE694E00E942534809160046D
:108C600041E3481B9DE1E92E97E1F92E22E065E002
:108C70008CE694E00E94253421E5E22E27E1F22ED5
:108C800000E123E04FE262E18CE694E00E942534AB
:108C900031E8E32E37E1F32E23E04FE267E68CE67E
:108CA00094E00E9425341DC08091600444E0481B7C
:108CB00052E0E52E57E1F52E0CE022E062E48CE66E
:108CC00094E00E942534A8CF4AE1E42E47E1F42E37
:108CD00001E023E044E16CE38CE694E00E9425345B
:108CE000A4CF0F91FF90EF90DF90CF90BF90AF9007
:108CF0009F908F900895CF92EF920F93CF93DF9331
:108D0000C8E6D4E01B821A8284E793E099838883C3
:108D1000CC24CA94EE24EA9402E522E143E164E122
:108D200072E0CE010E94A63A80E893E0998388839E
:108D3000DF91CF910F91EF90CF9008955A9887FDD2
:108D400052C05B9800000000000000005A9A5A9838
:108D5000282F220F86FD53C05B9800000000000002
:108D600000005A9A5A98922F990F26FD46C05B9898
:108D700000000000000000005A9A5A98892F880FBE
:108D800096FD39C05B9800000000000000005A9A70
:108D90005A98982F990F86FD2CC05B980000000010
:108DA000000000005A9A5A98892F880F96FD1FC01C
:108DB0005B9800000000000000005A9A5A98982F13
:108DC000990F86FD12C05B980000000000000000B3
:108DD0005A9A5A9896FD15C05B9800000000000052
:108DE00000005A9A08955B9AADCF5B9AEDCF5B9ADB
:108DF000E0CF5B9AD3CF5B9AC6CF5B9AB9CF5B9A31
:108E0000ACCF5B9AEACF2F923F925F927F929F9274
:108E1000AF92BF92CF92DF92EF92FF920F931F9388
:108E2000CF93DF937C011B01942E69018AE04817E0
:108E300009F47BC0A5E14A134EC0DB011296ED9107
:108E4000FC9113971281C681D7815D9A88E28A9539
:108E50000000E9F700EE010F80E1582E510E98E274
:108E6000792E88EF6BDF872D8A950000E9F71032A5
:108E700008F046C0812F8077806860DF812F82955F
:108E8000807F5CDF872D8A950000E9F780E856DF58
:108E900080E054DF872D8A950000E9F78AEF4EDFE6
:108EA000872D8A950000E9F75E01B0E1AB0EB11C99
:108EB0008881807F43DF89918295807F3FDFCA155B
:108EC000DB05B1F7872D8A950000E9F71F5F0F5F7B
:108ED0001511C7CF5D989601492DB101C701DF91EA
:108EE000CF911F910F91FF90EF90DF90CF90BF90A7
:108EF000AF909F907F905F903F902F900C945F3544
:108F0000802F807780681ADF802F8295807F16DF20
:108F1000872D8A950000E9F780E810DF80E80EDFF2
:108F2000872D8A950000E9F7B9CF559A5D98539A35
:108F30005B98529A5A9A5D9AC8E28C2F8A950000E3
:108F4000E9F788E790E00E947C3488EFF7DE8C2F09
:108F50008A950000E9F780E2F1DE80E0EFDE8C2FF9
:108F60008A950000E9F780E0E9DE80E8E7DE8C2FF3
:108F70008A950000E9F780E0E1DE80E1DFDE8C2FFA
:108F80008A950000E9F78FE090E00E947C3480E24F
:108F9000D5DE80E4D3DE8C2F8A950000E9F780E2ED
:108FA000CDDE80E6CBDECA950000E9F710E0D8E21E
:108FB00008E2812F80778068C1DE812F8295807FD3
:108FC000BDDE8D2F8A950000E9F780E8B7DE80E0EE
:108FD000B5DE8D2F8A950000E9F78AEFAFDE8D2F81
:108FE0008A950000E9F7C0E280E0A8DE80E0A6DE16
:108FF0009D2F9A950000E9F7C150B1F788EF9EDEEA
:10900000802F8A950000E9F71F5F103209F0D1CF59
:1090100080E094DE80EC92DE88E28A950000E9F739
:109020005D9859CFCF93DF931F921F92CDB7DEB7D4
:1090300089839A830E94ED7A20E040E060E070E04E
:1090400089819A810F900F90DF91CF910C94A07B32
:109050000F93CF93DF9361E081E00E94A97CD091D0
:109060007206C0E0D11117C080917106811104C051
:109070000E94B980811165C080912202882309F481
:1090800057C081E090917106911180E004E024E0E6
:1090900047E756E24BC0D130C1F480917106813070
:1090A00021F40E94B980811154C08091220288234A
:1090B00009F43EC081E090917106913009F080E0A2
:1090C00003E02EE34EE656E231C0D230B9F480918F
:1090D0007106823021F40E94B980811143C08091D1
:1090E0002202882329F181E090917106923009F0E3
:1090F00080E003E02EE345E656E218C0D330C1F429
:1091000080917106833021F40E94B980811133C0AF
:1091100080912202882361F081E090917106933062
:1091200009F080E003E02EE34FE556E26C2F6EDBA2
:10913000CF5FDF5FC53009F095CF84E08093700684
:1091400021C00E94D37B80913E06882309F494CFEE
:1091500019C084EC90E766DF80913E06882309F40D
:10916000A4CF10C085EE95E75DDF80913E06882391
:1091700009F4B5CF07C08BEF99E754DF80913E0625
:10918000882331F2DF91CF910F910895CF92DF9232
:10919000EF92FF920F931F9380912F09811103C0CB
:1091A00081E799E002C08FE299E02BEBC22E26E224
:1091B000D22E7C010EEA16E223ED3BE74DEE58E499
:1091C00067EA76E281EA96E20E94B47D1F910F91F0
:1091D000FF90EF90DF90CF90089581E799E00E9493
:1091E000958B0E94CC7B0C94CD860E94319021E01F
:1091F00030E0811102C020E030E0309399062093E6
:1092000098061092720681E080933E0683E0809378
:1092100022020895CF92DF92EF92FF920F931F9355
:10922000CF93DF930E9435916C0161E081E00E9451
:10923000A97CC0917206D0E081E0C81AD108C111A2
:1092400017C080917106811104C00E94B9808111FC
:1092500095C080912202882359F081E09091710697
:10926000911180E004E024E04CE956E26D2FCEDA63
:1092700061E779E088EF98E00E942E97809171096C
:109280008F3201F180917E0983FF1CC0C130C1F48F
:1092900080917106813021F40E94B980811176C0DD
:1092A00080912202882361F081E0909171069130D3
:1092B00009F080E000E22EE348E956E26D2FA6DADD
:1092C00092E001C091E080912202882309F44EC00F
:1092D000760111E01C0F8FEFE816F80609F446C07E
:1092E000C9133FC060E070E0C7010E940A8D9091F1
:1092F0007E098091710694FF1CC08C134EC00E94A1
:10930000B980882309F449C081E799E00E94DB8F86
:109310001092720682E090E09093990680939806EE
:1093200081E080933E0610929B0683E080932202A8
:1093300052C08C1304C00E94B98081113DC080913D
:109340002202882361F081E0909171069C1380E0F5
:1093500000E02CEF36E14CE756E26D2FEADB912F6F
:1093600001C09F5F81E0E81AF108B5CFDF5FCF5FF2
:10937000D53009F064CF909370062DC00E94D37B46
:1093800080913E06882309F464CF25C02EDF8091AA
:109390003E06882309F484CF1EC0809122028823D0
:1093A000F1F281E0909171069C1380E001E02CEFD6
:1093B00036E14AE856E2D1CF0E94ED7A20E040E063
:1093C00060E070E086EC98E40E94A07B80913E060D
:1093D000882309F4B4CFDF91CF911F910F91FF90B3
:1093E000EF90DF90CF900895CF93DF93EC01CB0106
:1093F000BA010F94B1520F9483526883DF91CF91D9
:109400000895CF93DF93EC01CB01BA010F94B152D1
:109410002FE632E143E85AE30F944D546883798391
:109420008A839B83DF91CF91089564EF79E481E291
:109430009AE40C94E87B61E07AE48EE39AE40C947D
:10944000E87B0F94B1520F948352862F0D94E4441D
:10945000CF93DF9300D01F92CDB7DEB769837A83B5
:109460008B839C8360E2CE0101960F9408480F9095
:109470000F900F900F90DF91CF9108950F94B152FC
:109480002FE632E143E85AE30F944D54E1CF2F9297
:109490003F924F925F926F927F928F929F92AF9284
:1094A000BF92CF92DF92EF92FF920F931F93CF93D1
:1094B000DF93CDB7DEB729970FB6F894DEBF0FBEA6
:1094C000CDBF1C0179876887CA01B901E982FA8298
:1094D0000B831C83DE82CD82AF8220E030E04AE73E
:1094E00054E40F944D546B017C0120E030E040E0E7
:1094F00057EC0F94125418162CF0C12CD12CE12CDF
:1095000027ECF22EC701B6010F947E522B013C01CD
:1095100020E030E04AE754E469817A818B819C81C4
:109520000F944D544B015C0120E03EEF4FEF56E4A9
:109530000F940F5287FD07C0812C9EEF992EAA240D
:10954000AA9496E4B92E20E030E04AE754E4E88596
:10955000F98560817181828193810F944D546B01F3
:109560007C01C301B2010F94B1529B01AC01C70150
:10957000B6010F9435510F94835269837A838B839C
:109580009C83C501B4010F947E527B018C01E418C9
:10959000F50806091709FF81FF938D809E808BE1F6
:1095A000A82E8AE4B82EC980DA80A30192016885CA
:1095B0007985C1010E94147B0F9029960FB6F8940B
:1095C000DEBF0FBECDBFDF91CF911F910F91FF90F6
:1095D000EF90DF90CF90BF90AF909F908F907F9053
:1095E0006F905F904F903F902F9008958F929F9231
:1095F000AF92BF92CF92DF92EF92FF920F931F93A1
:10960000CF93DF9361E081E00E94A97CD091720644
:10961000C0E0D11119C080917106811104C00E946F
:10962000B9808111C4C080912202882309F4B6C098
:1096300081E090917106911180E004E024E043EF15
:1096400056E26C2FE3D8AAC0D130E1F480917106C4
:10965000813021F40E94B9808111B1C08091220231
:10966000882309F49BC011E080917106813009F0D4
:1096700010E08091820C0F94E44400E09C014DEDD9
:1096800056E289C0D23009F580917106823021F40A
:109690000E94B9808111B4C080912202882309F40C
:1096A0007DC011E080917106823009F010E0609178
:1096B000830C7091840C8091850C9091860CC8DE8F
:1096C00000E09C0149ED56E266C0D33009F5809177
:1096D0007106833021F40E94B9808111AAC0809163
:1096E0002202882309F45AC011E080917106833068
:1096F00009F010E06091870C7091880C8091890CC2
:1097000090918A0CA5DE00E09C0145ED56E243C035
:10971000D43001F580917106843021F40E94B98023
:109720008111A0C0809122028823C1F111E08091B3
:109730007106843009F010E060918B0C70918C0CF4
:1097400080918D0C90918E0C83DE00E09C0141EDA8
:1097500056E221C0D53011F580917106853021F493
:109760000E94B980811197C0809122028823B1F0B4
:1097700011E080917106853009F010E060912602B9
:1097800070912702809128029091290261DE00E009
:109790009C014DEB56E26C2F812F6CD8CF5FDF5FC1
:1097A000C53009F036CF86E0809370068CC00E94E9
:1097B000D37B80913E06882309F435CF84C081E0B5
:1097C0000E94AE80C090820CD12C1F92812C912CD3
:1097D00045E1A42E4AE4B42EE12CF12C8701EA9451
:1097E00020E030E0A90162E87CE088EE96E20E9489
:1097F000147B0F9080913E06882309F42FCF63C01D
:1098000081E00E94AE80A12CC12CD12C16E6E12E65
:10981000FE2C0EE111E420E030E0A90163E87CE0D9
:109820008BED96E234DE80913E06882309F434CF36
:109830004AC081E00E94AE80A12CC12CD12C16E63A
:10984000E12EFE2C0EE111E420E030E0A90167E8F2
:109850007CE087ED96E21BDE80913E06882309F4CA
:109860003ECF31C081E00E94AE80A12CC12CD12C12
:1098700016E6E12EFE2C0EE111E420E030E0A90115
:109880006BE87CE083ED96E202DE80913E06882361
:1098900009F448CF18C081E00E94AE80A12CC12CF1
:1098A000D12C16E6E12EFE2C0EE111E420E030E092
:1098B000A90166E272E087EC96E2E9DD80913E065E
:1098C000882309F451CFDF91CF911F910F91FF9021
:1098D000EF90DF90CF90BF90AF909F908F900895C2
:1098E000CF93DF93EC01CB01BA010F94B15220E08A
:1098F00030E048EC52E40F944D540F948352688347
:1099000079838A839B83DF91CF910895CF93DF93EF
:10991000EC01CB01BA010F94B1522AE037ED43E2DA
:109920005CE30F944D54688379838A839B83DF9132
:10993000CF910895CF93DF93EC01CB01BA010F943F
:10994000B152688379838A839B83DF91CF91089595
:10995000CF93DF93EC01CB01BA010F94B15220E019
:1099600030E048EC51E40F944D54688379838A8346
:109970009B83DF91CF910895CF93DF93EC01CB01CF
:10998000BA010F94B15220E030E048EC52E40F9459
:109990004D54688379838A839B83DF91CF910895A7
:1099A000CF93DF93EC01CB01BA010F94B15220E0C9
:1099B00030E048EC51E40F944D540F948352688387
:1099C00079838A839B83DF91CF910895CF93DF932F
:1099D000EC01CB01BA010F94B1522AE037ED43E21A
:1099E0005CE30F944D54688379838A839B83DF9172
:1099F000CF910895CF93DF93EC01CB01BA010F947F
:109A0000B1522DEC3CEC4CEC5DE30F944D5468836B
:109A100079838A839B83DF91CF91089560E77CE40B
:109A200082E19EE40C94E87B66E87CE48FE59DE4AB
:109A30000C94E87B6AE97CE486EF9DE40C94E87B77
:109A40006CEB7CE489E99DE40C94E87B68EA7CE4B7
:109A50008CE79DE40C94E87B60ED7CE484E39EE479
:109A60000C94E87B66EE7CE486EB9DE40C94E87B4A
:109A70006AEF7CE482E49DE40C94E87B0D94E200C0
:109A80000D942901CF93DF9300D01F92CDB7DEB79D
:109A90000F94B1522DEC3CEC4CEC5DE30F944D5423
:109AA00069837A838B839C83CE0101960F94264A27
:109AB0000F900F900F900F90DF91CF910895CF935B
:109AC000DF9300D01F92CDB7DEB70F94B1522AE0DA
:109AD00037ED43E25CE30F944D5469837A838B83C3
:109AE0009C83CE0101960F94CA460F900F900F9061
:109AF0000F90DF91CF910895CF93DF9300D01F9205
:109B0000CDB7DEB70F94B15220E030E048EC51E41D
:109B10000F944D5469837A838B839C83CE01019685
:109B20000F9451490F900F900F900F90DF91CF91AC
:109B30000895CF93DF9300D01F92CDB7DEB70F9477
:109B4000B15220E030E048EC52E40F944D54698368
:109B50007A838B839C83CE0101960F9451490F9099
:109B60000F900F900F90DF91CF910895CF93DF93D7
:109B700000D01F92CDB7DEB70F94B1522AE037ED77
:109B800043E25CE30F944D5469837A838B839C8317
:109B9000CE0101960F9486490F900F900F900F9071
:109BA000DF91CF910895CF92DF92EF92FF926B01F8
:109BB0007C0120E030E0A9010F940F5287FD05C021
:109BC00020E030E040E05FE304C020E030E040E02F
:109BD0005FEBC701B6010F9436510F947E52CB0153
:109BE000FF90EF90DF90CF900D948F450F94B1527E
:109BF000DACFCF93DF9300D01F92CDB7DEB70F94AB
:109C000083520F94AF5269837A838B839C83CE01F6
:109C100001960F9451490F900F900F900F90DF9184
:109C2000CF9108950F94B15220E030E048EC52E417
:109C30000F944D54DECFCF93DF9300D01F92CDB75A
:109C4000DEB70F9483520F94AF5269837A838B836C
:109C50009C83CE0101960F9451490F900F900F9065
:109C60000F90DF91CF9108950F94B15220E030E032
:109C700048EC51E40F944D54DECF0F931F93CF93D4
:109C8000DF9361E081E00E94A97CC0917206D0E080
:109C9000C1111AC080917106811104C00E94B9805F
:109CA000811104C180912202882309F461C081E0FE
:109CB00090917106911180E004E024E049E457E2BC
:109CC0006D2F0E94064454C0C130D9F480917106B2
:109CD000813021F40E94B9808111F0C0809122026C
:109CE000882309F445C081E090917106913009F014
:109CF00080E003E02EE340E457E26D2F0E9406442B
:109D000037C0C230D1F480917106823021F40E94B4
:109D1000B9808111DCC080912202882349F181E061
:109D200090917106923009F080E003E02EE343E366
:109D300057E26D2F0E9406441BC0C330C9F48091C6
:109D40007106833021F40E94B9808111C9C08091CD
:109D50002202882369F081E090917106933009F026
:109D600080E003E02EE34EE257E26D2F0E940644AE
:109D70000E94897B81111DC0C430E9F48091710675
:109D8000843021F40E94B9808111B3C080912202F5
:109D9000882309F4B7C081E090917106943009F0EE
:109DA00080E003E02EE345E257E26D2F0E94064477
:109DB000A9C014E001C015E0C1131BC08091710659
:109DC0008C1304C00E94B98081119EC08091220230
:109DD000882371F081E0909171069C1380E003E08C
:109DE0002EE34CE157E26D2F0E9406441C2F01C068
:109DF0001C2F81E0810FC81318C0809171068C134D
:109E000004C00E94B980811188C0809122028823F9
:109E100061F081E0909171069C1380E003E02EE3F5
:109E20004DE057E26D2F0E94064482E0810FC81377
:109E300018C0809171068C1304C00E94B9808111F2
:109E400075C080912202882361F081E090917106B3
:109E50009C1380E003E02EE341E057E26D2F0E9467
:109E6000064483E0810FC81318C0809171068C13DB
:109E700004C00E94B980811162C0809122028823AF
:109E800061F081E0909171069C1380E003E02EE385
:109E900048EF56E26D2F0E940644DF5FCF5FD5305A
:109EA00009F0F6CE1C5F1093700651C00E94D37B60
:109EB00080913E06882309F4F5CE49C08BE897E5EA
:109EC000B1D880913E06882309F408CF40C08EE6C1
:109ED00091E5A8D880913E06882309F41CCF37C0AD
:109EE00089E599E59FD880913E06882309F42FCF14
:109EF0002EC08DE89BE596D880913E06882309F414
:109F000045CF25C015E075CF86EF9AE48BD88091B8
:109F10003E06882309F45ACF1AC081E690E582D81C
:109F200080913E06882309F470CF11C089E296E53E
:109F300079D880913E06882309F483CF08C086EF44
:109F400094E570D880913E06882309F496CFDF917E
:109F5000CF911F910F9108952F923F924F925F9250
:109F60006F927F928F929F92AF92BF92CF92DF9229
:109F7000EF92FF920F931F93CF93DF93CDB7DEB78E
:109F800029970FB6F894DEBF0FBECDBF1C017987AD
:109F90006887E982FA820B831C83DE82CD82AF82DE
:109FA000CA01B9010F94AF522AE037ED43E25CE3F6
:109FB0000F944D546B017C0120E030E040E057EC01
:109FC0000F94125418162CF0C12CD12CE12C27EC34
:109FD000F22EC701B6010F947E522B013C0169811C
:109FE0007A818B819C810F94AF522AE037ED43E256
:109FF0005CE30F944D544B015C0120E03EEF4FEFCA
:10A0000056E40F940F5287FD07C0812C9EEF992EC6
:10A01000AA24AA9496E4B92EE885F9856081718115
:10A02000828193810F94AF522AE037ED43E25CE3E3
:10A030000F944D546B017C01C301B2010F94B152D6
:10A040009B01AC01C701B6010F9435510F948352A7
:10A0500069837A838B839C83C501B4010F947E52FC
:10A060007B018C01E418F50806091709FF81FF93AD
:10A070008D809E808EE0A82E8DE4B82EC980DA8077
:10A08000A301920168857985C1010E94147B0F901C
:10A0900029960FB6F894DEBF0FBECDBFDF91CF91EA
:10A0A0001F910F91FF90EF90DF90CF90BF90AF90F6
:10A0B0009F908F907F906F905F904F903F902F90E8
:10A0C0000895AF92CF92DF92EF92FF920F931F937A
:10A0D000CF93DF9361E081E00E94A97CD09172066A
:10A0E000C0E0D1111AC080917106811104C00E9494
:10A0F000B980811194C080912202882309F486C01E
:10A1000081E090917106911180E004E024E04EE935
:10A1100059E26C2F0E94064479C0D13039F5809104
:10A120007106813021F40E94B980811180C0809134
:10A130002202882309F46AC011E0809171068130FF
:10A1400009F010E060919A0D70919B0D80919C0D2B
:10A1500090919D0D0F94AF524CDD00E09C0148E9B9
:10A1600059E26C2F812F0E943A4450C0D23039F509
:10A1700080917106823021F40E94B980811171C0F2
:10A1800080912202882309F441C011E08091710678
:10A19000823009F010E060919E0D70919F0D8091CA
:10A1A000A00D9091A10D0F94AF5223DD00E09C0112
:10A1B00044E959E26C2F812F0E943A4427C0D330E2
:10A1C00029F580917106833021F40E94B9808111B4
:10A1D00062C0809122028823C9F011E0809171064B
:10A1E000833009F010E06091A20D7091A30D809171
:10A1F000A40D9091A50D0F94AF52FBDC00E09C01E3
:10A2000040E959E26C2F812F0E943A44CF5FDF5F13
:10A21000C53009F066CF84E08093700655C00E9477
:10A22000D37B80913E06882309F465CF4DC0A12CD5
:10A2300047E8C42E4FECD42E10EDE12E17E0F12E9E
:10A2400000E010E024E630E040E050E06AE97DE024
:10A250008BE999E281DE80913E06882309F467CF7D
:10A2600033C0A12C27E8C22E2FECD22E10EDE12E08
:10A2700017E0F12E00E010E024E630E040E050E08E
:10A280006EE97DE086E999E267DE80913E068823EB
:10A2900009F476CF19C0A12C87E8C82E8FECD82EF0
:10A2A00010EDE12E17E0F12E00E010E024E630E0A2
:10A2B00040E050E062EA7DE082E999E24DDE809183
:10A2C0003E06882309F485CFDF91CF911F910F912E
:10A2D000FF90EF90DF90CF90AF9008956F927F92B4
:10A2E0008F929F92AF92BF92CF92DF92EF92FF92A6
:10A2F0000F931F93CF93DF9300D01F92CDB7DEB79C
:10A3000061E081E00E94A97C60907206712C61106E
:10A310001AC080917106811104C00E94B980811118
:10A320004EC180912202882309F440C181E09091BE
:10A330007106911180E004E024E045E758E2672DC2
:10A340000E94064433C181E068122CC080917106DE
:10A35000813021F40E94B980811139C1809122029B
:10A36000882309F423C111E080917106813009F03E
:10A3700010E08091B50E9091B60EA091B70EB091FD
:10A38000B80E89839A83AB83BC83CE0101960F9468
:10A39000514900E09C0149E658E2672D812F0E9457
:10A3A0003A4404C182E068122CC080917106823068
:10A3B00021F40E94B980811142C180912202882338
:10A3C00009F4F4C011E080917106823009F010E0C8
:10A3D0008091B90E9091BA0EA091BB0EB091BC0EB7
:10A3E00089839A83AB83BC83CE0101960F94514934
:10A3F00000E09C0145E558E2672D812F0E943A4418
:10A40000D5C083E068122CC080917106833021F49E
:10A410000E94B98081114BC180912202882309F4E6
:10A42000C5C011E080917106833009F010E0809181
:10A43000BD0E9091BE0EA091BF0EB091C00E89834B
:10A440009A83AB83BC83CE0101960F94514900E0FF
:10A450009C0143E458E2672D812F0E943A44A6C034
:10A4600084E0681227C080917106843021F40E9434
:10A47000B980811154C180912202882309F496C0C9
:10A4800011E080917106843009F010E06091810E36
:10A490007091820E8091830E9091840E0F94AF5232
:10A4A000CADB00E09C0145E358E2672D812F0E9442
:10A4B0003A447CC085E0681227C0809171068530DF
:10A4C00021F40E94B980811166C180912202882303
:10A4D00009F46CC011E080917106853009F010E03C
:10A4E0006091850E7091860E8091870E9091880EF6
:10A4F0000F94AF52A0DB00E09C0147E258E2672DC9
:10A50000812F0E943A4452C086E0681227C0809191
:10A510007106863021F40E94B980811178C1809142
:10A520002202882309F442C011E08091710686302E
:10A5300009F010E06091890E70918A0E80918B0E67
:10A5400090918C0E0F94AF5276DB00E09C0149E1B4
:10A5500058E2672D812F0E943A4428C087E0681294
:10A5600025C080917106873021F40E94B980811145
:10A5700083C1809122028823C9F011E08091710685
:10A58000873009F010E060918D0E70918E0E8091F1
:10A590008F0E9091900E0F94AF522BDB00E09C0138
:10A5A0004BE058E2672D812F0E943A4473946394E4
:10A5B00085E07812ACCE88E08093700679C10E9465
:10A5C000D37B80913E06882309F4ABCE71C181E034
:10A5D0000E94AE802AE037ED43E25DE36091B50E64
:10A5E0007091B60E8091B70E9091B80E0F944D54A5
:10A5F00020E030E040E85FE30F9435510F94835240
:10A600001F92812C912C56E2A52E5DE4B52E6B0194
:10A6100017E7E12E1FE0F12E00E010E021E030E02E
:10A6200040E050E065EB7EE08FE698E20E94147B0C
:10A630000F9080913E06882309F490CE39C181E0C5
:10A640000E94AE802AE037ED43E25CE36091B90EF0
:10A650007091BA0E8091BB0E9091BC0E0F944D5428
:10A6600020E030E040E85FE30F9435510F948352CF
:10A670001F92812C912C30E2A32E3DE4B32E6B016E
:10A680001DEDE12E13E0F12E00E010E021E030E0BE
:10A6900040E050E069EB7EE08FE598E20E94147B99
:10A6A0000F9080913E06882309F487CE01C181E096
:10A6B0000E94AE802AE037ED43E25DE36091BD0E7B
:10A6C0007091BE0E8091BF0E9091C00E0F944D54AC
:10A6D00020E030E040E85FE30F9435510F9483525F
:10A6E0001F92812C912C96E2A92E9DE4B92E6B012C
:10A6F00017E7E12E1FE0F12E00E010E021E030E04E
:10A7000040E050E06DEB7EE08CE498E20E94147B28
:10A710000F9080913E06882309F47ECEC9C081E067
:10A720000E94AE806091810E7091820E8091830EA6
:10A730009091840E0F94AF522AE037ED43E25DE32F
:10A740000F944D5420E030E040E850E40F94355130
:10A750000F9483521F92AEE38A2EADE49A2EBCE290
:10A76000AB2EBDE4BB2E6B0114E7E12E1FE0F12EF2
:10A7700000E010E024E030E040E050E061E87EE0FE
:10A780008CE398E20E94147B0F9080913E06882310
:10A7900009F471CE8DC081E00E94AE806091850E7B
:10A7A0007091860E8091870E9091880E0F94AF5213
:10A7B0002AE037ED43E25DE30F944D5420E030E0B2
:10A7C00040E850E40F9435510F9483521F925EE39A
:10A7D000852E5DE4952EECE2AE2EEDE4BE2E6B01EF
:10A7E00014E7E12E1FE0F12E00E010E024E030E05D
:10A7F00040E050E065E87EE08EE298E20E94147B43
:10A800000F9080913E06882309F45FCE51C081E00D
:10A810000E94AE806091890E70918A0E80918B0E9D
:10A8200090918C0E0F94AF522AE037ED43E25DE336
:10A830000F944D540F9483521F922EE3822E2DE4D9
:10A84000922E3CE2A32E3DE4B32E6B0118E7E12EDD
:10A850001FE0F12E00E010E020E030E0A90169E8FF
:10A860007EE080E298E20E94147B0F9080913E0689
:10A87000882309F454CE1CC081E00E94AE80A12C34
:10A880008EE3C82E8DE4D82E18EBE12E12E8F12EBF
:10A8900001E010E024E630E040E050E06DE87EE0CA
:10A8A00082E198E259DB80913E06882309F461CE6B
:10A8B0000F900F900F900F90DF91CF911F910F91FC
:10A8C000FF90EF90DF90CF90BF90AF909F908F90D0
:10A8D0007F906F9008952F923F924F925F926F9268
:10A8E0007F928F929F92AF92BF92CF92DF92EF9220
:10A8F000FF920F931F93CF93DF9300D000D0CDB77B
:10A90000DEB71C017E836D8329013A01460120E0F8
:10A9100030E040E057ECB201C3010F941254181616
:10A920002CF0412C512C612C27EC01C0272DB201B9
:10A93000862D922F0F947E522B013C0120E03EEF9A
:10A940004FEF56E4B701C8010F940F5287FD06C0C0
:10A95000B12C9EEFF92E0FEF16E401C0BE2CC301FF
:10A96000B2010F94B1529B01AC01ED81FE81608177
:10A970007181828193810F9435510F948352698341
:10A980007A838B839C836B2D7F2DC8010F947E521D
:10A990007B018C01E418F50806091709AF928AE1DA
:10A9A000A82E8DE4B82EC980DA80A30192016D81B2
:10A9B0007E81C1010E94147B0F9026960FB6F894F9
:10A9C000DEBF0FBECDBFDF91CF911F910F91FF90E2
:10A9D000EF90DF90CF90BF90AF909F908F907F903F
:10A9E0006F905F904F903F902F9008956F927F925D
:10A9F0008F929F92AF92BF92CF92DF92EF92FF928F
:10AA00000F931F93CF93DF9300D01F92CDB7DEB784
:10AA100061E081E00E94A97C60907206712C611057
:10AA20001AC080917106811104C00E94B980811101
:10AA300098C080912202882309F48AC081E0909115
:10AA40007106911180E004E024E04EE759E2672DA1
:10AA50000E9406447DC081E068122CC0809171067E
:10AA6000813021F40E94B980811183C0809122023B
:10AA7000882309F46DC011E080917106813009F0DE
:10AA800010E08091F20D9091F30DA091F40DB09132
:10AA9000F50D89839A83AB83BC83CE0101960F9415
:10AAA000CA4600E09C014AE659E2672D812F0E94C8
:10AAB0003A444EC082E0681225C08091710682300F
:10AAC00021F40E94B980811182C0809122028823E2
:10AAD00009F43EC011E080917106823009F010E067
:10AAE00060914C0C70914D0C80914E0C90914F0CDC
:10AAF0005AD800E09C0146E559E2672D812F0E945B
:10AB00003A4426C083E0681223C0809171068330E6
:10AB100021F40E94B980811172C0809122028823A1
:10AB2000B9F011E080917106833009F010E0609176
:10AB3000500C7091510C8091520C9091530C33D861
:10AB400000E09C0146E459E2672D812F0E943A44BF
:10AB50007394639485E0781262CF84E080937006EA
:10AB600065C00E94D37B80913E06882309F461CFA3
:10AB70005DC020E030E048EC52E46091F20D70914D
:10AB8000F30D8091F40D9091F50D0F944D540F94A9
:10AB900083521F92812C912C24E1A22E2DE4B22EFF
:10ABA0006B01EE24EA941FE7F12E00E010E020E0B4
:10ABB00030E0A90162EF7DE084E799E20E94147B16
:10ABC0000F9080913E06882309F450CF2FC081E07A
:10ABD0000E94AE80A12CC12CD12CE12CF12C08E4D8
:10ABE00013E420E030E0A9016CE47CE080E699E227
:10ABF00072DE80913E06882309F467CF17C081E09A
:10AC00000E94AE80A12CC12CD12CE12CF12C08E4A7
:10AC100013E420E030E0A90160E57CE08EE499E2F5
:10AC20005ADE80913E06882309F477CF0F900F906B
:10AC30000F900F90DF91CF911F910F91FF90EF90A8
:10AC4000DF90CF90BF90AF909F908F907F906F904C
:10AC500008956F927F928F929F92AF92BF92CF9200
:10AC6000DF92EF92FF920F931F93CF93DF9300D069
:10AC70001F92CDB7DEB761E081E00E94A97C6090B1
:10AC80007206712C61101AC080917106811104C086
:10AC90000E94B9808111BFC080912202882309F4EB
:10ACA000B2C081E090917106911180E004E024E04F
:10ACB00044E359E2672D0E940644A5C081E0681272
:10ACC00023C080917106813021F40E94B9808111E6
:10ACD000AAC080912202882309F495C080911F0E9A
:10ACE000811103C024E239E202C028E239E281E0A6
:10ACF00090917106913009F080E001E04BE159E25A
:10AD0000672D0E943A447FC082E0681226C080917D
:10AD10007106823021F40E94B980811192C0809125
:10AD20002202882309F46FC011E0809171068230FD
:10AD300009F010E060917D0270917E0280917F02A7
:10AD4000909180020E94D34D00E09C014DE059E2B9
:10AD5000672D812F0E943A4456C083E0681226C0B6
:10AD600080917106833021F40E94B98081117EC0E8
:10AD700080912202882309F446C011E08091710677
:10AD8000833009F010E0609181027091820280911D
:10AD90008302909184020E94D34D00E09C014FEF0A
:10ADA00058E2672D812F0E943A442DC084E068123A
:10ADB0002AC080917106843021F40E94B9808111EB
:10ADC0006AC0809122028823F1F011E0809171061F
:10ADD000843009F010E08091790290917A02A0917C
:10ADE0007B02B0917C0289839A83AB83BC83CE01C2
:10ADF00001960F94CA4600E09C014FEE58E2672D81
:10AE0000812F0E943A447394639485E078123ACF7C
:10AE1000709270066DC00E94D37B80913E0688239D
:10AE200009F43ACF65C040E050E06FE17EE08BE28C
:10AE300099E20E947B7B80913E06882309F449CFEA
:10AE400057C0A12CC12CD12CE12CF12C01E913E429
:10AE500020E030E0A9016DE772E084E199E23BDD9A
:10AE600080913E06882309F45ACF42C0A12CC12C00
:10AE7000D12CE12CF12C01E913E420E030E0A90110
:10AE800061E872E086E099E226DD80913E06882343
:10AE900009F46ECF2DC020E030E048EC52E4609120
:10AEA000790270917A0280917B0290917C020F94DA
:10AEB0004D540F9483521F92812C912C84E1A82E23
:10AEC0008DE4B82E6B0118EEE12E13E0F12E00E0B8
:10AED00010E020E030E0A90169E772E087EF98E236
:10AEE0000E94147B0F9080913E06882309F469CF5D
:10AEF0000F900F900F900F90DF91CF911F910F91B6
:10AF0000FF90EF90DF90CF90BF90AF909F908F9089
:10AF10007F906F900895AF92CF92DF92EF92FF9261
:10AF20000F931F93CF93DF9361E081E00E94A97C90
:10AF3000D0917206C0E0D1111AC0809171068111C2
:10AF400004C00E94B980811109C180912202882326
:10AF500009F4FBC081E090917106911180E004E05A
:10AF600024E04DED58E26C2F0E940644EEC0D13033
:10AF700031F580917106813021F40E94B9808111F0
:10AF8000F5C080912202882309F4DFC011E080918E
:10AF90007106813009F010E06091A50E7091A60E47
:10AFA0008091A70E9091A80E0E94D34D00E09C01C5
:10AFB0004FEC58E26C2F812F0E943A44C6C0D23029
:10AFC00031F580917106823021F40E94B98081119F
:10AFD000E7C080912202882309F4B7C011E0809174
:10AFE0007106823009F010E06091A90E7091AA0EEE
:10AFF0008091AB0E9091AC0E0E94D34D00E09C016D
:10B0000041EC58E26C2F812F0E943A449EC0D3300D
:10B0100031F580917106833021F40E94B98081114D
:10B02000D9C080912202882309F48FC011E0809159
:10B030007106833009F010E06091AD0E7091AE0E94
:10B040008091AF0E9091B00E0E94D34D00E09C0114
:10B0500043EB58E26C2F812F0E943A4476C0D430E3
:10B0600031F580917106843021F40E94B9808111FC
:10B07000CBC080912202882309F467C011E080913F
:10B080007106843009F010E06091B10E7091B20E3B
:10B090008091B30E9091B40E0E94D34D00E09C01BC
:10B0A00045EA58E26C2F812F0E943A444EC0D530B9
:10B0B00031F580917106853021F40E94B9808111AB
:10B0C000BDC080912202882309F43FC011E0809125
:10B0D0007106853009F010E06091C10E7091C20ECA
:10B0E0008091C30E9091C40E0E94D34D00E09C014C
:10B0F0004BE958E26C2F812F0E943A4426C0D6308B
:10B1000021F580917106863021F40E94B980811169
:10B11000AEC0809122028823C1F011E080917106B7
:10B12000863009F010E06091C50E7091C60E8091D6
:10B13000C70E9091C80E0E94D34D00E09C0147E8D5
:10B1400058E26C2F812F0E943A44CF5FDF5FC530F9
:10B1500009F0F1CE87E080937006A1C00E94D37BF6
:10B1600080913E06882309F4F0CE99C081E00E94C8
:10B17000AE80A12CC12CD12CE12C10ECF12E09E7D2
:10B1800014E420E030E040E85FE365EA7EE086ED2D
:10B1900098E2A1DB80913E06882309F4F2CE7FC0BD
:10B1A00081E00E94AE80A12CC12CD12CE12C10ECAE
:10B1B000F12E09E714E420E030E040E85FE369EABB
:10B1C0007EE088EC98E287DB80913E06882309F4D4
:10B1D00000CF65C081E00E94AE80A12CC12CD12C93
:10B1E000E12C10ECF12E09E714E420E030E040E817
:10B1F0005FE36DEA7EE08AEB98E26DDB80913E06CC
:10B20000882309F40ECF4BC081E00E94AE80A12CB0
:10B21000C12CD12CE12C10ECF12E09E714E420E034
:10B2200030E040E85FE361EB7EE08CEA98E253DBDC
:10B2300080913E06882309F41CCF31C081E00E9432
:10B24000AE80A12CC12CD12CE12C10ECF12E09E701
:10B2500014E420E030E0A90161EC7EE080EA98E2AD
:10B260003ADB80913E06882309F42BCF18C081E099
:10B270000E94AE80A12CC12CD12CE12C10ECF12E1F
:10B2800009E714E420E030E0A90165EC7EE081E903
:10B2900098E221DB80913E06882309F43ACFDF91C2
:10B2A000CF911F910F91FF90EF90DF90CF90AF90D3
:10B2B00008956F927F928F929F92AF92BF92CF929A
:10B2C000DF92EF92FF920F931F93CF93DF9300D003
:10B2D0001F92CDB7DEB761E081E00E94A97C60904B
:10B2E0007206712C61101AC080917106811104C020
:10B2F0000E94B9808111C2C080912202882309F482
:10B30000B5C081E090917106911180E004E024E0E5
:10B3100049EF57E2672D0E940644A8C081E06812F9
:10B3200026C080917106813021F40E94B98081117C
:10B33000ADC080912202882309F498C011E0809169
:10B340007106813009F010E06091510E7091520E3B
:10B350008091530E9091540E0E94D34D00E09C01B9
:10B3600049EE57E2672D812F0E943A447FC082E068
:10B37000681226C080917106823021F40E94B98043
:10B3800081119EC080912202882309F46FC011E0D0
:10B3900080917106823009F010E06091550E709135
:10B3A000560E8091570E9091580E0E94D34D00E09A
:10B3B0009C0149ED57E2672D812F0E943A4456C007
:10B3C00083E068122CC080917106833021F40E94C2
:10B3D000B98081118FC080912202882309F446C070
:10B3E00011E080917106833009F010E08091590ED0
:10B3F00090915A0EA0915B0EB0915C0E89839A8356
:10B40000AB83BC83CE0101960F94864900E09C017A
:10B4100049EC57E2672D812F0E943A4427C084E00F
:10B42000681224C080917106843021F40E94B98092
:10B43000811198C0809122028823C1F011E080918F
:10B440007106843009F010E060915D0E70915E0E1F
:10B4500080915F0E9091600E0E94D34D00E09C01A0
:10B4600049EB57E2672D812F0E943A44739463940D
:10B4700085E0781237CF709270068DC00E94D37B22
:10B4800080913E06882309F437CF85C081E00E9471
:10B49000AE80A12CC12CD12CE12C10E8F12E07E7B5
:10B4A00014E420E030E040E85FE361E57EE081EF16
:10B4B00097E211DA80913E06882309F43ACF6BC0F7
:10B4C00081E00E94AE80A12CC12CD12CE12C10E88F
:10B4D000F12E07E714E420E030E040E85FE365E5A3
:10B4E0007EE081EE97E2F7D980913E06882309F449
:10B4F00049CF51C081E00E94AE8020E030E048ECAE
:10B5000052E46091590E70915A0E80915B0E9091A9
:10B510005C0E0F944D5420E030E040E251E40F9473
:10B5200035510F9483521F92812C912C92E3A92EB6
:10B530009DE4B92E6B0115EFE12E1FE7F12E00E01F
:10B5400010E02AE030E040E050E069E57EE081ED87
:10B5500097E20E94147B0F9080913E06882309F4A5
:10B560003ACF19C081E00E94AE80A12CC12CD12C11
:10B57000E12C10E8F12E07E714E420E030E040E889
:10B580005FE36DE57EE081EC97E2A5D980913E0610
:10B59000882309F44FCF0F900F900F900F90DF91F9
:10B5A000CF911F910F91FF90EF90DF90CF90BF90C0
:10B5B000AF909F908F907F906F9008952F923F92C1
:10B5C0004F925F926F927F928F929F92AF92BF92B3
:10B5D000CF92DF92EF92FF920F931F93CF93DF935F
:10B5E000CDB7DEB729970FB6F894DEBF0FBECDBF3B
:10B5F0001C0179876887CA01B901E982FA820B8345
:10B600001C83DE82CD82AF8220E030E040E251E454
:10B610000F944D546B017C0120E030E040E057EC8A
:10B620000F94125418162CF0C12CD12CE12C27ECBD
:10B63000F22EC701B6010F947E522B013C0120E08F
:10B6400030E040E251E469817A818B819C810F94E2
:10B650004D544B015C0120E03EEF4FEF56E40F9458
:10B660000F5287FD07C0812C9EEF992EAA24AA9421
:10B6700096E4B92E20E030E040E251E4E885F98517
:10B6800060817181828193810F944D546B017C01A3
:10B69000C301B2010F94B1529B01AC01C701B601C5
:10B6A0000F9435510F94835269837A838B839C83E3
:10B6B000C501B4010F947E527B018C01E418F5089A
:10B6C00006091709FF81FF938D809E8088E3A82ECD
:10B6D0008DE4B82EC980DA80A3019201688579854E
:10B6E000C1010E94147B0F9029960FB6F894DEBF1B
:10B6F0000FBECDBFDF91CF911F910F91FF90EF90C3
:10B70000DF90CF90BF90AF909F908F907F906F9081
:10B710005F904F903F902F9008959F92AF92BF926D
:10B72000CF92DF92EF92FF920F931F93CF93DF930D
:10B7300000D01F92CDB7DEB761E081E00E94A97C06
:10B7400090907206B12C91101AC0809171068111EF
:10B7500004C00E94B9808111D4C080912202882344
:10B7600009F4C7C081E090917106911180E004E076
:10B7700024E047EA57E26B2D0E940644BAC081E0FC
:10B7800098122CC080917106813021F40E94B980FA
:10B790008111BFC080912202882309F4AAC011E060
:10B7A00080917106813009F010E08091950E9091A2
:10B7B000960EA091970EB091980E89839A83AB83D1
:10B7C000BC83CE0101960F94264A00E09C0143E918
:10B7D00057E26B2D812F0E943A448BC082E0981271
:10B7E0002CC080917106823021F40E94B9808111B1
:10B7F000ACC080912202882309F47BC011E08091C3
:10B800007106823009F010E08091990E90919A0EA5
:10B81000A0919B0EB0919C0E89839A83AB83BC83CD
:10B82000CE0101960F94264A00E09C014FE757E2B3
:10B830006B2D812F0E943A445CC083E098122CC08B
:10B8400080917106833021F40E94B980811199C0E2
:10B8500080912202882309F44CC011E08091710686
:10B86000833009F010E080919D0E90919E0EA09182
:10B870009F0EB091A00E89839A83AB83BC83CE01C7
:10B8800001960F94264A00E09C014BE657E26B2D8F
:10B89000812F0E943A442DC084E098122AC08091E2
:10B8A0007106843021F40E94B980811186C0809194
:10B8B00022028823F1F011E080917106843009F0B2
:10B8C00010E08091A10E9091A20EA091A30EB091D4
:10B8D000A40E89839A83AB83BC83CE0101960F9417
:10B8E000264A00E09C0147E557E26B2D812F0E941C
:10B8F0003A44B394939485E0B81225CFB092700681
:10B9000077C00E94D37B80913E06882309F425CF1F
:10B910006FC081E00E94AE80A12C60E4C62E6DE471
:10B92000D62EE12C1CE3F12E0CE116E420E030E0F1
:10B9300040EA50E465E97EE08DE997E23FDE8091E0
:10B940003E06882309F426CF53C081E00E94AE80D2
:10B95000A12C40E4C42E4DE4D42EE12C1CE3F12EA6
:10B960000CE116E420E030E040EA50E469E97EE0D2
:10B9700089E897E223DE80913E06882309F439CFD7
:10B9800037C081E00E94AE80A12C20E4C22E2DE4BD
:10B99000D22EE12C1CE3F12E0CE116E420E030E085
:10B9A00040EA50E46DE97EE085E797E207DE8091AA
:10B9B0003E06882309F44CCF1BC081E00E94AE8074
:10B9C000A12C80E4C82E8DE4D82EE12C1CE3F12EAE
:10B9D0000CE116E420E030E040EA50E461EA7EE069
:10B9E00081E697E2EBDD80913E06882309F45FCF84
:10B9F0000F900F900F900F90DF91CF911F910F91AB
:10BA0000FF90EF90DF90CF90BF90AF909F90089500
:10BA10000F93CF93DF9361E081E00E94A97CC091F6
:10BA20007206D0E0C11118C080917106811104C066
:10BA30000E94B9808111B5C080912202882361F0F3
:10BA400081E090917106911180E004E024E04EE0E5
:10BA50005AE26D2F0E9406448091D10D8770873085
:10BA600009F058C0C130D9F480917106813021F4B9
:10BA70000E94B98081119DC080912202882309F41F
:10BA8000C0C081E090917106913009F080E003E040
:10BA90002EE347E05AE26D2F0E940644B2C0C23046
:10BAA000D9F480917106823021F40E94B98081110D
:10BAB0008AC080912202882309F4A3C081E090917A
:10BAC0007106923009F080E003E02EE340E05AE294
:10BAD0006D2F0E94064495C0C330D1F58091710648
:10BAE000833021F40E94B980811177C080912202B5
:10BAF000882309F486C081E090917106933009F0A3
:10BB000080E003E02EE349EF59E26D2F0E940644E6
:10BB100084E03EC0C130F1F480917106813021F49F
:10BB20000E94B980811163C080912202882309F4A8
:10BB30006AC081E090917106913009F080E000E2E6
:10BB40002EE34BEE59E26D2F0E94064482E020C0A6
:10BB500084E001C082E0C8131BC0809171068C1381
:10BB600004C00E94B980811150C0809122028823B4
:10BB700071F081E0909171069C1380E003E02EE368
:10BB800042EE59E26D2F0E9406448C2F01C08C2F8B
:10BB9000DF5FCF5FD53009F045CF8F5F80937006B0
:10BBA0003DC00E94D37B80913E06882309F444CF98
:10BBB00035C08BEC91E60E94124880913E068823A6
:10BBC00009F45ACF2BC080ED91E60E941248809173
:10BBD0003E06882309F46DCF21C085ED91E60E94D1
:10BBE000124880913E06882309F480CF17C085EF64
:10BBF00099E20E94127B80913E06882309F494CF3B
:10BC00000DC084E0C5CF82E0C3CF8AED91E60E94EB
:10BC1000124880913E06882309F4A7CFDF91CF9187
:10BC20000F910895CF92DF92EF92FF92CF93C82F9A
:10BC30000E94C82E6B017C0124EA30E74DE75FE3E8
:10BC40006091890670918A0680918B0690918C068E
:10BC50000F940F5287FD05C04AEF50E060E070E09E
:10BC600003C040E050E0BA01C40ED51EE61EF71E28
:10BC7000C0928506D0928606E0928706F0928806EA
:10BC8000C0932302CF91FF90EF90DF90CF90089563
:10BC90002F923F924F925F926F927F928F929F92DC
:10BCA000AF92BF92CF92DF92EF92FF921F93CF930A
:10BCB000DF93CDB7DEB728970FB6F894DEBF0FBE7F
:10BCC000CDBF1C01162F0E94B980882329F0109245
:10BCD000A0060E94D37BDAC0209198063091990685
:10BCE0003E832D83232B09F49DC0E4E01E9FC001F9
:10BCF000112498878F83FC01E759FD4F8080918044
:10BD0000A280B38020E030E04AE754E4C501B401EA
:10BD10000F9435512B013C0120E030E04AE754E418
:10BD2000C501B4010F9436516B017C0180915E0214
:10BD30008823B9F1113029F198F0123091F5409033
:10BD40005602509057026090580270905902C0906D
:10BD50005A02D0905B02E0905C02F0905D0221C03C
:10BD6000409046025090470260904802709049020D
:10BD7000C0904A02D0904B02E0904C02F0904D02ED
:10BD800010C040904E0250904F0260905002709050
:10BD90005102C0905202D0905302E0905402F090B1
:10BDA00055022D813E81B901330F880B990B0F94F9
:10BDB000B1522091890630918A0640918B065091AC
:10BDC0008C060F944D549B01AC01C501B4010F9436
:10BDD0003651EF81F885E759FD4F5F01608371832C
:10BDE000828393832D813E8137FF0CC0A301920192
:10BDF0000F940F5287FF11C0F50140825182628279
:10BE000073820BC0A70196010F94125418162CF4DC
:10BE1000F501C082D182E282F382812F03DF81E0CB
:10BE20008093220210929906109298068091220225
:10BE3000882361F124E0129FF0011124E759FD4F9E
:10BE400080819181A281B38189839A83AB83BC83F2
:10BE50002DEC3CEC4CEC5DE36091890670918A0618
:10BE600080918B0690918C060F94125487FD05C02B
:10BE7000CE0101960F94904705C060E2CE01019675
:10BE80000F940848BC01C1010E949B4428960FB63C
:10BE9000F894DEBF0FBECDBFDF91CF911F91FF9011
:10BEA000EF90DF90CF90BF90AF909F908F907F905A
:10BEB0006F905F904F903F902F90089560E08FE8D3
:10BEC0009AE2E6CE61E088E89AE2E2CE62E081E8BA
:10BED0009AE2DECECF93DF9300D01F92CDB7DEB7CC
:10BEE0000E94B980882329F01092A0060E94D37B7B
:10BEF00057C060919806709199066115710569F1B6
:10BF0000072E000C880B990B0F94B15220918906D3
:10BF100030918A0640918B0650918C060F944D54B7
:10BF20009B01AC016091750270917602809177025D
:10BF3000909178020F943651609375027093760257
:10BF4000809377029093780283E06CDE81E08093A7
:10BF5000220210929906109298068091220288235C
:10BF6000F9F02091A8053091A9054091AA055091BA
:10BF7000AB05609175027091760280917702909185
:10BF800078020F94355169837A838B839C83CE0129
:10BF900001960F949047BC0185E19AE20E949B4470
:10BFA0000F900F900F900F90DF91CF91089521E0A7
:10BFB0002093A0066093890670938A0680938B066F
:10BFC00090938C0620E040E060E070E08091A60550
:10BFD0009091A7050C94A07B60E070E080E291E472
:10BFE000E6CF60E070E080E89FE3E1CF6DEC7CECB1
:10BFF0008CEC9DE3DCCF6DEC7CEC8CEC9CE3D7CF40
:10C00000FF920F931F93CF93DF93F82E7093A705A2
:10C010006093A60561E081E00E94A97CD091720640
:10C02000C0E091E081E0F81659F1F81628F082E0BE
:10C03000F81609F449C06CC0D111D1C0992389F018
:10C040008091710618166CF020919806309199062F
:10C050002F5F3F4F30939906209398068F5F809310
:10C06000710680912202882309F42EC100E010E0BD
:10C0700021E041E06AE77AE28C2F0E94A34324C1C9
:10C08000D111ADC0992389F08091710618166CF01A
:10C0900020919806309199062F5F3F4F3093990673
:10C0A000209398068F5F80937106809122028823E7
:10C0B00009F42AC100E010E021E041E063E77AE200
:10C0C0008C2F0E94A34320C1D11189C0992389F0EC
:10C0D0008091710618166CF020919806309199069F
:10C0E0002F5F3F4F30939906209398068F5F809380
:10C0F000710680912202882309F404C100E010E057
:10C1000021E041E06CE67AE28C2F0E94A343FAC062
:10C110004091750250917602609177027091780299
:10C120004093A8055093A9056093AA057093AB05A9
:10C13000D11120C0992389F08091710618166CF0F6
:10C1400020919806309199062F5F3F4F30939906C2
:10C15000209398068F5F8093710680912202882336
:10C1600049F000E010E021E041E063E67AE28C2F44
:10C170000E94A34383E0F81232C060910B0D7091CE
:10C180000C0D80910D0D90910E0D2091D50C21116B
:10C1900026C00F947E5220913602309137026217EA
:10C1A0007307ECF4D130C9F480917106813021F429
:10C1B0000E94B9808111B2C080912202882369F067
:10C1C00081E090917106913009F080E004E024E074
:10C1D00043E55AE26C2F0E94064482E096C0D130BB
:10C1E000D9F480917106813021F40E94B9808111C7
:10C1F0009DC080912202882309F466C081E090915D
:10C200007106913009F080E004E024E049E45AE24C
:10C210006C2F0E94064458C0D230D9F48091710628
:10C22000823021F40E94B980811188C0809122025D
:10C23000882309F449C081E090917106923009F099
:10C2400080E003E02EE34FE35AE26C2F0E940644A5
:10C250003BC0D330D1F480917106833021F40E9429
:10C26000B980811175C080912202882369F181E033
:10C2700090917106933009F080E003E02EE346E3ED
:10C280005AE26C2F0E9406441FC0D430E9F480911A
:10C290007106843021F40E94B980811163C08091BD
:10C2A0002202882389F081E090917106943009F090
:10C2B00080E003E02EE34BE25AE26C2F0E9406443A
:10C2C00082E0F81221C01EC082E0F8121DC0D530F5
:10C2D000C9F480917106853021F40E94B9808111E2
:10C2E0004BC080912202882369F081E09091710611
:10C2F000953009F080E003E02EE34EE15AE26C2F26
:10C300000E94064486E001C085E0CF5FDF5F90E0D9
:10C31000C53009F087CE8093700637C00E94D37B6A
:10C3200080913E06882309F447CF2FC00E94D37B1B
:10C3300080913E06882309F45CCF27C08CEE9FE5F0
:10C340000E94124880913E06882309F46FCF1DC0D9
:10C3500081EF9FE50E94124880913E06882309F4F0
:10C3600082CF13C086EF9FE50E94124880913E065F
:10C37000882309F494CF09C08BEF9FE50E941248EF
:10C3800080913E06882309F4ACCFDF91CF911F91B5
:10C390000F91FF9008954FEF6EE57FE580E030CE7E
:10C3A0004FEF62E67FE581E02BCE4FEF66E67FE55B
:10C3B00082E026CE4FEF6AE67FE583E021CE0F9341
:10C3C000CF93DF9361E081E00E94A97CD091720657
:10C3D000C0E0D1111AC080917106811104C00E9481
:10C3E000B98081116FC080912202882309F461C055
:10C3F00081E090917106911180E004E024E04DED20
:10C4000059E26C2F0E94064454C0D130D9F4809177
:10C410007106813021F40E94B98081115BC0809146
:10C420002202882309F445C081E090917106913081
:10C4300009F080E003E02EE343ED59E26C2F0E9407
:10C44000064437C0D230D1F480917106823021F495
:10C450000E94B980811148C080912202882349F14D
:10C4600081E090917106923009F080E000E22EE3C5
:10C4700045EC59E26C2F0E9406441BC0D330C9F42E
:10C4800080917106833021F40E94B980811136C0F9
:10C4900080912202882369F081E0909171069330A7
:10C4A00009F080E000E22EE340EB59E26C2F0E949D
:10C4B0000644CF5FDF5FC53009F08BCF84E0809307
:10C4C000700624C00E94D37B80913E06882309F425
:10C4D0008ACF1CC088E09DE50E94124880913E06EC
:10C4E000882309F49CCF12C08FEC99E20E94127B42
:10C4F00080913E06882309F4AFCF08C081EC99E211
:10C500000E94127B80913E06882311F2DF91CF9129
:10C510000F910895CF93DF93EC01CB01BA010F94F3
:10C52000B1520F947E5279836883DF91CF91089541
:10C530006AE872E681E293E60C94E87B0F931F931E
:10C54000CF93DF9361E081E00E94A97CC0917206E5
:10C55000D0E081E0C11122C0882389F0809171066A
:10C5600018166CF020919806309199062F5F3F4F76
:10C5700030939906209398068F5F8093710680917F
:10C580002202882309F441C000E010E020E041E0ED
:10C5900067EF7BE28D2F0E94A34337C0C130D1F4F7
:10C5A00080917106813021F40E94B980811137C0D9
:10C5B00080912202882349F181E0909171069130A7
:10C5C00009F080E000E22EE34CEE5BE26D2F0E946A
:10C5D00006441BC0C230C9F480917106823021F438
:10C5E0000E94B980811122C080912202882369F0C3
:10C5F00081E090917106923009F080E000E22EE334
:10C6000043EE5BE26D2F0E940644DF5FCF5F80E068
:10C61000D53009F09FCF83E0809370060DC0C093A2
:10C62000540C80913E06882319F206C0C093540C26
:10C6300080913E068823C1F2DF91CF911F910F9127
:10C6400008950F94B1520F947E52CB010D948F45F3
:10C65000EF92FF920F931F93CF93DF93CDB7DEB787
:10C660002B970FB6F894DEBF0FBECDBF7C01409173
:10C67000AD05842F042E000C990B2091AE052230BD
:10C6800051F0233019F025E33CE20AC047FF06C011
:10C6900021E43CE205C023E53CE202C02AE43CE29E
:10C6A0009F934F933F932F938E010F5F1F4F1F93C5
:10C6B0000F930F94B75A40913402509135024F5066
:10C6C000510997010F900F900F900F900F900F90BE
:10C6D0004E155F050CF49A013093100D20930F0D49
:10C6E00080E00E9451B4C8010E94917D2B960FB644
:10C6F000F894DEBF0FBECDBFDF91CF911F910F9198
:10C70000FF90EF900895E091AD0587E1E802F00118
:10C710001124E95FF24F808591859ACF7F928F92A5
:10C720009F92AF92BF92CF92DF92EF92FF920F93C0
:10C730001F93CF93DF93782E8093AE056093AD0562
:10C7400061E081E00E94A97CD0917206C0E081E0A6
:10C75000D1112EC0882389F08091710618166CF0D3
:10C7600020919806309199062F5F3F4F309399069C
:10C77000209398068F5F8093710680912202882310
:10C7800009F494C022E0721649F033E0731203C03A
:10C7900067E17CE205C067E07CE202C067E27CE220
:10C7A00000E010E021E041E08C2F0E94A3437EC016
:10C7B000D130D9F480917106813021F40E94B98082
:10C7C00081117DC080912202882309F46FC081E02D
:10C7D00090917106913009F080E004E024E042E994
:10C7E0005CE26C2F0E94064461C0D230D9F4809183
:10C7F0007106823021F40E94B980811168C0809155
:10C800002202882309F452C081E09091710692308F
:10C8100009F080E000E22EE346E85CE26C2F0E9423
:10C82000064444C0D330D1F480917106833021F4A2
:10C830000E94B980811156C0809122028823B1F1F3
:10C8400081E090917106933009F080E000E22EE3E0
:10C850004AE75CE26C2F0E94064428C0D43031F5D0
:10C8600080917106843021F40E94B980811145C005
:10C87000809122028823D1F011E0809171068430EA
:10C8800009F010E02091AD0537E12303F0011124F8
:10C89000E95FF24F808591850F948F4500E09C0100
:10C8A0004CE55CE26C2F812F0E943A44CF5FDF5F42
:10C8B00080E0C53009F04CCFC09370065BC00E9489
:10C8C000D37B80913E06882309F47CCF53C08091AE
:10C8D000B5059091B605BCDE80913E06882309F42B
:10C8E0008ECF48C08091B7059091B805B1DE809198
:10C8F0003E06882309F4A0CF3DC081E00E94AE80AF
:10C900000091AD0527E1020380011124F801E95FE0
:10C91000F24F60857185072E000C880B990B0F94E0
:10C92000B15220E030E040EF52E40F9435510F94C3
:10C930008352F801E15FF24F1F9283E8882E83E66D
:10C94000982E98E9A92E92E6B92E6B011AEAE12EEB
:10C95000F12C00E010E028E730E040E050E0BF01BB
:10C960008BE69CE20E94147B0F9080913E06882308
:10C9700009F47ECFDF91CF911F910F91FF90EF903F
:10C98000DF90CF90BF90AF909F908F907F90089551
:10C9900060E081E0C3CE8F929F92AF92BF92CF9220
:10C9A000DF92EF92FF920F931F93CF93DF934C018F
:10C9B0005B016A0160E085E00E94A97CD09172066B
:10C9C000F12C82E0E82ED1111AC080912202882336
:10C9D00021F180912502823041F0833019F468EB17
:10C9E0007BE205C06BEA7BE202C068EC7BE200E020
:10C9F00010E021E041E08F2D0E94A3430EC0D13012
:10CA000061F480912202882341F000E010E020E0F0
:10CA100041E0B4018F2D0E94A343A114B10481F021
:10CA2000D23081F480912202882309F46EC000E0A4
:10CA300010E020E041E0B5018F2D0E94A34365C0C6
:10CA4000C2E001C0C3E0C114D10491F0DC130FC0F7
:10CA500080912202882351F000E010E020E041E0C4
:10CA6000B6018F2D0E94A343CD2F01C0CD2FCF5FE4
:10CA700021E030E0A114B10411F420E030E081E0C5
:10CA800090E0C114D10411F480E090E0820F931F74
:10CA9000029781F0DC130DC080912202882349F0B7
:10CAA00000E010E020E041E061EE7BE28F2D0E948B
:10CAB000A343CF5FDC1314C080912202882371F05E
:10CAC00000E010E021E040E066ED7BE28F2D0E9467
:10CAD000A3436091AC058F2D0E943D43E09222025A
:10CAE000F394DF5F85E0F8126ECFCF5FC0937006DE
:10CAF000DF91CF911F910F91FF90EF90DF90CF903A
:10CB0000BF90AF909F908F900895C3E0C114D1045F
:10CB100009F0ADCFADCF40E050E060E070E080EADA
:10CB20009BE239CF47E95BE267E87BE28EE79BE275
:10CB300032CF40E050E06EE67BE285E69BE22BCF11
:10CB400040E050E066E57BE287E49BE224CF40E0F2
:10CB500050E068E37BE28BE29BE21DCF4FE15BE2BA
:10CB60006EE07BE28EEF9AE216CF40E050E060EF9D
:10CB70007AE287EE9AE20FCF40E050E067ED7AE28A
:10CB80008AEC9AE208CF40E050E06DEB7AE28EEA60
:10CB90009AE201CF40E050E06FE97AE286E99AE25A
:10CBA000FACE6111609325024093AC05082E000C6B
:10CBB000990BAA0BBB0B8C309105A0F5FC018827C3
:10CBC000EA56FF4F8F4F0D94975582E995E61FC0A7
:10CBD00089E995E61CC08CEB95E619C08EEA95E6CE
:10CBE00016C085EB95E613C08AEC95E610C083EC81
:10CBF00095E60DC087EA95E60AC080EA95E607C08B
:10CC00001092540C8EE992E602C08BE895E60097EC
:10CC100049F021E02093A00620E040E060E070E0D1
:10CC20000C94A07B0C94CC7BCF92DF92EF92FF927E
:10CC30000F931F9384E6C82E8DE2D82EE12CF12CA1
:10CC400009E51DE223ED3BE74DEE56E864E57DE2A4
:10CC50008FE49DE20E94B47D1F910F91FF90EF90B1
:10CC6000DF90CF90089590917E0993FB882780F9FB
:10CC700093FF06C081E09091AE07911101C080E062
:10CC80000895EF92FF920F931F93CF93DF9361E08C
:10CC900081E00E94A97CC091720610E0C11118C009
:10CCA00080917106811104C00E94B9808111C8C1B0
:10CCB00080912202882361F081E0909171069111A8
:10CCC00080E004E024E043E45DE2612F0E9406443A
:10CCD00080917E0982FB002700F982FD07C0D1E028
:10CCE0009091EE16913019F0D0E001C0D02F83FB67
:10CCF000EE24E0F883FF03C0B6DFF82E01C0F12C6C
:10CD0000DD2309F458C0C130D9F480917106813017
:10CD100021F40E94B98081119BC180912202882355
:10CD200009F4A8C181E090917106913009F080E08A
:10CD300000E22EE347E35DE2612F0E9406449AC1C0
:10CD4000C230D9F480917106823021F40E94B980FA
:10CD5000811186C180912202882309F48BC181E070
:10CD600090917106923009F080E003E02EE34CE2EE
:10CD70005DE2612F0E9406447DC1C33009F063C0AB
:10CD800080917106833021F40E94B980811174C1B1
:10CD900080912202882309F46DC181E0909171068F
:10CDA000933009F080E003E02EE347E25DE2612F7B
:10CDB0000E9406445FC18091EE16823029F053DF55
:10CDC0008823F9F001111DC0C130E9F4809171068A
:10CDD000813021F40E94B980811158C180912202D2
:10CDE000882309F45BC181E090917106913009F0CC
:10CDF00080E000E22EE34AE15DE2612F0E940644FA
:10CE00004DC1D1E001C0D2E0CD131BC080917106AD
:10CE10008C1304C00E94B980811142C1809122020A
:10CE2000882371F081E0909171069C1380E003E00B
:10CE30002EE343E15DE2612F0E940644DC2F01C036
:10CE4000DC2FDF5F01C0D4E0CD131BC080917106E1
:10CE50008C1304C00E94B98081112CC180912202E0
:10CE6000882371F081E0909171069C1380E003E0CB
:10CE70002EE347E05DE2612F0E940644DC2F01C0F3
:10CE8000DC2F81E08D0FC81318C0809171068C13C0
:10CE900004C00E94B980811117C1809122028823A9
:10CEA00061F081E0909171069C1380E003E02EE335
:10CEB00049EF5CE2612F0E94064482E08D0F4091B1
:10CEC0000F0D5091100D9091D50C911107C020912C
:10CED00036023091370242175307DCF0C81333C0D3
:10CEE000809171068C1304C00E94B9808111F6C034
:10CEF00080912202882339F181E0909171069C1380
:10CF000080E000E22EE341EE5CE2612F0E940644E5
:10CF10001AC0C81318C0809171068C1304C00E94F7
:10CF2000B9808111E5C080912202882361F081E0FF
:10CF3000909171069C1380E003E02EE341ED5CE2EA
:10CF4000612F0E940644DD5FCD1318C080917106E9
:10CF50008C1304C00E94B9808111D4C08091220238
:10CF6000882361F081E0909171069C1380E003E0DA
:10CF70002EE343EC5CE2612F0E94064491E09D0F9A
:10CF8000EE2009F43BC0F11053C0C91318C08091C2
:10CF900071068C1304C00E94B9808111BDC08091BC
:10CFA0002202882361F081E0909171069C1380E059
:10CFB00000E22EE340EB5CE2612F0E94064482E037
:10CFC0008D0FC81318C0809171068C1304C00E9485
:10CFD000B9808111ABC080912202882361F081E089
:10CFE000909171069C1380E003E02EE342EA5CE23C
:10CFF000612F0E94064493E09D0F1AC0C91316C00A
:10D00000809171068C1302C00E94B9808091220227
:10D01000882361F081E0909171069C1380E000E22A
:10D020002EE347E95CE2612F0E94064492E09D0FE7
:10D030001F5FCF5F153009F031CE909370067FC02F
:10D040000E94D37B80913E06882309F431CE77C0BD
:10D050000E94008780913E06882309F45ECE6FC04F
:10D0600084E196E60E94124880913E06882309F4E6
:10D0700071CE65C0D4E005CF8DEF99E60E941248CD
:10D0800080913E06882309F483CE59C00E941187FF
:10D0900080913E06882309F4A1CE51C0D2E0D1CEC2
:10D0A0008FED91E60E94124880913E06882309F494
:10D0B000B5CE45C08EE79CE60E94124880913E06A0
:10D0C000882309F4CBCE3BC081E09AE70E94124846
:10D0D00080913E06882309F4E0CE31C081EF9CE2C6
:10D0E0000E94127B80913E06882309F401CF27C05D
:10D0F00088EC94E60E94124880913E06882309F449
:10D1000012CF1DC087EF9BE60E94124880913E0619
:10D11000882309F423CF13C08FEB9CE20E94127B7B
:10D1200080913E06882309F43ACF09C08AE099E449
:10D130000E94124880913E06882309F44CCFDF916B
:10D14000CF911F910F91FF90EF9008956091050D81
:10D1500070E080E00C943DAF6091890270918A028A
:10D16000072E000C880B990B0F94B1522AE037ED73
:10D1700043E25CE30F944D54609385027093860202
:10D1800080938702909388020895CF93DF93EC01F8
:10D19000CB01BA010F94B1520F9483526883DF918F
:10D1A000CF91089580E00C9451B465EC78E68BED56
:10D1B00098E60C94E87B0F94B1520F948352862F1B
:10D1C0000D941345EF92FF920F931F93CF93DF932C
:10D1D00000D01F92CDB7DEB7082F7B010E94B98027
:10D1E000882329F01092A0060E94D37B3BC0609157
:10D1F0009806709199066115710551F01092990683
:10D200001092980681E080932202802F0E9498A7B6
:10D2100080912202882331F184E0089F800111244B
:10D220000F59114F60913E0C70913F0C072E000C6E
:10D23000880B990B0F94B1529B01AC01F8016081EE
:10D240007181828193810F944D5469837A838B839A
:10D250009C8360E2CE0101960F94A048BC01C701F7
:10D260000E949B440F900F900F900F90DF91CF91F1
:10D270001F910F91FF90EF9008956BED7DE280E09C
:10D28000A1CF60ED7DE281E09DCF20E040E060E055
:10D2900070E00E94A07B81E08093A00610923F0C7A
:10D2A00010923E0C08958DE399E6EFCF81E499E664
:10D2B000ECCF2F923F924F925F926F927F928F921C
:10D2C0009F92AF92BF92CF92DF92EF92FF920F9315
:10D2D0001F93CF93DF93CDB7DEB729970FB6F8949E
:10D2E000DEBF0FBECDBF1C017987688769011A8335
:10D2F0000983EB82BA01550F880B990B0F94B15239
:10D300004B015C0120E030E040E057EC0F941254F8
:10D3100018162CF0812C912CA12C27ECB22EC501D3
:10D32000B4010F947E522B013C01B601DD0C880B39
:10D33000990B0F94B1524B015C0120E03EEF4FEF8F
:10D3400056E40F940F5287FD07C0812C9EEF992E53
:10D35000AA24AA9496E4B92EE885F98560817181A2
:10D36000072E000C880B990B0F94B1526B017C01B6
:10D37000C301B2010F94B1529B01AC01C701B601C8
:10D380000F9435510F9483526C837D838E839F83DA
:10D39000C501B4010F947E527B018C01E418F5089D
:10D3A00006091709FB81FF9389809A8088E9A82ED6
:10D3B00082E6B82ECC80DD80A30192016885798554
:10D3C000C1010E94147B0F9029960FB6F894DEBF1E
:10D3D0000FBECDBFDF91CF911F910F91FF90EF90C6
:10D3E000DF90CF90BF90AF909F908F907F906F9085
:10D3F0005F904F903F902F9008958F929F92AF92A1
:10D40000BF92CF92DF92EF92FF920F931F93CF9331
:10D41000DF9361E081E00E94A97CD0917206C0E0B8
:10D42000D1111AC080917106811104C00E94B98087
:10D43000811121C180912202882309F413C181E066
:10D4400090917106911180E004E024E04BEC5DE2E4
:10D450006C2F0E94064406C1D13011F580917106EF
:10D46000813021F40E94B98081110DC18091220286
:10D47000882309F4F7C011E080917106813009F02A
:10D4800010E080916302909164020F948F4500E058
:10D490009C014FEB5DE26C2F812F0E943A44E2C069
:10D4A000D23011F580917106823021F40E94B9804A
:10D4B0008111FBC080912202882309F4D3C011E0BE
:10D4C00080917106823009F010E080910F0D9091EB
:10D4D000100D0F948F4500E09C0141EB5DE26C2F35
:10D4E000812F0E943A44BEC0D33011F5809171065D
:10D4F000833021F40E94B9808111ECC08091220216
:10D50000882309F4AFC011E080917106833009F0DF
:10D5100010E08091EB0C9091EC0C0F948F4500E0A3
:10D520009C0149EA5DE26C2F812F0E943A449AC027
:10D53000D43001F580917106843021F40E94B980C5
:10D540008111DDC080912202882309F48BC011E093
:10D5500080917106843009F010E08091050D0F94E0
:10D56000134500E09C0145E95DE26C2F812F0E948C
:10D570003A4478C0D53011F580917106853021F498
:10D580000E94B9808111DEC080912202882309F4B3
:10D5900069C011E080917106853009F010E080913A
:10D5A000890290918A020F948F4500E09C014BE81C
:10D5B0005DE26C2F812F0E943A4454C0D630D9F4DA
:10D5C00080917106863021F40E94B9808111CCC00F
:10D5D00080912202882309F445C081E09091710670
:10D5E000963009F080E003E02EE340E85DE26C2F26
:10D5F0000E94064437C0D730D1F48091710687303D
:10D6000021F40E94B9808111B9C08091220288233F
:10D6100049F181E090917106973009F080E003E0D4
:10D620002EE345E75DE26C2F0E9406441BC0D83014
:10D63000C9F480917106883021F40E94B98081116B
:10D64000A7C080912202882369F081E09091710641
:10D65000983009F080E003E02EE346E65DE26C2FAF
:10D660000E940644CF5FDF5FC53009F0D9CE89E064
:10D670008093700696C00E94D37B80913E068823DB
:10D6800009F4D8CE8EC0E12C00E010E027EE33E0A4
:10D690004AE050E063E672E085EC9DE20ADE8091AC
:10D6A0003E06882309F4E2CE7CC081E00E94AE8071
:10D6B000E12C02ED18E622E231E040E050E06FE0BC
:10D6C0007DE088EB9DE2F5DD80913E06882309F43C
:10D6D000F1CE67C081E00E94AE80E12C0EE914EB30
:10D6E0002CE830E040E050E06BEE7CE08DEA9DE21B
:10D6F000E0DD80913E06882309F400CF52C081E02E
:10D700000E94AE80C090050DD12C1F9286EA882E13
:10D7100088E6982E95EDA92E98E6B92EE12CF12CED
:10D720008701EA9420E030E0A90165E07DE08FE91F
:10D730009DE20E94147B0F9080913E06882309F49D
:10D7400001CF2FC0E12C0CEA18E627EE33E04AE0C7
:10D7500050E069E872E080E99DE2ABDD80913E0631
:10D76000882309F411CF1DC083E599E60E94124871
:10D7700080913E06882309F42BCF13C086E599E6F5
:10D780000E94124880913E06882309F43ECF09C0CA
:10D790008FE09DE70E94124880913E06882309F49D
:10D7A00050CFDF91CF911F910F91FF90EF90DF90BD
:10D7B000CF90BF90AF909F908F9008950E94B980B6
:10D7C000882321F01092A0060E94D37B0C94D242B1
:10D7D0000E94B980882341F020E040E060E070E0E2
:10D7E0008EED9BE60E94A07B80E00C944B9F0F93F4
:10D7F000CF93DF9361E081E00E94A97CD091720613
:10D80000C0E0D11117C080917106811104C00E943F
:10D81000B98081114CC080912202882309F43EC056
:10D8200081E090917106911180E004E024E049EFDD
:10D830005DE231C0D130B9F480917106813021F4BC
:10D840000E94B98081113BC080912202882331F16E
:10D8500081E090917106913009F080E003E02EE3C1
:10D860004CEE5DE218C0D530C9F480917106853068
:10D8700021F40E94B98081112CC08091220288235A
:10D8800069F081E090917106953009F080E003E045
:10D890002EE346EE5DE26C2F0E940644CF5FDF5F11
:10D8A000C53009F0AECF86E0809370061AC00E94A2
:10D8B000D37B80913E06882309F4ADCF12C088EE59
:10D8C0009BE60E94124880913E06882309F4BCCF53
:10D8D00008C088E298E40E94124880913E0688239E
:10D8E00061F2DF91CF910F91089560E070E080E0E8
:10D8F0000E943DAF0E94EBB40C94CC7B8F929F9220
:10D90000AF92BF92CF92DF92EF92FF920F931F934D
:10D91000CF93DF9361E081E00E94A97CD0917206F1
:10D92000C0E0D1111AC080917106811104C00E941B
:10D93000B9808111ABC080912202882309F474C0A0
:10D9400081E090917106911180E004E024E041E3D0
:10D950005EE26C2F0E94064467C0D13011F58091C1
:10D960007106813021F40E94B980811197C08091A5
:10D970002202882309F458C011E080917106813099
:10D9800009F010E080910F0D9091100D0F948F45CC
:10D9900000E09C0143E25EE26C2F812F0E943A443A
:10D9A00043C0D23009F580917106823021F40E9483
:10D9B000B980811199C0809122028823A9F111E0D8
:10D9C00080917106823009F010E08091EB0C90910B
:10D9D000EC0C0F948F4500E09C014BE15EE26C2F54
:10D9E000812F0E943A4420C0D330F1F48091710617
:10D9F000833021F40E94B98081119BC08091220262
:10DA0000882391F011E080917106833009F010E0D5
:10DA10008091050D0F94E44400E09C0147E05EE234
:10DA20006C2F812F0E943A4480910F0D9091100D20
:10DA30002091EB0C3091EC0C232B11F4892BE9F0A5
:10DA4000D430C9F480917106843021F40E94B980E9
:10DA5000811192C080912202882369F081E0909127
:10DA60007106943009F080E000E22EE34EEF5DE2B3
:10DA70006C2F0E94064485E001C084E0CF5FDF5F29
:10DA8000C53009F04ECF809370067CC00E94D37BD6
:10DA900080913E06882309F44ECF74C081E00E9435
:10DAA000AE80C0900F0DD090100D1F9262ED862EAB
:10DAB00068E6962E78E9A72E72E6B72E12E2E12EDE
:10DAC000FF24F39400E010E020E030E0A9016FE0D3
:10DAD0007DE08AE29EE20E94147B0F9080913E06D8
:10DAE000882309F444CF4EC081E00E94AE80C090EC
:10DAF000EB0CD090EC0C1F923EE9832E34EB932E6E
:10DB000048E9A42E42E6B42E1CE8E12EF12C00E0F8
:10DB100010E020E030E0A9016BEE7CE08FE19EE2B6
:10DB20000E94147B0F9080913E06882309F443CF16
:10DB300029C081E00E94AE80C090050DD12C1F92BB
:10DB400086EA882E88E6982E95E1A92E9AE4B92EC9
:10DB5000E12CF12C8701EA9420E030E0A90165E096
:10DB60007DE081E19EE20E94147B0F9080913E0651
:10DB7000882309F443CF06C0B8DE80913E0688238F
:10DB800009F468CFDF91CF911F910F91FF90EF9033
:10DB9000DF90CF90BF90AF909F908F90089580E0DE
:10DBA00095E29093C9058093C8058CE491E0909329
:10DBB000CD058093CC0580EC9EEF9093CB058093B0
:10DBC000CA059091C40580E2890F863740F080EF46
:10DBD000890F20E431E03093CB052093CA051092E1
:10DBE000C6058093C7058FEF8093C50508958F9272
:10DBF0009F92BF92CF92DF92EF92FF920F931F936B
:10DC0000CF93DF931F92CDB7DEB7F5D7882309F402
:10DC1000D6C180919806863214F085E202C087FD55
:10DC200080E0282F082E000C330B309399062093A8
:10DC30009806982F990F890F8093C4058091280624
:10DC4000882309F4BCC12091CA053091CB0500910D
:10DC5000C6051091C705020F131FE090C805F0908C
:10DC6000C9058091CC059091CD05E80EF91E0130D3
:10DC70004FE7140768F03195219531093093CB05B2
:10DC80002093CA056CED70E085E090E00F94124C93
:10DC9000F7FE15C08091CC059091CD0591958195A9
:10DCA00091099093CD058093CC0568E171E085E002
:10DCB00090E00F94124C81E08093C50517C081E07D
:10DCC000E81680E4F80694F06BE470E084EF91E0ED
:10DCD0000F94124C8091BA0581508093BA05882325
:10DCE00011F05DDF6CC11092280669C12091CC054E
:10DCF0003091CD05C7019A508130934108F098C00A
:10DD00008F2D992787FD9A950A9765E070E00F940B
:10DD10004655812F17FF02C087E0810F482F459598
:10DD20004595459581E090E0A0E0B0E004C0880F03
:10DD3000991FAA1FBB1F4A95D2F7FB01EE0FFF1FC9
:10DD4000E454FA4F408151818A0108231923012BA1
:10DD500009F419C18095909584239523918380833C
:10DD600084E090E0861B970B4091290650912A068B
:10DD7000840F951F90932A06809329068091BB05F6
:10DD800081508093BB05811103C082E080932806F7
:10DD9000932F9095991F9927991F8091C505881FEA
:10DDA0008827881F9817F1F0319521953109309314
:10DDB000CD052093CC0520E130E040E050E060EF5D
:10DDC0007FEF8FEF9FEF0E9464392091CA05309159
:10DDD000CB05620F731F7093CB056093CA0560E794
:10DDE00073E021C08091CA059091CB0591958195F2
:10DDF00091099093CB058093CA0520E130E040E083
:10DE000050E060EF7FEF8FEF9FEF0E946439209129
:10DE1000CC053091CD05620F731F7093CD056093D3
:10DE2000CC0560E872E085E090E00F94124CABC046
:10DE3000121613060CF0A7C0FDE3FF1A41E0E4162A
:10DE400042E0F40608F09FC08091C405181B103111
:10DE500008F099C03195219531093093CD05209373
:10DE6000CC0560E773E083E090E00F94124C8FEFF5
:10DE70008093C50521E012300CF020E08EEF810F79
:10DE80008C30A0F08091CA059091CB0541E050E024
:10DE90001816190614F040E050E030E0421753071E
:10DEA00009F055C091958195910927C0143050F51E
:10DEB00020E030E0A90160EC7FEF8FEF9FEF0E9440
:10DEC00064392091CA053091CB05620F731F70939E
:10DED000CB056093CA0561157E4F34F480E09EEF58
:10DEE0009093CB058093CA058091CA059091CB058C
:10DEF0008130924064F180E092E09093CB05809372
:10DF0000CA0525C01C301CF120E430E040E050E0A0
:10DF100060E070E0CB010E9464392091CA05309125
:10DF2000CB05620F731F7093CB056093CA05611513
:10DF30007E4F34F480E09EEF9093CB058093CA052A
:10DF40008091CA059091CB0581309240A4F68091D2
:10DF500028068230C1F480E48093BB058FEF9FEFE9
:10DF60009093BD058093BC059093BF058093BE053B
:10DF70009093C1058093C0059093C3058093C2051B
:10DF800081E0809328062091C6053091C7058091D5
:10DF9000CA059091CB05820F931F9093C70580937C
:10DFA000C6052091C8053091C9058091CC05909196
:10DFB000CD05820F931F9093C9058093C80561E03A
:10DFC0008CE694E00E94FB338091A0048E3130F007
:10DFD0008091A0048E3308F456C05AC08091A204E8
:10DFE0008A30B0F38AEBE82E85E0F82E9AE0892E8D
:10DFF000912CB82C8091A00490E094012C5F3F4FAD
:10E00000281739075CF442E0E40EF11C85E0880E25
:10E01000911CEEE18E16910461F7DACF8091A20493
:10E02000881588F330E0C12CD12CF70182819381CF
:10E03000A0E0B0E00C2C04C0B695A7959795879505
:10E040000A94D2F780FD07C0FFEFCF1ADF0A385FCE
:10E05000303859F7D8CF00E010E0A801480D591D1D
:10E060008091A00490E0481759073CF08091A204E9
:10E0700090E0841795070CF055C00F5F1F4F0430D8
:10E08000110559F7E1CF8091A2048C3308F055C0F7
:10E09000809128068823B1F08091C905482F582F18
:10E0A000550F550B9A0133272F5F3F4F8091A004E6
:10E0B00090E0281739073CF08091A204841708F0FB
:10E0C0004DC001C0B1D58091A0048B30D0F469E07F
:10E0D00080E00E94C53A8091290690912A060E940C
:10E0E000CA3A69E08EE60E94C53A2091BA0583E0FB
:10E0F00090E0821B91096FEF7FEF8A5C914D0E9447
:10E100001F3B0E94B980882391F10F90DF91CF913E
:10E110001F910F91FF90EF90DF90CF90BF909F9055
:10E120008F90BFC527E04B2D400F632F8CE694E006
:10E1300039830E940C363981A0CF20E14DE36091F4
:10E14000C4058CE694E00E940C3620E14CE360911B
:10E15000C4058CE694E00E940C369ACF6091C70506
:10E1600002E022E08CE694E00E944D36ACCF0F90A6
:10E17000DF91CF911F910F91FF90EF90DF90CF90A3
:10E18000BF909F908F90089567EF7DE682E078D5ED
:10E19000EAEBF5E088E3828783E0808380E4818393
:10E1A00013821282158214821782168211861086BB
:10E1B000F6DC82E190E090939906809398060895AA
:10E1C0008F929F92AF92BF92CF92DF92EF92FF9287
:10E1D0006091E50520E030E090E080E0F901E65450
:10E1E000FA4FC7A4CC2011F061E0620F8C29722F86
:10E1F0007295707F40E050E0D12CE12CF12C46016B
:10E200005701042E04C0B694A794979487940A9457
:10E21000D2F780FE08C0E92FF0E0E654FA4FA72FAE
:10E22000A42BA2AB9F5F4F5F5F4F4530510539F77D
:10E230002F5F3F4F2330310589F66093E50540E0BD
:10E2400050E020E090E0A0E0B0E06C017D01042E01
:10E2500004C0F694E794D794C7940A94D2F7C0FE0A
:10E2600005C02093E3052AE335E007C02E504F5F39
:10E270005F4F4530510549F7F4CF422F3150A0F0A0
:10E28000225F6C017D01032E04C0F694E794D794BD
:10E29000C7940A94D2F7C0FEF0CF4093E405809172
:10E2A000E605823069F403C02093E405F8CF80913D
:10E2B000E205181614F08CEF01C084E08093E205AB
:10E2C000FF90EF90DF90CF90BF90AF909F908F9096
:10E2D000089580E090E0FC01E654FA4F1682039620
:10E2E0008E319105C1F70895EAEBF5E010828AE0DE
:10E2F000818383E080A78FE084A78FE187A780AB2D
:10E3000081AB5EDFE6CF1F93CF93DF93EC01162F37
:10E31000E0DF8091BD058093DF0587E38093E00512
:10E3200086E08093E1056AE070E088EE93E00F9468
:10E33000124C9091BC0591509093BC05992351F0DB
:10E340001092DE0518831092BD0510929906109266
:10E35000980601C01882DF91CF911F9108952F92E6
:10E360003F925F926F927F928F929F92AF92BF92F5
:10E37000CF92DF92EF92FF920F931F93CF93DF9391
:10E380001F92CDB7DEB784E08093220280919A0677
:10E39000882309F470C280919806909199068E3175
:10E3A000910514F08DE190E097FF02C080E090E0CD
:10E3B0009093990680939806880F991F880F991F4C
:10E3C0002091BD05422F022E000C550B481759070E
:10E3D00074F42D5FAC01421B510927FD5395423067
:10E3E00051051CF02093BD0502C08093BD0520910E
:10E3F000BD05422F022E000C550B841795077CF4A7
:10E400002350422F022E000C550B481B590B423053
:10E4100051051CF02093BD0502C08093BD0580917D
:10E420002806882309F427C22091FC05222349F0FD
:10E430009091FB05920F9093FB05933F14F410927B
:10E44000FC05823070F0815080932806823011F4F0
:10E450004BDF11C2843609F00EC281E0809328069A
:10E460000AC28091E8058F5F8093E8054091E60538
:10E4700090E0242F30E035952795281739070CF0C8
:10E48000B3C09091FD0581E089278093FD0510922E
:10E49000E805442309F4A8C09091E2058091BA05EB
:10E4A000890F2091E305821724F02091E4052817B5
:10E4B000D4F491959093E2052091BB052B5F2093B6
:10E4C000BB058093BA058091E5053AE08302C0015F
:10E4D0001124820F911D27FD9A95C99724F064E1BC
:10E4E00088E296E010DF9091E2058091BA05890FED
:10E4F0008093BA058091E605882309F475C024E16C
:10E5000030E040E050E060E070E0CB010E94643910
:10E51000672B682B692B09F067C0E0ECF5E080E021
:10E5200090E0208121115AC09C01220F331F8901E4
:10E53000080F191FC80182549A4F892B09F454C03F
:10E540002091E60530E02F5F3F4F032E000C440B77
:10E55000550B60E070E0CB010E946439FB01E6548A
:10E56000FA4F42A9242F30E0B4E035952795BA95AB
:10E57000E1F7F901E257FC4F808190E006541A4F11
:10E580004F705091BA056EE0469F500D1124452FF3
:10E59000FC01E557FC4F5081450FFC01E857FC4F4B
:10E5A00090819695842F890FF80184838091BB0513
:10E5B00082502F5F3F4FFAE02F9F800D1124F8010A
:10E5C000858322E030E040E050E060E070E0CB0185
:10E5D0000E9464396E5FF801668306C00196339627
:10E5E0008A30910509F09DCF9091DE05992341F085
:10E5F0008091DD05890F8093DD0587FD1092DE0592
:10E600008091DE05882309F4A2C02091DD05E09108
:10E61000BB052E170CF49BC0022E000C330B0E2EE4
:10E62000000CFF0BCF014D96821793070CF48FC09F
:10E630001091BA05E090DC05CE2C0E2C000CDD0804
:10E64000C601811B910917FD93956EE070E00F9450
:10E650004655F62E653008F07AC02E1B3F0BC901D7
:10E6600002966AE070E00F944655062F633008F07A
:10E670006EC0812C912C540183940F2C04C0880C03
:10E68000991CAA1CBB1C0A94D2F7A62F660FBB0BC1
:10E69000BD0166547A4FFB0197A5892F882109F4A3
:10E6A00056C0FD01E257FC4FE0814E2F50E0812F14
:10E6B000FEE0FF9E800D11249A0125573C4FF90181
:10E6C000F080F80EEF140CF442C0FA01E857FC4F4A
:10E6D0001081412F50E04F0D511DF7FC5A95C41683
:10E6E000D506ACF51092DE05282D20952923FB01D7
:10E6F00027A723E030E02A1B3B0B8091290690914D
:10E700002A06280F391F30932A06209329066AE02B
:10E7100070E088E290E00F94124C2091BB05FAE083
:10E720000F9F200D1124912F96958F2D890F8550C5
:10E730008093DF052093E00584E08093E1058091DC
:10E74000E60581508093E605882321F039DD00EC51
:10E7500015E012C084E180932806BBDDF8CF8291DA
:10E76000890F808380346CF0F80110820D5F1F4F99
:10E77000F5E00E3D1F07E9F0F80190819923B1F310
:10E78000EECF87339CF3F801329720818091BD054D
:10E79000281764F3022E000C330B082E000C990B83
:10E7A0000A968217930714F368E788E296E0ABDDD8
:10E7B000DDCF8091FC05811124C024EF31E040E0E1
:10E7C00050E060E070E0CB010E946439672B682B59
:10E7D000692BB9F422E030E040E050E060E070E006
:10E7E000CB010E946439672B682B692B09F098C113
:10E7F0008FEF8093FC05813009F494C18FE78093FB
:10E80000FB058091DE058823B1F18091FC0588230A
:10E8100091F18091DD05873074F52091DC058091C0
:10E82000FB05281744F1022E000C330B082E000CB8
:10E83000990B0C9682179307F4F01092FC05109236
:10E84000DE058091290690912A060A9690932A0661
:10E85000809329066AE070E088E290E00F94124C01
:10E860008091FB058F5F8093DF0581E08093E00559
:10E8700084E08093E1058091A20682FF04C080912C
:10E88000E705815001C08AE08093E7050E94B980C6
:10E890008823C1F080912806811103C01092E705FA
:10E8A00011C0813079F48091DE0581110BC0809117
:10E8B000BD058B5F8093DC0584E38093DD058CEFE1
:10E8C0008093DE058091E705811101C0EAD161E006
:10E8D0008CE694E00E94FB333091BB05632F032E3E
:10E8E000000C770B8091E505AB012AE08202400D18
:10E8F000511D1124425051098091A00490E08417C9
:10E9000095072CF08091FC0581116BC06FC0809140
:10E91000A20490E086179707ACF3FEE86F2EF3E0B1
:10E920007F2EC12CD12CF30121913F01432F032EC7
:10E93000000C550BBA01695F7F4F8091A00490E0F5
:10E94000681779074CF4365FFFEFCF1ADF0A23E030
:10E95000C216D10441F7D6CF8091A20490E084176B
:10E9600095078CF31091BA0546E4542E510EA12C54
:10E97000B12CC60186549A4F4C01822F90E01C01A5
:10E98000220C331CF40187A590E0A0E0B0E00A2C33
:10E9900004C0B695A795979587950A94D2F780FFFE
:10E9A00019C08091FD057101E80EF11CC701E4E07A
:10E9B000880F991FEA95E1F7AC014759514D7A014B
:10E9C00008E022E0432F612F8CE694E039830E9417
:10E9D00025343981125F5FEFA51AB50A1511D2CF20
:10E9E000B2CF8091A004883008F49EC080912806A0
:10E9F000882369F09091A0049F3348F49091A20479
:10EA0000973328F0823008F49DC081FD9BC080912F
:10EA1000DE058823B1F04091DD05242F042E000C83
:10EA2000330BB9016D5F7F4F8091A00490E06817B0
:10EA300079073CF08091A20490E0821793070CF0D4
:10EA40008FC000E010E0F801E654FA4F8681882379
:10EA500099F04581842F042E000C990B2091A0047D
:10EA600030E08217930744F002972091A20430E02F
:10EA7000281739070CF07CC00D5F1F4F0E311105B0
:10EA800011F78091E1058823B1F04091E005242F32
:10EA9000042E000C330BB9016A5F7F4F8091A004F4
:10EAA00090E0681779073CF08091A20490E082170B
:10EAB00093070CF065C080912806811101C0B4D085
:10EAC0008091A0048A3008F06DC069E080E00E9467
:10EAD000C53A8091290690912A060E94CA3A8091EF
:10EAE000BC05882309F45EC011E060E1C62ED12C7C
:10EAF0008091BC05811708F455C0B601611B7109EE
:10EB0000660F660F660F74E5E72E7EE2F72E05E0CE
:10EB100021E041E08CE694E00E9425341F5FE8CFBD
:10EB200081E067CE83EF6BCE2CE3E22E2EE2F22E55
:10EB300005E022E042E06091FB058CE694E00E9453
:10EB4000253454CF99E5E92E9EE2F92E08E022E023
:10EB500047E36091BD058CE694E00E94253457CFD1
:10EB600024E06091DC058CE694E00E942C3669CFAD
:10EB7000425023E064818CE694E00E942C367CCFE6
:10EB800086E4E82E8EE2F82E07E022E06091DF05B1
:10EB90008CE694E00E9425348091E10581508093B9
:10EBA000E10589CF0F90DF91CF911F910F91FF90D9
:10EBB000EF90DF90CF90BF90AF909F908F907F901D
:10EBC0006F905F903F902F900895CF93DF936FEAFF
:10EBD00071E784E155D0CAEBD5E083E08A838AE00F
:10EBE0008DA71CA281DB1B821092990610929806B9
:10EBF000DF91CF91089580919A06882319F082E0E1
:10EC00008093B90584E080932202809128068823AE
:10EC100049F09091B9058FEF890F8093B90581E094
:10EC200019160CF080E008950F938091A0048532AE
:10EC300028F58091A2048B3108F160E08CE694E025
:10EC40000E94FB3309E028E34BE164E28CE694E0A8
:10EC50000E949D3661E08CE694E00E94FB330E94A6
:10EC60000282882359F063E285E20E94C53A6FEF81
:10EC70007FEF89EC9EE20F910C941F3B0F9108955A
:10EC8000FB0110922A06109229068093280620E0A4
:10EC900040E060E070E0CF0153D581E08093A006B2
:10ECA00008951092A0067FC58091BF059091C1057F
:10ECB00089130DC08091C0059091C205891714F089
:10ECC0002FEF01C021E0820F8093C00508C0891793
:10ECD00014F02FEF01C021E0820F8093BF0589134C
:10ECE0001BC02091270621502093270630E0832F58
:10ECF00090E0DC01AA0FBB1FA654BA4F880F991FE2
:10ED0000FC01E454FA4F8581968116969C938E936C
:10ED100015973F5F231758F70895EF92FF921F93BF
:10ED2000CF93DF93109127062091BC05E22E022E8F
:10ED3000000CFF083091BB05C32F032E000CDD0B28
:10ED4000E2ECF5E040E0411709F446C0CF0103973B
:10ED5000DC019C91BF0161507109DB018C9198131A
:10ED60001DC0692F092E000C770B61507109C61761
:10ED7000D70711F039132DC09081BF01625071097E
:10ED8000DB018C91582F98170CF4592F25170CF193
:10ED900089170CF4892F8217E4F020C0BF0162505C
:10EDA0007109DB015C91652F052E000C770B61501A
:10EDB0007109E616F70611F025130BC0582F9817A6
:10EDC0000CF4592F35172CF089170CF4892F831761
:10EDD0002CF44F5F3296B7CF80E001C081E0DF9125
:10EDE000CF911F91FF90EF90089528E130E040E02F
:10EDF00050E060E070E0CB010E9464396093BB0595
:10EE00002AE030E040E050E060E070E0CB010E949A
:10EE100064396093BC0581DF8111E7CF089590913B
:10EE2000BA05811102C08FEF01C081E0980F937085
:10EE30009093BA05809127068F5F8093270690E014
:10EE4000FC01EE0FFF1FE654FA4F209124062583A4
:10EE5000880F991FFC01E054FA4F809126068083A9
:10EE600008951F93CF93DF93CAEBD5E080E091E044
:10EE7000909324068093230680E095E090932606E5
:10EE8000809325061882109227061D8215E01E83A6
:10EE900081E0C5DF1B8310929906109298061C82B0
:10EEA000DF91CF911F910895EF92FF920F931F93DF
:10EEB000CF93DF9380912706843008F4DEC090E082
:10EEC000FC01EE0FFF1FE854FA4F3581FC01EE0FF5
:10EED000FF1FE654FA4F6581AC01425051093617C5
:10EEE00039F0C0E0880F991FFC01E254FA4F82C04C
:10EEF000F12CDC01AA0FBB1FA054BA4F880F991F39
:10EF0000FC01E254FA4F8F2D90E0841795070CF026
:10EF1000B4C0BC01660F771F66547A4FEB016D8158
:10EF20008C01000F111F04541A4FE8012D81621744
:10EF3000F1F0722F62170CF4762F3717ECF12617C9
:10EF40000CF4262F2317C4F1880F991F80549A4F71
:10EF5000EC01288191E0808128170CF090E081E09D
:10EF60006C9162170CF480E0981731F188C0361369
:10EF700023C07C9120818C01000F111F0E531A4F6A
:10EF8000E8016881880F991F80549A4FEC018881AD
:10EF9000122F72170CF4172F982F86170CF4962F38
:10EFA000911754F0922F27170CF4972F68170CF431
:10EFB000862F98170CF063C0F394A5CF7C01DFEF88
:10EFC000ED1AFD0A8C01000F111F00541A4FD801D1
:10EFD0007C918C01000F111F0E531A4FD8012C91F8
:10EFE000721729F1A081B22F72170CF4B72FAB174B
:10EFF0003CF4CF5F8C2F90E084179507FCF23DC066
:10F0000027170CF4272F2A17A4F3880F991FDC0168
:10F01000A654BA4F15962C9191E023170CF090E06E
:10F0200081E062170CF480E0981719F328C0208162
:10F030002713DFCFD701AA0FBB1FA654BA4F1596CF
:10F040002C91880F991FDC01A654BA4F15968C910C
:10F05000762F36170CF4732F982F82170CF4922FFB
:10F0600097173CF2962F63170CF4932F28170CF484
:10F07000822F98170CF4BDCF02C080E001C081E060
:10F08000DF91CF911F910F91FF90EF900895BF9264
:10F09000CF92DF92EF92FF920F931F93CF93DF9364
:10F0A0001F92CDB7DEB7A7DD882309F486C0809113
:10F0B000230690912406392F40912506509126066B
:10F0C0002091BA05213061F02CF4211116C0CA013B
:10F0D000C3970AC0223031F0233079F4C39709C0B6
:10F0E000C39607C0CA01C39690932606809325064F
:10F0F00004C0909324068093230610912406009167
:10F100002606311303C0051709F457C0183110F44F
:10F110000A3048F01092280668E270E080E991E039
:10F120000F94124C4AC08091270690E0FC01EE0F2C
:10F13000FF1FE654FA4F1583880F991FFC01E05416
:10F14000FA4F0083809198069091BE05282F291BC5
:10F1500039F08093BE0581E012160CF080E05FDE8E
:10F160008091BD05882321F081508093BD0501C0A9
:10F170009BDD9ADE8111CECF8091BB0518131DC097
:10F180008091BC05081319C06CED70E085E090E03B
:10F190000F94124C68E171E085E090E00F94124CFE
:10F1A0008091290690912A06019690932A068093D1
:10F1B000290682E08093BD0518DE61E08CE694E0CC
:10F1C0000E94FB338091A004893050F467E080E016
:10F1D0000E94C53A8091290690912A060E94CA3A57
:10F1E00006E32CE749E062E08CE694E00E944D36AD
:10F1F00010E0809127063091A004181708F084C011
:10F20000412F50E0BA01660F771FFB01E654FA4F19
:10F21000A581FB01E454FA4F2581CA010396A2138C
:10F2200051C0FB01EE53FA4F2081880F991FFC015A
:10F23000E654FA4FC080DC2CC2160CF4D22E8D2D71
:10F2400095E08902A0011124425F5F4F832F90E077
:10F25000481759070CF456C02C150CF4C22EEC2D8F
:10F26000F5E0EF0290011124265F3F4F8091A20448
:10F2700090E0281739070CF045C08C2D880F880FB7
:10F280008C0DEBE0BE2EB80ECB0181549A4F7C0161
:10F29000DC14C4F12B2D0B2C000C330BA9014D5F9A
:10F2A0005F4F8091A00490E0481759073CF080918F
:10F2B000A20490E0821793070CF053C0C39495E02A
:10F2C000B90EE6CF880F991FFC01E654FA4F8081F2
:10F2D000982F990F990F890F5BE0E52EE80E4E2DC0
:10F2E0000E2C000C550BBA016D5F7F4F832F90E001
:10F2F000681779073CF06091A20470E06417750705
:10F300000CF03EC01F5F75CF4091BC05842F880F65
:10F31000880F480F455F642F042E000C770BFB010C
:10F320003396832F90E0E817F9073CF08091A20410
:10F3300090E0861797070CF045C080912806811150
:10F3400001C072DC16D7882309F44AC00F90DF9100
:10F35000CF911F910F91FF90EF90DF90CF90BF90D2
:10F36000A0CCF7016081862F880F880F680F6C5F33
:10F3700004E024E04B2D8CE694E00E949D369ECF65
:10F38000D22EA2170CF4DA2EC22E2A170CF4CA2E93
:10F39000FD2CFF0CFF0C8F2D8D0D30E094E0F92E2D
:10F3A000F80ECD140CF4AECF6F2D630F04E024E003
:10F3B0004E2D8CE694E039830E949D36D39439819A
:10F3C0003B5FEFCF6091BB05862F880F880F680FDA
:10F3D0006C5F04E024E08CE694E00E944D36ADCFF3
:10F3E0000F90DF91CF911F910F91FF90EF90DF90E1
:10F3F000CF90BF90089567E478E781E041DC31DD8C
:10F40000F4CC0F931F93CF93DF9361E081E0A1D2FF
:10F41000D0917206C0E0D11116C0809171068111A1
:10F4200003C0A7D681119AC080912202882309F4D3
:10F430003CC081E090917106911180E004E024E0ED
:10F4400042E25FE22FC0D130B1F480917106813089
:10F4500019F48FD6811189C080912202882329F165
:10F4600081E090917106913009F080E003E02EE395
:10F4700040E15FE217C0D230C1F480917106823062
:10F4800019F477D681117BC080912202882369F01C
:10F4900081E090917106923009F080E003E02EE364
:10F4A00041E05FE26C2F0E94064433D1182FD33025
:10F4B000D1F480917106833019F45BD6811169C053
:10F4C00080912202882309F476C081E09091710630
:10F4D000933009F080E000E22EE342EF5EE26C2F11
:10F4E0000E94064468C0811168C0D430B1F4809194
:10F4F0007106843019F43DD6811152C080912202E8
:10F50000882319F181E090917106943009F080E030
:10F5100000E22EE344EE5EE215C0D530B1F48091F6
:10F520007106853009F443C080912202882369F076
:10F5300081E090917106953009F080E000E22EE3C1
:10F5400043ED5EE26C2F0E94064486E0CF5FDF5FF2
:10F55000C53009F060CF809370063AC024D1809105
:10F560003E06882309F460CF33C08DE39EE40E94F9
:10F57000124880913E06882309F46ECF29C08FE09F
:10F580009DE70E94124880913E06882309F47CCFB3
:10F590001FC0CFD280913E06882309F491CF18C0B6
:10F5A000CBD280913E06882309F4A8CF11C0E1D5C3
:10F5B000811105C0B9CF112341F284E0C7CF0E9469
:10F5C00046D581E018D280913E06882309F4ACCF5D
:10F5D000DF91CF911F910F910895E0913F06E630A2
:10F5E00000F581E08E0F80933F0680919806909100
:10F5F0009906A0E0B0E0309172062091700648E0D4
:10F60000E49FF0011124E05CF94F40919306509182
:10F6100094065183408382839383A483B583368386
:10F62000278308950D940F3A2F923F924F925F9245
:10F630006F927F928F929F92AF92BF92CF92DF9202
:10F64000EF92FF920F931F93CF93DF9300D000D0E0
:10F65000CDB7DEB71C012B833C834D835E8369836A
:10F660007A83BBDF83E08093220230923D062092B2
:10F670003C0669817A8170933B0660933A062B8140
:10F680003C814D815E81209336063093370640934E
:10F69000380650933906E0923206F0923306009312
:10F6A000340610933506D0929906C0929806B0920F
:10F6B0009406A092930690923106809230068C8D2B
:10F6C00080932F0626960FB6F894DEBF0FBECDBFEF
:10F6D000DF91CF911F910F91FF90EF90DF90CF902E
:10F6E000BF90AF909F908F907F906F905F904F9062
:10F6F0003F902F900895FB01908181E089278083BE
:10F7000083E0809322024115510511F0FA0119940A
:10F7100008958091CF0E9091CC0E891B8F7071F45B
:10F7200090917E0992FB882780F992FD08C081E0C4
:10F730009091EE16913019F080E0089581E00895DF
:10F74000E0919306F0919406E817F90721F13091C2
:10F75000A30637FD1092A306909394068093930618
:10F7600070939906609398064093720620937006F2
:10F770008951904821F41092A00610923F060E94F1
:10F780003C4382E08093220281E080933E06109207
:10F790009B0610922B06089520E040E060E070E0A8
:10F7A00089E190E8CDCFE0913F06EE2381F0E15072
:10F7B000E0933F0688E0E89FF0011124E05CF94FF8
:10F7C0002781468160E070E080819181B9CFE4CFEC
:10F7D000CF93DF93FC01EB018091980690919906FD
:10F7E00097FF04C010929906109298064091320635
:10F7F00050913306609134067091350680919806D9
:10F8000090919906092E000CAA0BBB0B48175907BB
:10F810006A077B0724F450939906409398068091D9
:10F8200022028823D1F02091980630919906809188
:10F83000360690913706A0913806B0913906BC0182
:10F84000CD01620F731F811D911D1995BC0180911F
:10F850003C0690913D060E949B4480918D0681114B
:10F8600008C080912F06882381F18091220288238D
:10F8700061F180913A0690913B06009791F02091BA
:10F88000980630919906409136065091370660915E
:10F89000380670913906420F531F611D711DFE011C
:10F8A0001995E0913006F0913106309741F0809142
:10F8B0002F06811103C080918D068111199559D4AD
:10F8C000882319F0DF91CF916ECFDF91CF9108950A
:10F8D0000F931F93CF93DF9380912202882359F0D7
:10F8E00060912C0670912D0600E010E020E041E0D0
:10F8F00081E00E94A34380912E0681111CC081E00B
:10F9000080932E06C0919306D091940620E040E0AB
:10F9100060E070E088E69CE713DF0E949BF11092A4
:10F920002E0620E040E060E070E0CE01DF91CF9154
:10F930001F910F9105CFDF91CF911F910F910895E6
:10F94000009711F486E39FE290932D0680932C0696
:10F95000BFCF282F10929206809198069091990619
:10F960008130904820F0109299061092980680916C
:10F970009A06882331F08091980680937106109240
:10F980003E06809170061816BCF4082E000C990BE8
:10F99000821B910920917106022E000C330B28174F
:10F9A000390754F097FF02C080E090E08093710621
:10F9B0009093990680939806809171066623C1F012
:10F9C00090917206891714F4809372062091720642
:10F9D000022E000C330B2C5F3F4F482F082E000CDB
:10F9E000550B2417350734F484508093720608951C
:10F9F000809372060895882361F063E972E084E6DB
:10FA000090E00F94124C6AEB72E084E690E00D9463
:10FA1000124C68EB71E084E190E00D94124CCF92AF
:10FA2000DF92EF92FF92CF93DF93A3D3882349F025
:10FA30001092A006DF91CF91FF90EF90DF90CF90D2
:10FA4000B2CE81E08093A006C0919806D09199062D
:10FA5000209709F442C01092990610929806BE01B0
:10FA60000D2E000C880B990B0F94B1522091690E4A
:10FA700030916A0E40916B0E50916C0E0F944D5464
:10FA80002091A90D3091AA0D4091AB0D5091AC0D74
:10FA90000F9436516B017C0120E030E040E050ECE7
:10FAA0000F94125487FD19C020E030E040EA50E482
:10FAB000C701B6010F940F5218167CF0BE0182E008
:10FAC0000E9498A7C092A90DD092AA0DE092AB0D0A
:10FAD000F092AC0D82E08093220280912202882372
:10FAE000C9F089EA9DE00F942C46BC0187E29FE2B1
:10FAF0000E949B446091A90D7091AA0D8091AB0D5D
:10FB00009091AC0DDF91CF91FF90EF90DF90CF906F
:10FB10000C94CA45DF91CF91FF90EF90DF90CF908A
:10FB2000089521E020932E060F94143A10922E0689
:10FB300008950E948CD15FCF0E9447E05CCF209156
:10FB40009806309199062115310559F081E0121679
:10FB500013060CF080E080932B0610929906109209
:10FB6000980680912B0608954F925F926F927F9234
:10FB70008F929F92AF92BF92CF92DF92EF92FF92BD
:10FB80000F931F93CF93DF931F921F92CDB7DEB7D2
:10FB90005C014A01390128018701760169837A8372
:10FBA000CEDFD82EE6D2C82E69817A81811104C0B9
:10FBB000809122028823F9F092014D2DC5010E9407
:10FBC0006E45CC20C1F0DD2011F0F40101C0F3013D
:10FBD0000F900F90DF91CF911F910F91FF90EF90B9
:10FBE000DF90CF90BF90AF909F908F907F906F905D
:10FBF0005F904F9019940F900F90DF91CF911F91CC
:10FC00000F91FF90EF90DF90CF90BF90AF909F90BB
:10FC10008F907F906F905F904F900895FC0180814E
:10FC20000895FC01849108954F925F926F927F92A4
:10FC30008F929F92AF92BF92CF92DF92EF92FF92FC
:10FC40000F931F93CF93DF936C017B015A0129011E
:10FC5000672B31F088248394912CC0E0D0E019C048
:10FC6000F8011182108227C03701680C791C769444
:10FC70006794E3012197A201BE01C601F501199520
:10FC80001816190654F0892BC9F04301FFEF8F1A9B
:10FC90009F0AE814F90440F702C07E01FACFCE159E
:10FCA000DF0530F4CE0102968816990620F02196E1
:10FCB000F801D183C0838FEF9FEF05C0F801D18396
:10FCC000C08380E090E0DF91CF911F910F91FF9072
:10FCD000EF90DF90CF90BF90AF909F908F907F90EC
:10FCE0006F905F904F9008958F929F92AF92BF92C6
:10FCF000CF92DF92EF92FF920F931F93CF93DF93F8
:10FD0000EC016B017A01FB01199587FD06C0082FF4
:10FD100010E020E030E0219620C1982F907E903CAA
:10FD2000C1F4082F0F7110E020E030E048015901C4
:10FD300086E0880C991CAA1CBB1C8A95D1F7CE01C1
:10FD40000196F60119958F7395018401082B22966F
:10FD500004C1982F907F903E19F58F70882E912CBA
:10FD6000A12CB12C16E0880C991CAA1CBB1C1A955E
:10FD7000D1F7CE010196F60119958F73882A06E016
:10FD8000880C991CAA1CBB1C0A95D1F7CE010296BF
:10FD9000F60119958F7395018401082B2396DDC018
:10FDA000982F987F903F81F58770882E912CA12CF9
:10FDB000B12CF6E0880C991CAA1CBB1CFA95D1F753
:10FDC000CE010196F60119958F73882AA6E0880C5A
:10FDD000991CAA1CBB1CAA95D1F7CE010296F6016C
:10FDE00019958F73882AB6E0880C991CAA1CBB1C35
:10FDF000BA95D1F7CE010396F60119958F73950147
:10FE00008401082B2496A9C0982F9C7F983FE9F580
:10FE10008370882E912CA12CB12C56E0880C991C53
:10FE2000AA1CBB1C5A95D1F7CE010196F601199573
:10FE30008F73882A66E0880C991CAA1CBB1C6A95E3
:10FE4000D1F7CE010296F60119958F73882A76E0D4
:10FE5000880C991CAA1CBB1C7A95D1F7CE0103967D
:10FE6000F60119958F73882AE6E0880C991CAA1C64
:10FE7000BB1CEA95D1F7CE010496F60119958F7354
:10FE800095018401082B259668C0982F9E7F9C3F82
:10FE900009F04AC08170882E912CA12CB12C86E0EB
:10FEA000880C991CAA1CBB1C8A95D1F7CE0101961F
:10FEB000F60119958F73882A96E0880C991CAA1C64
:10FEC000BB1C9A95D1F7CE010296F60119958F7356
:10FED000882A26E0880C991CAA1CBB1C2A95D1F7FD
:10FEE000CE010396F60119958F73882A36E0880CA7
:10FEF000991CAA1CBB1C3A95D1F7CE010496F601B9
:10FF000019958F73882A46E0880C991CAA1CBB1C83
:10FF10004A95D1F7CE010596F60119958F73950193
:10FF20008401082B269619C0982F907C903849F4AC
:10FF3000082F007C003871F42196CE01F601199546
:10FF4000F7CF082F0E7F0D3F28F02196CE01F60146
:10FF50001995F7CF00E010E09801E114F10429F0C1
:10FF6000F7010083118322833383CE01DF91CF9188
:10FF70001F910F91FF90EF90DF90CF90BF90AF90C7
:10FF80009F908F9008951F93CF93DF9300D01F927F
:10FF9000CDB7DEB710E0AE014F5F5F4F6EE07EE79A
:10FFA000A3DE49815A816B817C81452B462B472BEF
:10FFB00011F01F5FF0CF812F0F900F900F900F90D7
:10FFC000DF91CF911F9108951F93CF93DF9300D0BE
:10FFD0001F92CDB7DEB710E0AE014F5F5F4F61E11A
:10FFE0007EE782DE49815A816B817C81452B462BDD
:10FFF000472B11F01F5FF0CF812F0F900F900F90C4
:020000021000EC
:100000000F90DF91CF911F910895FC01A081B181E4
:100010001C92A281B3818C918F5F8C930280F381BB
:10002000E02D80816CE0689F600D112480E00C94CD
:10003000C53A1092920680918D0610928D06882303
:1000400049F020E040E060E070E081E496E678DB93
:100050000C94084320916302309164024091980609
:1000600050919906C901840F951F2436310551F42A
:100070004730510514F0069720C04A3F5F4F64F5A2
:1000800006961BC02436310524F48536910524F5E7
:1000900004C08436910524F41FC08A3091053CF0D9
:1000A000883E43E094072CF087EE93E002C08AE09C
:1000B00090E02817390731F40DC08A30910584F794
:1000C0008AE090E090936402809363021092990614
:1000D000109298060C949A3B84E690E0E1CFCF937F
:1000E000DF931F92CDB7DEB780912F09811103C036
:1000F00081E799E02FC0211103C08FE299E02AC067
:100100008DE0815048F0440F411DE82FF0E0EF589A
:10011000F64F90814927F5CF809184068417A9F086
:10012000409384068FE299E069832DDF90E0698136
:10013000861B910997FF02C080E090E080939506AE
:100140001092960688E0809324028091960690E0B3
:10015000815D964F0F90DF91CF9108958093920625
:1001600010928E0610928F061092900610929106B1
:10017000089580918D0610928D0608957F928F923A
:100180009F92AF92BF92CF92DF92EF92FF920F9326
:100190001F93CF93DF93CDB7DEB728970FB6F894B0
:1001A000DEBF0FBECDBF7C014B016A015901FB01CF
:1001B00080816CE0689F600D1124F7018081982F89
:1001C000990F890F880F0E94C53AC114D10409F410
:1001D00096C0FE82ED8298868F82011103C01C2D8D
:1001E0000D2D74C09D2C0C2D1D2DD12C8824839495
:1001F000AE014F5F5F4FB5018C2D992D75DDC82E77
:10020000992E89819A81AB81BC8177247394009760
:10021000A105B105C9F0712C80329105A105B10588
:1002200081F0AC01BD014D525109610971094230A3
:1002300051056105710540F08B97A105B10589F560
:1002400003C0DD2009F455C0F70120818D2D90E019
:10025000820F911D46972CF0253018F0CE0105969F
:10026000D4DE372D3825D30EF70180818D0D8083A4
:10027000DD2089F0DA94AE014F5F5F4FB501C80110
:1002800033DD8C0169817A818B819C814FEF5FEF37
:100290000E94D03AEDCF711032C00C2D192DD12C07
:1002A000A7CFD3940115110509F0A2CF0C2D192D5C
:1002B0009FCF4FEF5FEF0E94D03AF70120812F5F71
:1002C0002083253118F0CE0105969FDEAE014F5FE9
:1002D0005F4FB501812F902F07DD182F092F6981FE
:1002E0007A818B819C81611571058105910509F7E2
:1002F00006C00115110589F20F5F1F4FD3CF289655
:100300000FB6F894DEBF0FBECDBFDF91CF911F9126
:100310000F91FF90EF90DF90CF90BF90AF909F90A4
:100320008F907F900895AF92BF92CF92DF92EF921D
:10033000FF920F931F93CF93DF931F921F92CDB71E
:10034000DEB75C016B017A013FDE182FE114F10486
:1003500019F0C70139DE01C080E01A821982C11488
:10036000D104C1F4412F50E090E09A01280F391FC9
:10037000263131057CF425E130E0241B350B281BA8
:10038000390B37FF02C02F5F3F4F359527952A83E2
:1003900081E0898301E021E13EE7A501BE016F5FB5
:1003A0007F4FCE010296EADEC114D10489F08A8122
:1003B000882321F01A8289818F5F898300E02EE0F3
:1003C0003EE7A601BE016F5F7F4FCE010296D6DEEB
:1003D000E114F10451F000E021E13EE7A701BE0184
:1003E0006F5F7F4FCE010296C9DE0F900F90DF91B5
:1003F000CF911F910F91FF90EF90DF90CF90BF9022
:10040000AF900895CF92DF92EF92FF920F931F93D8
:100410000E94C82E009180061091810620918206CC
:10042000309183066B017C01C01AD10AE20AF30AFB
:10043000F7FC13C020917F06209520937F06DC01F6
:10044000CB018A549C4FAF4FBF4F8093800690934F
:100450008106A0938206B093830681E090917F0687
:10046000911101C080E01F910F91FF90EF90DF90FC
:10047000CF900895CF9393E0909322028111109230
:10048000A2060E94C82EDC01CB018C509E4FAF4FBC
:10049000BF4F80939C0690939D06A0939E06B093B9
:1004A0009F0668E873E182E090E00F94124CC6E08A
:1004B000C15049F00F94A74B62E070E080E090E0FB
:1004C0000E94F92EF5CFCF910895AF92BF92CF92AF
:1004D000DF92EF920F931F93CF93DF9300D01F9281
:1004E000CDB7DEB7809123028F3F09F444C00E944C
:1004F000C82E0091850610918606209187063091BE
:100500008806DC01CB01801B910BA20BB30BB7FD5E
:1005100032C09091CC0E8091CF0E8F5F8F70981764
:1005200051F1E091230284E0E802F0011124EF563A
:10053000FC4F20E030E040E752E46081718182812D
:1005400093810F94165269837A838B839C83A12CA9
:10055000B12C6501E12C8E010F5F1F4F25E732E0C2
:1005600041E752E06DE672E089E692E00E94FDFE0E
:100570008FEF809323020F900F900F900F90DF91D9
:10058000CF911F910F91EF90DF90CF90BF90AF90E0
:1005900008950F931F930E94C82E00919C061091FE
:1005A0009D0620919E0630919F06DC01CB01801BA9
:1005B000910BA20BB30BB7FD11C08091030181FB1E
:1005C000992790F981E089279091030192FF826039
:1005D0009091000196FF84608093A2068091A2060C
:1005E00081709091A20691FD8260909173068917A7
:1005F00041F18130A9F028F0823041F0833059F088
:100600001EC0913089F09230A9F019C0992361F091
:10061000933081F014C0913069F0923081F404C0BD
:10062000992341F0933059F490919706915090930B
:10063000970605C0909197069F5F909397068093C9
:1006400073061F910F910895CF93DF930E94084383
:10065000E4E0F1E080818D7F8083C5E0D1E0888196
:100660008095827043E051E0DA018C9380818B7F2A
:1006700080838881809584708C9321E031E0D9015A
:100680008C918F7B8C9380910201809580748093F4
:10069000000180818E7F8083888180958170FA013E
:1006A000808382E08093A10674DF10929706DF9129
:1006B000CF910895CF93C091E80684EA96E063DC79
:1006C000C81790F48091E8068F5F21E0280FE82F8B
:1006D000F0E0EC55F94F9081907C903811F4822F26
:1006E000F4CF8093E80602C01092E806CF910895F7
:1006F0000F931F93CF93DF938C01C091E806D0E056
:10070000CC55D94FCE013FDCF8018083CE01DF917B
:10071000CF911F910F91089581E09091A4069111BE
:1007200001C080E00895CF93DF932091E706211167
:1007300020C0FC0101900020E9F73197EF01C81BB0
:10074000D90BC334D10534F031972081207C203877
:10075000D9F3F4CFBC01DD27AE0184EA96E00F9413
:100760009D5ACC55D94F18821092E80683E08093A9
:100770002202DF91CF910895CF93DF93CDB7DEB7FB
:100780008E819091E706891790F08093E7069E018D
:10079000275F3F4F4F81588562E470E084EA96E01E
:1007A0000F94E65A1092E80683E080932202DF91CC
:1007B000CF9108950F931F93CF93DF938C0167FF21
:1007C00003C01092E70660E08091E70690E0262FD4
:1007D000062E000C330B281739071CF16093E7062F
:1007E000C8010F94FF59F801E80FF91FEF01C01B72
:1007F000D10BC334D10534F031978491807C80389B
:10080000D9F3F4CFDD27AE01B80184EA96E00F9466
:10081000205ACC55D94F18821092E80683E0809375
:100820002202DF91CF911F910F9108954F925F9215
:100830006F927F928F929F92AF92BF92CF92DF92F0
:10084000EF92FF920F931F930E94C82E6B017C01C1
:100850003CDE9FDE8091A20682FF15C080917E065D
:10086000811113C091E090937E062091FB16211117
:1008700003C080912E06892780938D061092FB1667
:1008800081E0F8DD02C010927E0680910301809520
:1008900081701091A106811749F18093A1068823E8
:1008A00009F4CAC164EF71E080E090E00E94A39F68
:1008B0000E945B90123009F0BAC10E9432910E94EE
:1008C000084383E0809322020E94C82E6B017C01C2
:1008D000DC01CB018C599F4FAF4FBF4F80937A06FD
:1008E00090937B06A0937C06B0937D0680917A0658
:1008F00090917B06A0917C06B0917D06A7019601A0
:10090000281B390B4A0B5B0B57FF05C080919B06D8
:10091000882309F41DC2D701C6018C599F4FAF4FE0
:10092000BF4F80937A0690937B06A0937C06B0938A
:100930007D0660919706062E000C770B77FF03C0AB
:10094000719561957109062E000C770B880B990B38
:100950000F94B1522B013C0120E030E040E050E424
:100960000F94125487FF05C080918D0681117DC0C0
:100970008DC080919206882309F456C080908E061F
:1009800090908F06A0909006B090910681149104EB
:10099000A104B104E1F120E030E040E05FE3C301F5
:1009A000B2010F944D542B013C01C701B6016819E7
:1009B00079098A099B090F94AF529B01AC01C301CD
:1009C000B2010F94165220E030E04AE754E40F944D
:1009D0004D544B015C0120E030E040EA52E40F94BA
:1009E000125487FF0FC020E030E040EF51E4C50112
:1009F000B4010F94125487FD0AC02AE030E040E0B1
:100A000050E009C024E630E040E050E004C021E0BE
:100A100030E040E050E0C0928E06D0928F06E09227
:100A20009006F092910604C021E030E040E050E0F2
:100A3000A091970600919806109199060A2E000C35
:100A4000BB0B0F94BE5522E030E040E050E00F9425
:100A50007B55DA01C901800F911FA11DB11D909333
:100A600099068093980610929706D701C60188567A
:100A7000954CAF4FBF4F8093760690937706A09327
:100A80007806B093790681E0809322022091930644
:100A90003091940640E82931340741F480912402D2
:100AA000882309F4D4C08150809324022A50394409
:100AB00051F580912402882321F0815080932402F3
:100AC00022C084E080932402809196068F5F8093F9
:100AD000960690919506981728F4109296068CE049
:100AE0008093240281E080932202D701C6018856B8
:100AF000954CAF4FBF4F8093760690937706A093A7
:100B00007806B093790680916F0081FB222720F947
:100B100081FF05C080916F008D7F80936F00809171
:100B2000DE0D9091DF0DA091E00DB091E10D22233B
:100B300029F020916F00226020936F003AE0B69573
:100B4000A795979587953A95D1F7009721E0A20749
:100B5000B10520F08FEF9FEFA0E0B0E0969587956C
:100B600020912202211105C030919B063111ECC069
:100B700051C0009741F04091740650917506481796
:100B8000590708F047C080919B06811117C0223099
:100B900008F06DC08091A504811107C081E08093A9
:100BA000A5048CE694E00E949B338CE694E00E94BE
:100BB000D23381E080939A0680939B0683E00E9463
:100BC000A54261E08CE694E00E94FB33E09193063D
:100BD000F0919406199510929A0680919B068111C6
:100BE00052C010928D060E94C82EDC01CB018C19D8
:100BF0009D09AE09BF09009174061091750620E0A9
:100C000030E0081719072A073B0720F49093750670
:100C10008093740680919306909194068951904830
:100C200009F483C08091A00681117FC052C060E0AA
:100C300083EB9FE2BFDD43CEE9D5123009F43FCE0E
:100C400060E086EA9FE2B6DD0E94CC7B38CE8CE085
:100C50008093240280917406909175060197909379
:100C600075068093740681E0809322021FCF2430A2
:100C700030F0243009F08ECF109222028BCF81E029
:100C80008093220287CF8CE694E00E94D63391E0D5
:100C9000811101C090E090939B06992309F4A1CFA4
:100CA0000E94C82EDC01CB018C199D09AE09BF0939
:100CB000C0907406D0907506E12CF12CC816D906A8
:100CC000EA06FB0608F044C090937506809374060C
:100CD0003FC08091760690917706A0917806B091FA
:100CE0007906C81AD90AEA0AFB0AF7FE0E94CC7BE9
:100CF00080919B0681112CC080912202813091F05D
:100D0000833031F51F910F91FF90EF90DF90CF90DE
:100D1000BF90AF909F908F907F906F905F904F901B
:100D20000C943C431092220213C048E9C40E4AE3DB
:100D3000D41EE11CF11CC0927606D0927706E09298
:100D40007806F0927906D4CF009709F437CF13CF05
:100D50001F910F91FF90EF90DF90CF90BF90AF90D9
:100D60009F908F907F906F905F904F90089561E07B
:100D700021DD0C94CC7BCF93DF931F921F92CDB7D4
:100D8000DEB789839A8360DC89819A81F0DF0F90D6
:100D90000F90DF91CF910C940D4380917E0982FDDD
:100DA00005C08091EE16823061F410C080912F0949
:100DB000811103C081E799E002C08FE299E061E010
:100DC000B2CC813031F085E79FE205C089E99FE22E
:100DD00002C08DE89FE26FEFEDCC1092FB161092EF
:100DE000900280917E09806280937E090E94FBAE12
:100DF0000F94594C60E087E69FE2DCDC0C94CC7BDE
:100E00008BE59FE20E94A07C60E08EE49FE2D2DC52
:100E100040E061E080E00E94D16584E49FE20D94AF
:100E20000F3ABBDF1092FB16109290020E943366BD
:100E3000882321F080917E0982FF04C00E94F3AED6
:100E40000D94D24C80E49FE20F940F3AF7CF80913B
:100E50007E0982FF2AC00E943366882319F180919F
:100E6000390790913A07A0913B07B0913C07009752
:100E7000A105B105B9F0BC01CD016D597F4F8F4F70
:100E80009F4F24E630E040E050E00F9459556091C8
:100E900035077091360780913707909138070F9486
:100EA000595501C020E02093A3068091A3068F77B7
:100EB000089589E190E890939406809393060895AD
:100EC00061E0FC0180810E94F8308FEF0C94D9A67C
:100ED000CF93DF93EC018A810E949BA660E088811A
:100EE000DF91CF910C94F8308F929F92AF92BF9286
:100EF000EF92FF920F931F93CF93DF93EC018B013F
:100F00007A010E94C82E4B015C012CE2820E21E086
:100F1000921EA11CB11C0E94B3A68B838F3F61F46B
:100F20000E94C82EDC01CB0188199909AA09BB09C6
:100F3000B7FDF1CF81E10DC08E3F51F4B701C8017B
:100F40000E94BAA60E94B3A60E94B3A611E003C0F5
:100F50008FE0898310E0CE01B3DF812FDF91CF9145
:100F60001F910F91FF90EF90BF90AF909F908F9047
:100F70000895CF92DF92EF92FF926A017B010E9467
:100F8000C82EC60ED71EE81EF91E0E94B3A68F3FBC
:100F900061F00E94C82EDC01CB018C199D09AE09BD
:100FA000BF09B7FDF2CF80E001C081E0FF90EF9074
:100FB000DF90CF900895EF92FF921F93CF93DF932E
:100FC00000D01F92CDB7DEB77C01162F29833A835C
:100FD0004B835C837DDF48E552E060E070E0C70151
:100FE000C8DF812F80640E94D9A68C810E94D9A677
:100FF0008B810E94D9A68A810E94D9A689810E94EC
:10100000D9A6112311F087E801C085E90E94D9A66D
:101010001C3011F40E94B3A610E00E94B3A6F701A1
:10102000838387FF04C01F3F11F01F5FF6CF0F902F
:101030000F900F900F90DF91CF911F91FF90EF9045
:1010400008958F929F92AF92BF92CF92DF92EF92CC
:10105000FF920F931F93CF93DF93EC01162F1C8207
:10106000198248830E94C82E6B017C0120EDC20EBC
:1010700027E0D21EE11CF11CA89561E088810E9446
:10108000F83061E088810E94BC300E94ACA685E007
:101090008A830E949BA60AE08FEF0E94D9A6015086
:1010A000D9F7A89520E030E0A90160E0CE0183DF08
:1010B0008B83813061F00E94C82EDC01CB018C193A
:1010C0009D09AE09BF09B7FDEDCF81E055C0A895D8
:1010D0002AEA31E040E050E068E0CE016CDF853084
:1010E00011F481E009C004E00E94B3A68B83015093
:1010F000D9F78A3A51F482E08C83A8958C818230AA
:1011000081F0812C912C540111C00E94C82EDC0169
:10111000CB018C199D09AE09BF09B7FDD9CF82E07B
:101120002BC0812C912CA12C80E4B82E20E030E043
:10113000A90167E3CE013FDFA501940169E2CE0179
:101140003ADF8B83882361F00E94C82EDC01CB013B
:101150008C199D09AE09BF09B7FDE8CF8AE00CC024
:101160008C818230D1F420E030E0A9016AE3CE0125
:1011700022DF882329F088E08983CE01A1DE16C012
:101180000E94B3A6807C803C11F483E08C830E9493
:10119000B3A60E94B3A60E94B3A6CE0191DE17307B
:1011A00018F41A8381E003C088E1898380E0DF912D
:1011B000CF911F910F91FF90EF90DF90CF90BF9054
:1011C000AF909F908F9008950F931F93CF93DF93CD
:1011D000EC0189018C81833039F089E0440F551F7F
:1011E000661F771F8A95D1F79A01AB0161E1CE01A5
:1011F000E2DE811109C040E052E0B801CE01DF918A
:10120000CF911F910F9170CE84E08983CE0158DE7B
:1012100080E0DF91CF911F910F910895CF93DF93DD
:10122000EC01862FBA010E94DEA68FEF0E94D9A69C
:101230008FEF0E94D9A60E94B3A68B83982F9F712F
:10124000953031F083E18983CE013ADE80E001C040
:1012500081E0DF91CF9108950F931F93CF93DF9398
:10126000EC0189018C81833039F089E0440F551FEE
:10127000661F771F8A95D1F79A01AB0168E1CE010D
:101280009ADE81111EC0A8016EEFCE01C7DF882350
:10129000E1F048E552E060E070E0CE016ADE8823CC
:1012A00071F020E030E0A9016DE0CE0184DE811113
:1012B0000AC00E94B3A6811106C011E007C087E1F1
:1012C00003C086E001C086E1898310E0CE01F8DD2D
:1012D000812FDF91CF911F910F910895CF93DF93CD
:1012E0001F92CDB7DEB72091FD163091FE16CE01CC
:1012F00001962115310519F0821B930B02C0835012
:1013000097410F90DF91CF910895FC012381211126
:101310000C949C9A089589EE96E0F7CF84E097E0CC
:10132000F4CF80911F07811107C00E9447E08823F6
:1013300019F081E080931F07089580917E09847FD2
:101340008B7F80937E09109235071092360710929A
:101350003707109238071092390710923A07109207
:101360003B0710923C071092AA071092E9078EE003
:1013700091E0EAEEF7E0DF019C011D922150304040
:10138000E1F78FEF80932E090895FC0120E03EE203
:10139000DB014C91403241F0283011F4308331961A
:1013A000DB014C91408331962F5F6F5F7F4F2B3075
:1013B00079F7108208952F923F924F925F926F9229
:1013C0007F928F929F92AF92BF92CF92DF92EF92D5
:1013D000FF920F931F93CF93DF93CDB7DEB7C35622
:1013E000D1090FB6F894DEBF0FBECDBF8C015B01F3
:1013F0004A014DB65EB6312C7E0187E5E80EF11C40
:101400009BE1292E4FE259E0BE016F5F7F4FC5017E
:101410000E940C9918160CF005C18C85282F287194
:10142000203109F074C0909134079150923008F443
:101430006EC06DB67EB6BE016F5F7F4FC701A5DF80
:101440000115110521F0F8018081811173C021E09F
:1014500081E090E0F70101900020E9F73197EE1963
:10146000FF09E80FF91F32968DB79EB78E1B9F0BB1
:101470000FB6F8949EBF0FBE8DBFEDB7FEB7319685
:101480006F01211102C0B80102C061EA73E0C60118
:101490000F94885AB701C6010F94725A61EA73E03B
:1014A000C6010F94725A1CAE1FAE21E0A701B50110
:1014B000CE01CC960E94989C81110DC0809134077A
:1014C000811109C00E94D59F84EB91E30E94C79FC0
:1014D000C7010E9471A5FE01FC96DE019196822D46
:1014E00001900D928A95E1F740E050E0BE016F5DFA
:1014F0007F4FC60160DFCE01819607DFCE01CC961B
:1015000004DF0FB6F8947EBE0FBE6DBE7BCF99810F
:10151000992309F487C0953E09F474CF9E3209F4EB
:1015200071CF90912F099E3209F46CCF8A7009F027
:1015300069CF0AC0F80101900020E9F73197CF0187
:10154000801B910B20E086CF81E0203109F080E004
:1015500090917E0980FB94F990937E09811108C0D7
:101560008985873409F04ECF8A858E3709F44ACFB2
:1015700080913407813021F068F08230B9F142CF98
:1015800080913207909133070196909333078093AF
:10159000320738CFBE016F5F7F4F81E799E0F5DEFC
:1015A0000115110511F0680105C081E7C82E89E019
:1015B000D82E08C0F60181916F018823B1F30E94F3
:1015C0001AA5F8CFF60181916F01882319F00E94C6
:1015D0001AA5F8CF80E20E941AA56D8D7E8D8F8DA1
:1015E00098A14AE050E00E9427A60CCFBE016F5F91
:1015F0007F4F81E799E0C9DE8114910441F061E7F2
:1016000079E0C4010F945F5A892B51F40BC0832DEC
:1016100090E020913007309131078217930711F045
:101620003394F0CE0FB6F8945EBE0FBE4DBECD59CA
:10163000DF4F0FB6F894DEBF0FBECDBFDF91CF9165
:101640001F910F91FF90EF90DF90CF90BF90AF90E0
:101650009F908F907F906F905F904F903F902F90D2
:101660000895CF93DF93CDB7DEB76B970FB6F8949D
:10167000DEBF0FBECDBF1092340740E050E0BA018C
:1016800083E199E00E94BB998BE1E3E1F9E0DE019F
:10169000119601900D928A95E1F740E050E0BE016D
:1016A0006F5F7F4F80E090E086DECE0101962DDEF9
:1016B0006B960FB6F894DEBF0FBECDBFDF91CF9112
:1016C00008950F931F93CF93DF93CDB7DEB72D9778
:1016D0000FB6F894DEBF0FBECDBF8091AE07882352
:1016E00091F0BE016F5F7F4F8BEA97E00E942E97CB
:1016F0008E010F5F1F4FF80181918F01882339F010
:101700000E941AA5F8CF8AEA91E30E94C79F8AE057
:101710000E941AA52D960FB6F894DEBF0FBECDBF5E
:10172000DF91CF911F910F910895CF92DF92EF92A9
:10173000FF920F931F93CF93DF93CDB7DEB7EDB634
:10174000FEB6DC010D900020E9F79D01281B390B46
:101750002C5F3F4F4DB75EB7421B530B0FB6F8944B
:101760005EBF0FBE4DBF0DB71EB70F5F1F4F9F93DC
:101770008F9384E691E39F938F931F930F930F941E
:10178000B75A680154E0C50ED11C0F900F900F900E
:101790000F900F900F90F6018081882349F0082E5A
:1017A000000C990B0F94E359F60181936F01F3CF6D
:1017B000C8010F94143A80E691E30F94223A0FB6D1
:1017C000F894FEBE0FBEEDBEDF91CF911F910F9139
:1017D000FF90EF90DF90CF90089580917E0983FF76
:1017E00003C0846080937E09089510924B0C809111
:1017F0007E098F7D8B7F80937E090E9433668823CC
:1018000021F08BEA97E00C949C9A0895EEDF80918A
:101810007E09877F80937E0908950F931F93CF934E
:10182000DF938B01EA01DB016D917C910E942E9781
:10183000D801ED91FC919081888191110EC089367B
:10184000B0F48FE28083F8018081918101969183C9
:10185000808388818F5F88830AC0893680F73196BC
:10186000D801ED93FC9388818F5F8883E1CFDF916E
:10187000CF911F910F9108950F931F93CF93DF93F3
:1018800000D0CDB7DEB79C012F5F3F4F3B832A834B
:101890002FE2FC01208381E0898310E00BE180913D
:1018A000E907181770F4019FC0011124AE014F5FC2
:1018B0005F4FBE016E5F7F4F8651984FAEDF1F5F57
:1018C000EECF89818B3570F4AE014F5F5F4FBE0163
:1018D0006E5F7F4F8BEA97E0A0DF8A819B81019743
:1018E0009B838A83EA81FB8110820F900F900F9077
:1018F000DF91CF911F910F91089580917E0982FF12
:101900001FC088E290E30E94C79F609135077091E5
:10191000360780913707909138074AE050E00E94DF
:101920001CA68FE20E941AA56091390770913A07B0
:1019300080913B0790913C074AE050E00C9427A629
:1019400087E190E30C94C79FEF92FF920F931F9350
:10195000CF93DF938C01FC0101900020E9F73197D0
:10196000EF01C81BD90B1092AB076EE470E00F9427
:101970007D5A7C01009729F4FE013197E00FF11F99
:101980000EC060E270E00F947D5A8C010F5F1F4F14
:101990006AE270E0C7010F947D5AFC0131978DE037
:1019A00081838AE082831382B8018BEA97E00E94E8
:1019B0002B9F8091AB07882361F00E94D89F80E025
:1019C00090E3DF91CF911F910F91FF90EF900C94D6
:1019D000C79FDF91CF911F910F91FF90EF900895D6
:1019E0008BEA97E00E94519A8BEA97E00E949C9ABA
:1019F00080917E098D7F8E7F80937E0910923507BE
:101A000010923607109237071092380781E08093C2
:101A10003C0C08950F931F93CF93DF93CDB7DEB7A0
:101A20006B970FB6F894DEBF0FBECDBF8B0122E0DF
:101A300020933407909331078093300740E050E0C3
:101A4000BA0188EF98E00E94BB998BE1E8EFF8E0DB
:101A5000DE01119601900D928A95E1F7A801BE0171
:101A60006F5F7F4F80E090E0A6DCCE0101964DDCF9
:101A70006B960FB6F894DEBF0FBECDBFDF91CF914E
:101A80001F910F910895CF93DF93CDB7DEB76B977A
:101A90000FB6F894DEBF0FBECDBF81E08093340750
:101AA000109233071092320740E050E0BA0188EFFD
:101AB00098E00E94BB998BE1E8EFF8E0DE01119617
:101AC00001900D928A95E1F740E050E0BE016F5F12
:101AD0007F4F80E090E06FDCCE01019616DC8091B4
:101AE0003207909133076B960FB6F894DEBF0FBEA6
:101AF000CDBFDF91CF9108952F923F924F925F9289
:101B00006F927F928F929F92AF92BF92CF92DF920D
:101B1000EF92FF920F931F93CF93DF9300D01F920A
:101B2000CDB7DEB77C018B01342E2DB73EB73C8399
:101B30002B838091280781110BC01092040710920B
:101B4000070781E0809328078EE899E80E94B33A5E
:101B50008091200781110BC01092E9061092EC06CB
:101B600081E0809320078BE899E80E94B33AF8015E
:101B700080818F3251F483E199E0F7019183808372
:101B80001092E9070F5F1F4F05C088EF98E0F7013B
:101B900091838083F7010190F081E02DFA83E9833E
:101BA00024E0A22E27E0B22E3BE1232E01151105E1
:101BB00009F47FC04DB65EB66FE270E0C8010F94C5
:101BC0007D5A3C010817190708F073C06C01C01A50
:101BD000D10ADD24C60101962DB73EB7281B390B6B
:101BE0000FB6F8943EBF0FBE2DBF8DB79EB70196BE
:101BF0004C01A601B8010F949D5AF401EC0DFD1D96
:101C00001082332019F0C4010E9471A5F701608190
